:020000040800F2
:10400000A84D002065410008B5A7000815770008F5
:1040100041930008855100080119010800000000C3
:1040200000000000000000000000000019CA0008A5
:10403000D1540008000000007B41000869EF00082F
:104040007F4100087F4100087F4100087F41000850
:104050007F4100087F4100087F4100087F41000840
:104060007F4100087F4100087F4100087F41000830
:10407000B55400087F410008B75400087F4100088C
:104080007F4100087F4100087F4100087F41000810
:104090007F4100087F4100087F4100087D560008ED
:1040A0007F4100087F4100087F4100087F410008F0
:1040B0007F4100087F4100087F4100087F410008E0
:1040C0007F4100087F4100087F4100087F410008D0
:1040D0007F410008690D0108710D0108790D010883
:1040E0007F4100087F4100087F4100080000000078
:1040F00000000000000000000000000000000000C0
:1041000000000000000000007F4100087F4100081F
:104110007F4100087F4100087F4100087F4100087F
:104120007F4100087F4100087F4100087F4100086F
:104130007F4100087F4100087F4100087F4100085F
:104140007F4100087F4100087F4100087F4100084F
:10415000DFF80CD000F0B6FB00480047ED2A01085C
:10416000A84D00200648804706480047FEE7FEE7C6
:10417000FEE7FEE7FEE7FEE7FEE7FEE7FEE7FEE717
:1041800079EF00085141000840EA01039B0703D082
:1041900009E008C9121F08C0042AFAD203E011F886
:1041A000013B00F8013B521EF9D27047D2B201E048
:1041B00000F8012B491EFBD270470022F6E710B52C
:1041C00013460A4604461946FFF7F0FF204610BD85
:1041D000421E12F8013F002BFBD111F8013B02F8FF
:1041E000013B002BF9D1704730B505462A460B46F6
:1041F00012F8010B13F8014B08B1A042F8D01CB122
:10420000002802D06D1CF1E7284630BD10B50446E9
:1042100004E00B7800F8013B03B1491C521EF8D2B0
:10422000204610BD421C10F8011B0029FBD1801A4A
:10423000704710B5002200E0521C835C8C5CA342E6
:1042400001D1002BF8D1D8B2E1B2401A10BD30B57F
:1042500004460020034600E05B1C934203D2E05C6E
:10426000CD5C401BF8D030BD034611F8012B00F89F
:10427000012B002AF9D11846704730B505460020B9
:10428000034600E05B1C934205D2EC5CC85C201A3C
:1042900001D1002CF6D130BD2DE9F04791460F46F3
:1042A00080460446002614F8015B2DB100F05AFA4E
:1042B0000068405DC007F6D12B2D02D02D2D18D0FF
:1042C000641E4A463946204600F050FA27B1396844
:1042D000A14201D1C7F8008071054FF002040BD54F
:1042E0004042002803DD0DF0EFFC0460A007BDE8AC
:1042F000F08746F48066E4E70028F8DA0DF0E4FC85
:1043000004606FF00040F2E770B506460DF0DCFC8B
:10431000046805460A2200213046FFF7BDFF2C60E5
:1043200070BD70B506460DF0CFFC046805460A2244
:1043300000213046FFF7B0FF2C6070BD2DE9FE4F25
:10434000804681EA0300C00F0C46009021F0004136
:1043500023F00045B8EB0200A94105D240462146B2
:1043600090461C460B46024623F00040104347D0BF
:10437000270DC7F30A00C3F30A510290401A0190B7
:1043800040286BDAC3F3130040F4801B0098924678
:1043900020B10023D2EB030A63EB0B0B01985946C3
:1043A000C0F14002504600F0ACF906460D465046BA
:1043B0005946019A00F0C4F910EB0800614100244D
:1043C00087EA115284EAE7731A4340D0009A62B335
:1043D000019A012A4FEA075215DC001B61EB02012A
:1043E0004FF0004202EA0752CDE90042001C41F5BD
:1043F000801132462B4600F017FA03B0BDE8F08F6B
:1044000040462146F9E7001B61EB0201001C41F523
:10441000801300185B412018A2F5001747EB030139
:1044200040EAD570B6196D4111E06D084FEA3606C5
:1044300045EAC0754FEA0752001B61EB0201001C00
:1044400041F5801149084FEA3000001951413246C8
:104450002B4603B0BDE8F04F00F0D7B90098012219
:1044600040000023D0EB020263EBE073009821468A
:104470004FEAE074B8EB000061EB0401E9E783F078
:1044800000435BE781F0004158E72DE9FE4F81EAE8
:10449000030404F0004421F0004100944FF0000BAD
:1044A00023F0004350EA01045ED052EA03045BD0DB
:1044B000C3F30A54C1F30A552C44A4F2F334019413
:1044C000A0FB0254C1F3130141F48011C3F31303A1
:1044D00043F4801301FB024400FB034E840A970A55
:1044E00044EA815447EA8357A4FB076802958D0A82
:1044F00005FB07854FEA932C04FB0C542705029D0E
:104500004FEA065847EA1637B5EB08056EEB070C7D
:10451000870E920E47EA811742EA8312A7FB020137
:10452000B6EB0B0164EB00042B0D43EA0C335E1871
:1045300044EB1C50DA465146E7FB0201C5F3130475
:104540004FEA0B3343EA14534FEA0432019C43EA27
:104550000603A4F10C040294009CCDE900B400F021
:1045600063F903B0BDE8F08F00200146F9E72DE9BB
:10457000F04D81EA030404F0004B21F0004514469D
:104580004FF0000A23F0004150EA050220D054EA1F
:1045900001021DD0C5F30A570246C5F31303C1F348
:1045A0001300C1F30A5640F4801543F48013A7EBBF
:1045B0000608101BD64608F2FD3873EB050002D33F
:1045C00008F1010801E092185B41B8F1000F03DA2D
:1045D00000200146BDE8F08D00204FF48011064612
:1045E00084460EE0171B73EB050705D3121B63EB24
:1045F000050306434CEA010C49084FEA30009218C3
:104600005B4150EA0107EDD152EA030012D082EA81
:10461000040083EA0501084305D0101BAB4106D214
:104620000122002306E000224FF0004302E06FF079
:10463000010253101AEB06004CEB085110EB0A0074
:1046400041EB0B01BDE8F04D00F0DFB80EB5C10F36
:1046500080EAE0700844CA07002140F233438DE845
:104660000E000A460B4600F0DFF803B000BDC1F3B0
:104670000A5210B5C1F3130140F2FF3341F4801127
:104680009A4201DA002010BD40F233439A42A2F26E
:10469000334203DC524200F043F810BD904010BD9D
:1046A0002DE9F05F0546002092469B468846064667
:1046B000814640241BE0284641464746224600F0FA
:1046C0002FF853465A46C01A914110D31146184646
:1046D000224600F016F82D1A67EB01084F462246D5
:1046E0000120002100F00DF817EB00094E41201EBB
:1046F000A4F10104DFDC484631462A464346BDE8C2
:10470000F09F202A04DB203A00FA02F100207047D3
:104710009140C2F1200320FA03F3194390407047FF
:10472000202A04DB203A21FA02F00021704721FA06
:1047300002F3D040C2F1200291400843194670476D
:10474000202A06DBCB17203A41FA02F043EAE07355
:1047500006E041FA02F3D040C2F120029140084342
:104760001946704700487047685301082DE9F05F0B
:1047700082460078002715468B460AF10104B946A7
:10478000302801D09DB113E014F8010B01277828DF
:1047900003D0582801D045B10AE00DB1102D07D142
:1047A0000027102514F8010B02E0082500E00A2577
:1047B0000026B0460EE005FB080005FB06F10127C8
:1047C00001EB10461FFA80F8B6F5803F00D3B946DA
:1047D00014F8010B294600F087F80028EBDABBF14A
:1047E000000F05D00FB1641E00E05446CBF8004026
:1047F000B9F1000F06D00DF067FA02210160C81E62
:10480000BDE8F09F48EA0640FAE710B5141E73F1C0
:10481000000408DA401C41F1000192185B411A4380
:1048200001D120F0010010BD2DE9F04D92469B46CC
:1048300011B1B1FA81F202E0B0FA80F22032904672
:10484000FFF75FFF04460F4640EA0A0041EA0B010A
:1048500053465A46084313D0114653EA010019D073
:10486000C8F140025046FFF75BFF05460E46504632
:1048700059464246FFF745FF084305D0012004E0B2
:1048800020463946BDE8F08D0020054346EAE07633
:104890002C4337430A986305E40AA0EB0800002282
:1048A000FD0A44EA47540A3002D500200146E9E7F0
:1048B000010510196941DDE9084500196941BDE8A4
:1048C000F04DA2E7064C074D06E0E06840F001031A
:1048D00094E8070098471034AC42F6D3FFF73CFC4D
:1048E00014570108345701083A2800D2303820F014
:1048F0002002412A01D3A2F13700884201D34FF0B0
:10490000FF30704770B58C1810F8015B15F0070385
:1049100001D110F8013B2A1106D110F8012B03E058
:1049200010F8016B01F8016B5B1EF9D12B0705D460
:104930000023521E0DD401F8013BFAE710F8013BA9
:10494000CB1A921C03E013F8015B01F8015B521EC5
:10495000F9D5A142D8D3002070BD000000B587B0C2
:104960000121480207F07AFC0121082007F076FCBB
:104970000120ADF8040048208DF8070001A919486E
:1049800001F06EFA642000F0A4FD00208DF807000D
:1049900001A9144801F064FAC82000F09AFD002033
:1049A00002908DF80C008DF80D004FF460200490FB
:1049B0000020059001208DF8180002A90A4800F097
:1049C0002DF8002301221946074800F04FF8012175
:1049D000054800F00BF80121034800F0A3F807B0E8
:1049E00000BD0000000801400024014021B18268A0
:1049F00042F00102826003E0826822F001028260DC
:104A000070470146C86C80B27047024600201368A8
:104A10000B400BB1012000E00020704730B502468A
:104A20000020002350680F4C20400D790C6844EAA8
:104A300005242043506090680B4C2040D1E902547B
:104A40002C434D7944EA450420439060D06A20F419
:104A500070000C7C641EE4B2234340EA0350D06231
:104A600030BD0000FFFEF0FFFDF7F1FFF0B504469A
:104A70000D4600200021092D11DDE068A5F10A0690
:104A800006EB4607072606FA07F18843A5F10A0652
:104A900006EB460603FA06F10843E0600CE02069E5
:104AA00005EB4507072606FA07F1884305EB45069F
:104AB00003FA06F108432061072A0FDA606B561EDD
:104AC00006EB86071F2606FA07F18843561E06EBFB
:104AD000860605FA06F10843606322E00D2A0FDA24
:104AE000206BD61F06EB86071F2606FA07F18843C0
:104AF000D61F06EB860605FA06F10843206310E090
:104B0000E06AA2F10D0606EB86071F2606FA07F1FA
:104B10008843A2F10D0606EB860605FA06F1084366
:104B2000E062F0BD21B1826842F4A002826003E03D
:104B3000826822F4A00282607047F0B504460A46FB
:104B400025460CE003F00F071E11304600F02EF84A
:104B500002F8010B384600F029F802F8010B15F8AD
:104B6000013B002BEED100201070F0BD2DE9F0418B
:104B700004460A4625464FF0040810E015F8013BAC
:104B800003F00F061F11384600F010F802F8010B71
:104B9000304600F00BF802F8010BA8F10108B8F15B
:104BA000000FEBD100201070BDE8F081002805DB7C
:104BB000092803DC00F13001C8B208E00A2805DB4F
:104BC0000F2803DC00F15701C8B200E0FF20704756
:104BD0002DE9F843074688463846FFF723FB06468B
:104BE000304606EBD0714910A6EB410111B100200F
:104BF000BDE8F883002546E017F815008DF80000A1
:104C00006800401C385C8DF8010000242DE01DF880
:104C1000040030280ADB1DF80400392806DC1DF8E2
:104C200004003038C0B20DF804001CE01DF8040088
:104C300061280ADB1DF80400662806DC1DF8040064
:104C40005738C0B20DF804000DE01DF804004128EB
:104C500009DB1DF80400462805DC1DF80400373880
:104C6000C0B20DF80400601CC4B2022CCFDB9DF86A
:104C70000000F02101EA00109DF80110084308F837
:104C80000500681CC5B206EBD671B5EB610FB3DB4E
:104C90002846ADE72DE9F041A0B0044650229A49DC
:104CA0000CA8FFF771FA99A1204605F00DFC80B918
:104CB000E07B2C2806D004F10F00FFF725FB964976
:104CC00008601DE104F11000FFF71EFB9249086027
:104CD00016E192A1204605F0F7FB30B9E01DFFF781
:104CE00013FB80460CF096FD0AE18EA1204605F0EC
:104CF000EBFB30B9A01DFFF707FB80460CF08AFDE7
:104D0000FEE08AA1204605F0DFFB90B904F10B001C
:104D1000FFF7FAFA88490860084688A22821036844
:104D200001A80CF0A9FF012201A9002009F044FF0D
:104D3000E6E088A1204605F0C7FB50B9607A31282B
:104D400003D1012086490870DAE002208449087006
:104D5000D6E084A1204605F0B7FB28B9617BE07A54
:104D600000220FF0ADF8CBE081A1204605F0ACFBAE
:104D700088BB0120034667A20D210090204600F069
:104D800023FF0546B0F1FF3F9BD06019FFF7BCFA47
:104D9000C6B20120034679A20D210090204600F002
:104DA00013FF0546B0F1FF3F8BD06019FFF7ACFA57
:104DB00087B20220012371A20D210090204600F04D
:104DC00003FF0546B0F1FF3F8ED061193A463046E9
:104DD0000FF01EF894E0FFE769A1204605F074FB90
:104DE00028B9E17A607A00220FF06AF888E067A1BA
:104DF000204605F069FB28B9A07A012200210FF0B6
:104E00005FF87DE064A1204605F05EFB002877D0C6
:104E100063A1204605F058FB002846D1A079202840
:104E200003D1E0798DF82C0002E0A0798DF82C00F8
:104E30009DF82C305CA250210CA80CF01DFF9DF8B1
:104E40002C0030380A2824D2DFE800F005230A0FAE
:104E500014192323231E57A10CA8FFF7B9F91DE04D
:104E600057A10CA8FFF7B4F918E058A10CA8FFF758
:104E7000AFF913E056A10CA8FFF7AAF90EE058A16C
:104E80000CA8FFF7A5F909E057A10CA8FFF7A0F9B6
:104E900004E056A10CA8FFF79BF900BF00BF012258
:104EA0000CA9002009F088FE2AE052A1204605F056
:104EB0000BFB30B90120524981F8B106002008727D
:104EC0001EE050A1204605F0FFFAC8B14FA12046D0
:104ED00005F0FAFAA0B14FA1204605F0F5FA78B135
:104EE0004EA1204605F0F0FA10B90DF085F907E063
:104EF0004DA1204605F0E8FA10B9601D01F0B4FE9E
:104F000020B0BDE8F0810000E04101085E53595334
:104F1000494E464F3A000000C80200202B4343533D
:104F2000513A00002B4353513A0000002B4D4F449F
:104F30004F445245583A0000C40200204D6F646F40
:104F4000647265785F4E657476616C75653D256445
:104F5000000000002B504F435F5050503A000000BB
:104F6000D50100202B5443505354415455533A001B
:104F70002B544350524543563A0000002C00000089
:104F80002B5443504F50454E3A0000002B54435091
:104F9000434C4F53453A00002B43434C4B3A0000DF
:104FA0005E4D4F44453A00005B4D6F6465202563BC
:104FB0005D0000004E6F2073657276657200000020
:104FC00043444D41204D6F646500000047534D0040
:104FD00054442D5343444D412F4556444F00000047
:104FE0005743444D410000004C544500556E6B6ED4
:104FF0006F7700002B504F433A53544152540000F6
:10500000D00700202B474749503A00002B47504912
:10501000503A00002B464F54413A00002B504F436A
:105020003A57414B455550002B5544503A0000002B
:105030002DE9F04707468846DFF8D890B8F1000F11
:1050400033D1B86A00F58055334E002411E04FF497
:105050008062294648460EF0C9FC4FF48062314612
:1050600048460EF039FD05F5806506F58066601C42
:10507000C4B2042CEBDBBD6A4FF4FF16002411E030
:105080004FF48062294648460EF0B0FC4FF480622F
:10509000314648460EF020FD05F5806506F5806630
:1050A000601CC4B2042CEBDB32E01B4DB86A00F587
:1050B0008056002411E04FF48062294648460EF0E5
:1050C00095FC4FF48062314648460EF005FD05F52B
:1050D000806506F58066601CC4B2042CEBDB4FF4DF
:1050E000FF15BE6A002411E04FF48062294648464D
:1050F0000EF07CFC4FF48062314648460EF0ECFC2A
:1051000005F5806506F58066601CC4B2042CEBDBF7
:10511000BDE8F087A837002000F01F0010B501F0AF
:1051200083FE0446002C01DD09480460094800782C
:10513000401CC0B207490870032800DC10BD0020E5
:10514000044908700248006800F048F800BFF5E71D
:10515000D8010020E101002008B50121052007F059
:105160007DF80220ADF8000018208DF80300032020
:105170008DF802006946024800F072FE08BD00008A
:105180000008014000BFFEE77047000010B5002096
:105190000B4908700B48006844F63821884208DD46
:1051A000012007490870012207A1002009F004FD31
:1051B00004E0012206A1002009F0FEFC10BD000061
:1051C0009100002078000020706F632D6F776E00D3
:1051D000706F632D7869616E0000000010B50446A1
:1051E000B4F5A57F13DA012214A1002009F0E4FC34
:1051F00018484079012801D10CF0BCFF0020154966
:10520000487104201449486109F08EFC14E0B4F59B
:10521000AA7F0EDA11480078401CC0B20F4908700E
:105220001E2809DD0020087001220DA109F0C4FC30
:1052300002E000200949087010BD00005662617448
:10524000206C6F772173687574646F776E206E6F52
:1052500077210000D007002000100140E00100206D
:10526000436861726765206261742121000000005B
:1052700000B585B00F48007820B1012807D002287A
:105280000FD109E00CA168460CF00AFD0BE00DA15E
:1052900068460CF005FD06E00DA168460CF000FD27
:1052A00001E005B000BD00BF684600F09BFD00BFF7
:1052B000F7E70000ED000020455652435F48414C9F
:1052C00046000000414D524E422D31323200000066
:1052D000455652435F46554C4C00000010B50446FD
:1052E00024B1012C36D0022C33D167E0012258A121
:1052F000002009F061FC59480470002240F2255159
:1053000057480BF0A1FD012240F2244154480BF014
:105310009BFD0122802152480BF056FD01224021C5
:105320004F480BF051FD002240F225514D480BF043
:105330008BFD012240F224414A480BF085FD0022FA
:10534000802148480BF040FD0122402145480BF0E8
:105350003BFD7AE0012244A1002009F02DFC3F48EA
:105360000470012240F225513D480BF06DFD0022F2
:1053700040F224413A480BF067FD00228021384872
:105380000BF022FD0122402135480BF01DFD0122CA
:1053900040F2255137480BF057FD002240F22441DE
:1053A00034480BF051FD0022802132480BF00CFDF7
:1053B000002240212F480BF007FD46E001222EA1DC
:1053C000002009F0F9FB25480470012240F2255124
:1053D00023480BF039FD002240F2244120480BF015
:1053E00033FD002280211E480BF0EEFC00224021FC
:1053F0001B480BF0E9FC0021234800F05DF8002178
:105400002148143000F058F8012240F22551154887
:105410000BF01AFD002240F2244112480BF014FD5B
:10542000002280210F480BF0CFFC002240210D48C4
:105430000BF0CAFC00211448283000F03DF8002190
:1054400011483C3000F038F800BF00BF10BD00002C
:10545000434F4D3C2D2D3E4D435521002C00002047
:105460000038014000440040434F4D3C2D2D3E4745
:105470005053210000480040434F4D3C2D2D3E4DE0
:105480006F64656D210000004400024010B50648BD
:10549000008838B1054805F021FF00200249088046
:1054A0000349088010BD000030000020BC0300202C
:1054B0002E0000207047704721B1026842F00102BF
:1054C000026004E002684FF6FE731A400260704703
:1054D000704710B54FF42F73002109E0002201E05E
:1054E00000BF521C03F59654A242F9D34C1CA1B242
:1054F0008142F3DB10BD01461CE000BF00BF00BFCE
:1055000000BF00BF00BF00BF00BF00BF00BF00BFA3
:1055100000BF00BF00BF00BF00BF00BF00BF00BF93
:1055200000BF00BF00BF00BF00BF00BF00BF00BF83
:1055300000BF00BF0A1EA1F1010399B2DDD170477F
:1055400070B586B002AC02AE4A48C1884A4800EB4A
:105550008100006800901022204600990EF046FA63
:105560009DF80900012812D143481638808870B18F
:10557000414816388088401E3F49163988800846C1
:10558000808820B90846007820F0010008703A4869
:105590001638408830B1384816384088401E3649A1
:1055A00016394880344816380078C0F3800060B15E
:1055B0003148163800788008401E2F49163909787E
:1055C00060F382012C48163801702B481638D0F849
:1055D0000600009988420FD005AD049800F10C0137
:1055E000042228460EF078FA04AD059800F108016F
:1055F000042228460EF070FA00200190012201A832
:1056000000990EF069FA1C481638D0F80600009987
:10561000884228D018481638D0F8061010222046A4
:105620000EF0E4F914481638D0F8060000F108012D
:10563000042268460EF050FA049800F10C0104228E
:1056400068460EF049FA009800F10801042204A807
:105650000EF042FA009800F10C01042206481038BE
:105660000EF03AFA04E0044916390598C1F806002C
:1056700006B070BD702800205625002010B54FF4EC
:10568000007000F01DF801280DD1074800780128AE
:1056900005D10420054908610120054908704FF42F
:1056A000007000F007F810BD9502002000100140C6
:1056B0007F02002001490860704700001404014087
:1056C00001460020034A12680A400AB1012000E0A6
:1056D0000020704714040140002123498279002AE8
:1056E0003AD00A46126803689A430B461A600A1DAC
:1056F000126803689A430B1D1A60027911440A6804
:1057000003681A430A60184A0832126803689A4309
:10571000154B08331A601A1D126803689A43124B1E
:105720000C331A604279102A0ED11A1F12680368CE
:105730001A430D4B08331A601A1D126803681A4386
:10574000094B0C331A600DE00749427911440A688D
:1057500003681A430A6005E0027911440A68036885
:105760009A430A60704700000004014010B50C2401
:1057700001200D49087000200C49087009F0D6FA84
:1057800009F0D4FA09F0D2FA01200BF05BFC0120F9
:1057900002F0B6FF082007F0D1FE012204A100208C
:1057A00009F00AFA10BD00008802002092020020D1
:1057B0005B456E74657254784D6F64655D000000E2
:1057C00030B5044604254FF4302000F06FF805464C
:1057D000042D17D10C48006940F002000A49086105
:1057E00008464461006940F0400008614FF43020F1
:1057F00000F05CF805460448006941F6FD71084078
:1058000001490861284630BD0020024004200B49B0
:10581000C96801F0010109B101200EE00749C9681A
:1058200001F0040109B1022007E00449C96801F050
:10583000100109B1032000E004207047002002405D
:105840000348006940F0800001490861704700008A
:105850000020024070B504460D460426F00200F018
:1058600025F80646042E11D10948006940F00100D0
:10587000074908612580F00200F018F80646044840
:10588000006941F6FE71084001490861304670BD6B
:1058900000200240024803494860034848607047BE
:1058A0002301674500200240AB89EFCD00B50246D9
:1058B0000423FFF7ABFF034603E0FFF7A7FF034610
:1058C000521E012B01D1002AF7D102B90523184637
:1058D00000BD10B500F002F810BD00002DE9F04148
:1058E0008CB04FF000084FF40A617A48FEF765FC6F
:1058F0000024002642E03022314668460EF076F859
:1059000075490B98884232D104EB440101EBC40283
:105910007049083101EB820014226946FEF734FC1D
:1059200004EB440101EBC4026A49083101EB820136
:1059300001F11400102205A9FEF726FC04EB440037
:1059400000EBC4026348083000EB82000999416211
:1059500004EB440000EBC4015E48083000EB81001A
:105960008662641C0A9808B10A9E07E009E05B4958
:105970000B98884200D104E006F5805658488642CC
:10598000B9DB00BF53484460012C06DA55A00CF087
:1059900063F901200CB0BDE8F08156484D4908601C
:1059A00004254968491E01EB410202EBC102494945
:1059B000083101EB820050A1FEF73BFC70B945496C
:1059C0004968491E01EB410202EBC102414908311D
:1059D00001EB8201886A0CF0EBFD054604274FF4C9
:1059E000FF100CF0E5FD07462DB943A144A00CF0D3
:1059F00033F90020CEE7002F64D1042D05D13EA15C
:105A000041A00CF029F9002604E03BA143A00CF0D2
:105A100023F9012630224FF4FF1168460DF0E6FF0E
:105A200004EB440101EBC4022A49083101EB820076
:105A300014226946FEF7A8FB04EB440101EBC40203
:105A40002449083101EB820101F11400102205A95B
:105A5000FEF79AFB04EB440000EBC4021D4808303B
:105A600000EB820009994162601E801B00EB40023E
:105A700002EBC0021748083000EB8200816A302236
:105A800068460DF0B3FF04EB440000EBC40211487C
:105A9000083000EB82000A998162A11B01EB4102F0
:105AA00002EBC1020B49083101EB82000121FFF733
:105AB000BFFA042D04D107484068401C05494860DE
:105AC000002067E73B462A460BA11AA00CF0C4F859
:105AD00002205FE7082F0020311B200812EFCDAB1A
:105AE000FFDF1F004E6F207265732066696C65735F
:105AF0000D0A0000F8DEBC8A7379732E696E6900A6
:105B00002573206F6B0D0A002573206C6F73742C46
:105B1000207265636F7665720D0A00002573206937
:105B20006E76616C69642C207265636F7665720DA8
:105B30000A0000002573206572726F722C20737446
:105B4000617475733A25642C25640D0A0000000009
:105B50002DE9F04F0146C1F3074CC1F3072801F0CE
:105B6000FF09DFF85CA00020002224E09300DFF8AA
:105B700054B01BF8035003F1010E1BF80E6003F143
:105B8000020E1BF80E40A9EB0505002D00DA6D4250
:105B9000A8EB0606002E00DA7642ACEB0404002CDB
:105BA00000DA644205EB060B0BEB0407574501DAFC
:105BB000BA461046521CFF2AD8DDBDE8F08F00001F
:105BC0003F420F00082B00202DE9F04704460E4607
:105BD00017461D46DDF820A04FF00008C14615E02D
:105BE0002A4639462046FEF732FB50B909F101003A
:105BF00000F0FF09D14504D108EB050000B2BDE873
:105C0000F087641C08F101001FFA80F82078B04288
:105C1000E6D14FF0FF30F2E710B501F029FE32482F
:105C2000007800B910BD31484078F0B12F480078B5
:105C3000A8B92F480078C0EB001084002B48408999
:105C4000401C80B229494881A0421BDD00204881C8
:105C5000012228A108F0B0FF06F03CFD12E0002070
:105C6000224948812A4908700CE020484089401C9C
:105C700080B21E494881B0F5616F03DD0020488184
:105C800006F028FD19484079012816D11748007AF6
:105C900010B900201F4908701448007A401CC0B297
:105CA00012490872282808DD0120087201221AA171
:105CB000002008F081FF06F00DFD1F48007800F07D
:105CC000010000280DDD1C484078401CC0B21A4974
:105CD00048700A2805DD0020487000F027FA0BF014
:105CE00069FC00BF9EE7000092020020D007002060
:105CF0007C020020506F634C6F737454696D656F44
:105D00007574215265736574204D6F64656D210053
:105D1000890200208A0200204D6F64656D52656320
:105D20007654696D656F7574215265736574204D85
:105D30006F64656D21000000C0220020F0B585B0C1
:105D400054239F222C21002001F002FA012042233B
:105D50008022322100901D2001F06FFA002520489A
:105D6000D0F8067001AE00242CE0102239463046EF
:105D70000DF03CFE9DF80400012807D100208DF8AD
:105D800004000122394630460DF0A6FE049F0A2089
:105D900094FBF0F100FB114008B901F069FD0A2005
:105DA00094FBF0F100FB114050B9012005F11D02F8
:105DB000034640210090342001F06BFA681CC5B204
:105DC000601C84B2B4F57A7FCFDB002004494880A0
:105DD00088800846007820F00100087005B0F0BD0A
:105DE00040250020F8B5054601222946002008F08C
:105DF000E3FE2846FEF716FAA021A1EBC0004608F4
:105E0000402421461023A022002001F05DF900204B
:105E100021460090B0B201232A4601F033FCF8BDC0
:105E200030B500228B071C0F0F2303FA04F20B4B33
:105E30008C1053F824309343084C8D1044F82530CF
:105E400023468C1053F824308C07240F00FA04F4F6
:105E50002343024C8D1044F8253030BD080001402A
:105E60002DE9F041024600250026002000230024F1
:105E7000002791F803C00CF00F0591F803C00CF057
:105E8000100CBCF1000F03D091F802C04CEA0505DC
:105E900091F800C0BCF1000F31D0146800202BE055
:105EA0004FF0010C0CFA00F3B1F800C00CEA030645
:105EB0009E4220D183004FF00F0C0CFA03F7BC4335
:105EC00005FA03FC4CEA040491F803C0BCF1280F66
:105ED00006D14FF0010C0CFA00FCC2F814C00AE025
:105EE00091F803C0BCF1480F05D14FF0010C0CFA3A
:105EF00000FCC2F810C0401C0828D1D31460B1F8CF
:105F000000C0BCF1FF0F34DD546800202EE000F12A
:105F1000080C4FF0010808FA0CF3B1F800C00CEAC5
:105F200003069E4221D183004FF00F0C0CFA03F7B9
:105F3000BC4305FA03FC4CEA040491F803C0BCF12D
:105F4000280F05D100F1080C08FA0CF8C2F81480EB
:105F500091F803C0BCF1480F07D100F1080C4FF0D5
:105F6000010808FA0CF8C2F81080401C0828CED3AB
:105F70005460BDE8F0810000F0B50A46002300241B
:105F80000021002500F00046B6F1004F02D11D4E61
:105F9000F16901E01B4E7168C0F3034583B200F460
:105FA0004016B6F5401F08D121F07061154E766895
:105FB00026F07066134F7E6012E000F48016B6F58E
:105FC000801F06D1032606FA05F4A14341F0706153
:105FD00006E0460D360103FA06F6B14341F0706162
:105FE00022B1460D360103FA06F6314300F00046B1
:105FF000B6F1004F02D1034EF16101E0014E716034
:10600000F0BD0000000001400246002093680B40F4
:106010000BB1012000E00020704741617047016131
:106020007047000008B53348007800B908BD314812
:10603000007801282BD110208DF8030003208DF863
:1060400002004FF40070ADF8000069462A48FFF7DF
:1060500007FF012229A1002008F0AEFD4FF40070D7
:10606000254908612848007820F001002649087079
:106070000846007820F002000870002048703221A5
:1060800022480DF0EFFF02201A4908702FE019484E
:106090000078022810D11D480DF0CCFF38B34FF422
:1060A000007015494861012219A1002008F084FD03
:1060B0000020104908701AE00E4800780A2816D10E
:1060C0004FF400700C490861012215A1002008F06E
:1060D00073FD0D48007820F001000B490870084658
:1060E000007820F00200087000200249087000BF0C
:1060F0009CE70000C00100200010014047505320E1
:10610000446F776E2E2E2E00C0220020C401002086
:1061100047505320537461727420446F6E650000C1
:1061200047505320446F776E000000000120014962
:1061300008707047C001002010B51548007802288B
:1061400000D110BD134800681349884217D1104888
:10615000007840B90020114908700D480078401CB3
:106160000B49087012E00D48007803280EDBFFF79A
:10617000FDFA07480078401C0549087006E004480D
:106180000078012802D100200149087000BFD8E73B
:106190008B020020400000202A04B40047000020A9
:1061A0002DE9F04194B004466079382874D1A07983
:1061B000302871D104F11D00FEF734F8801EC6B2FC
:1061C000482E00DB4826324604F11D0101A8FDF7E8
:1061D000DBFF002001A9885560771022694604F191
:1061E0001900FEF759F887B2002060761022694640
:1061F00004F11100FEF750F8804600206074102270
:10620000694604F10D00FEF747F885B21E2D03DD47
:10621000012014B0BDE8F0811DB901201F490867B5
:1062200004E01E48006F401C1C49086705EB450050
:1062300000EBC5011A4840F8218005EB450000EB52
:10624000C501174800EB810087809DF8040090B9D4
:10625000202105EB450000EBC502114800EB820050
:106260008171002105EB450000EBC5020C4800EBF5
:106270008200C1710AE005EB450000EBC502084849
:1062800000EB8200811D01A808F08EFD012003496A
:1062900081F86D00BDE7FFE70020BAE7D0070020D6
:1062A0004C0900200146024850F8210070470000C8
:1062B000080100202DE9F04F8BB080468B469146B7
:1062C0003448834503D200200BB0BDE8F08F484628
:1062D000FDF7A8FF07460E2F07D00F2F05D04B461E
:1062E0002DA2102108A80BF0C7FC5B462CA20C21A4
:1062F00008A80BF0C1FC08A8FDF794FF009000254A
:10630000A7F10A0405E019F8040004A948556D1C1A
:10631000641CBC42F7DB0026B246002407E008A854
:10632000005D464004A8005D80EA0A0A641C0A2C4D
:10633000F5DB86EA0A061C4810F806A000240CE0EB
:1063400008A8005D80EA0A0604A8005D704001A963
:106350000855154810F806A0641C0A2CF0DB00252F
:1063600004240FE001A8005D0A2190FBF1F201FB7B
:10637000120008F8050018F80500303008F805008C
:106380006D1C641C0A2CEDDB002088F8060001203F
:106390009AE700002058F208253031356C7500006E
:1063A000253031306C750000A84001082DE9F14F0F
:1063B000A2B0002017909A488069000E8DF81C004A
:1063C00097488069000C8DF81D009548008B000AE5
:1063D0008DF81E009248007E8DF81F00904840699D
:1063E000000E8DF818008E484069000C8DF81900D9
:1063F0008B48808A000A8DF81A008948007D8DF844
:106400001B0018A907A8FEF7B1FB00201690002476
:1064100004E018A8005D16A90855641C032CF8DBDD
:1064200016A8FDF771FF82460020139014900024F7
:1064300005E018A9E01C085C13A90855641C062C8B
:10644000F7DB13A8FDF760FF83464FF47A709BFBE0
:10645000F0F00590FEF7FAF8CDE90E010022714B3D
:10646000DDE90E01FEF783F8CDE90E014FF47A70F5
:106470009BFBF0F100FB11B0C0EB00108000059019
:10648000FEF7E4F8CDE90C010022674BDDE90C01D1
:10649000FEF76DF8CDE90C01DDE90C23DDE90E0115
:1064A000FDF74CFF05460E460022604B284631465C
:1064B000FDF7EBFFCDE902015D490AFB01F0FEF7B4
:1064C000C5F8CDE90001DDE90223FDF737FFCDE98D
:1064D0000401FEF7CCF85249486617A906A8FEF752
:1064E00045FB002404E017A8005D15A90855641CAD
:1064F000032CF8DB15A8FDF707FF8146002405E013
:1065000017A9E01C085C11A90855641C062CF7DBD0
:1065100011A8FDF7F9FE10904FF47A71109890FBD6
:10652000F1F00590FEF792F8CDE90A0100223D4B0B
:10653000DDE90A01FEF71BF8CDE90A014FF47A7193
:10654000109890FBF1F201FB1200C0EB00108000EC
:106550000590FEF77BF8CDE908010022324BDDE91A
:106560000801FEF704F8CDE90801DDE90823DDE9BB
:106570000A01FDF7E3FE0746884600222B4B38460A
:106580004146FDF782FFCDE90201294909FB01F0EF
:10659000FEF75CF8CDE90001DDE90223FDF7CEFE50
:1065A000CDE90401FEF763F81D49886622980028AA
:1065B00033D100221F4B38464146FDF766FFCDE937
:1065C0000201FEF754F805901BA31CA21E21CDE981
:1065D00000901AA80BF050FB002001231AAA1B21DF
:1065E000009001F04FF80022124B28463146FDF78B
:1065F0004CFFCDE90201FEF73AF8059014A315A26D
:106600001E21CDE900A01AA80BF036FB00200123C3
:106610001AAA2B21009001F035F823B0BDE8F08FC5
:10662000C022002000004E4040774B4180842E4124
:1066300040420F00006AF8405300000020CEB3B67D
:10664000C82025733A20252E33642E25303564006A
:106650005700000020BEADB6C82025733A2025643F
:106660002E2530356400000070B5054600240DE08D
:1066700004EB440101EBC402084901EB8200294606
:10668000FDF7D7FD08B9204670BD641C03480838E3
:106690004068A042ECD84FF0FF30F5E7102F002003
:1066A0000246002A01DA0020704702EB420000EBAC
:1066B000C203064800EB8300416A002902DB04485C
:1066C000814201DD0020EFE70846EDE7102F0020B2
:1066D000FFCF1F002DE9F04704460D4691469A462C
:1066E000A02C01DBA02D02DA0020BDE8F087A4F188
:1066F000A000C6B2A5F1A000C7B2BAF1000F10D138
:10670000781E711E5E2202FB010000EB40004FEA82
:10671000C0080B494B4618224868414605F0DEFE8A
:10672000E3E7781E711E5E2202FB01004FEA40186B
:1067300004494B4620224868414605F0CFFED4E785
:10674000FC2A0020F02A002010B538480078401CB0
:10675000C0B236490870022801DD002008703348B5
:10676000007820B901F050FD3149086003E001F0E4
:106770004BFD304908602E4800682E490968884260
:1067800001D0002010BD2C480068294909688842C2
:106790000FD0274800682849086008460068274944
:1067A000884203D001202649087002E000202449D5
:1067B00008702348007858B32248007888B12248EE
:1067C00000781F490978884209D01D4800781E4981
:1067D0000870194800681D4908600120D2E70020B0
:1067E000D0E717480078184908701948007840B970
:1067F0000F48006815490860642015490870012099
:10680000C0E713480078401E114908700020B9E71E
:1068100000200F4908700C48007820B100200A4978
:106820000870401EAEE70020ACE7000049000020E1
:1068300050000020540000204C0000202A04FC00DE
:106840004A000020450000204B00002040000020AE
:106850004800002000B589B009480A49097800EBD2
:106860008100094991F8F612435C08A21E2101A893
:106870000BF002FA01A803F023FD09B000BD0000EF
:106880008C400108900200207A1F002041542B4DBB
:106890004F444F445245583D25640D0A0000000006
:1068A0002DE9F74F90B00546BB484088052802DB2C
:1068B0004FF0050902E0B84890F802904FF0000B45
:1068C000002009904FF47A780DF1280A11980128D8
:1068D00012D1B148D0F80600AF49C1F812000846FD
:1068E000D0F80610102250460DF080F8AA490C98F6
:1068F000C1F80E00002011900024129864287CD169
:1069000076E0A548D0F812701022394650460DF0B6
:106910006DF8082207F110010EA80DF067F89DF838
:10692000280001284DD1BBF1000F07D10BF1010068
:1069300000F0FF0B98490C98C1F80E00DDF82A0012
:10694000C0F344400090DDF82A10C1F383534FF0A8
:106950003F0C0CEA916204EBC40C05F1DE0101EB83
:106960004C008EA10BF09CF904EBC40205F1DE0192
:1069700001EB42000EA9FDF72BFC9DF82900012830
:1069800008D1002104EBC40205F1DE0000EB420057
:10699000417407E0012104EBC40205F1DE0000EBC5
:1069A000420041747C490D98C1F8120001F11600B3
:1069B00000EB84000760601CC4B24C4508DB26462F
:1069C00017E07548D0F806007349C1F812000FE0CF
:1069D000A8F101001FFA80F8B8F1000F07D10122D9
:1069E00072A1002008F0E8F8264602E005E000BFAA
:1069F00087E700BF0020E880BEE072E06648D0F87C
:106A00000E701022394650460CF0F0FF082207F1B4
:106A100010010EA80CF0EAFF9DF8280001284CD1C7
:106A2000099838B90998401CC0B209905A490D9884
:106A3000C1F81200DDF82A00C0F344400090DDF8F0
:106A40002A10C1F383534FF03F0C0CEA916204EB20
:106A5000C40C05F1DE0101EB4C0057A10BF020F94D
:106A600004EBC40205F1DE0101EB42000EA9FDF7C3
:106A7000AFFB9DF82900012808D1002104EBC402D6
:106A800005F1DE0000EB4200417407E0012104EB58
:106A9000C40205F1DE0000EB420041743E490C984F
:106AA000C1F80E0001F1160000EB84000760601CC5
:106AB000C4B24C4506DB264614E037490C98C1F8B1
:106AC0000E000EE0A8F101001FFA80F8B8F1000FE7
:106AD00006D101223BA1002008F06EF8264601E015
:106AE00000BF8BE700BF0DF1100A304606EBD071F6
:106AF000C1F347010391002438E004EBC40105F120
:106B0000DE0000EB41000290701E001B00EBC00194
:106B100005F1DE0000EB410001901222504602997F
:106B2000FDF732FB1222DDE90110FDF72DFB1222E9
:106B300051460198FDF728FB1748163000EB8400FA
:106B40000768701E011B1448163000EB81000168B5
:106B50001148163000EB84000160701E011B0E48C6
:106B6000163000EB81000760601CC4B203988442B9
:106B7000C3DBA9F10100E880AE80002085F83E016A
:106B8000B5F83A11B5F83C0101F02EFF284602F0A5
:106B9000D1F913B0BDE8F08F4025002025303264D4
:106BA0002F253032642F2530326420005B534D5343
:106BB0005D6572723100000025642F25642F256405
:106BC000200000005B534D535D657272320000007F
:106BD0002DE9F04F87B082460E4617464FF0000968
:106BE0000024A3469AF8000008B1307818B90020B4
:106BF00007B0BDE8F08F0FE058460BF1010B01A97B
:106C000001F80080B8F13D0F02D0B8F13B0F01D17F
:106C10000020EDE7761C641C96F80080B8F1000FA8
:106C200001D0142CE8DB3D222046641C01A90A5443
:106C3000002008555046FDF7D7FA0546254405E0E3
:106C4000287838706D1C7F1C09F1010928782028EC
:106C500005DD28783B2802D0B9F1500FF0DD002087
:106C600038704846C4E700002DE9F041044620781A
:106C7000302801D1BDE8F08102262AE0A05D2C2851
:106C800025D1A01CFDF740FB0746A119481CFDF7C4
:106C90003BFB0546052F06D1192D04D1134890F86A
:106CA000300300B11BE0052F07D1372D05D10F4868
:106CB00090F83003012800D011E0052F07D1052DF1
:106CC00005D10A4890F83003022800D007E0701C74
:106CD00006B22046FDF7A6FAB042CFD8CAE703496C
:106CE00091F8300303F0C2FB00BFC3E77A1F002016
:106CF0000021064A00BF05E013780370401C521CB7
:106D00004B1CD9B20C29F7DB70470000E8F7FF1FD6
:106D10000346002227E04D2903D102F10C0082B284
:106D200021E0412905DB5A2903DC02F1080082B287
:106D300019E0612905DB7A2903DC02F1080082B23F
:106D400011E0302905DB392903DC02F1080082B2A9
:106D500009E0202905DB602903DC02F1080082B28A
:106D600001E0901D82B213F8011B0029D3D1D0B2EB
:106D700070470000F0B589B0074617B9002009B088
:106D8000F0BD06A8FFF7B4FF1BA00AF065FF0024C2
:106D900006E006A8015D1BA00AF05EFF601C04B2BD
:106DA0000C2CF6DB19A00AF057FF052408E030028E
:106DB00040EA15662D0206A8005D0543601E04B278
:106DC000002CF4DAB6B22A46334611A00AF044FF8A
:106DD00013A2102102A8CDE900560AF04DFF0024AD
:106DE00004E002A8005D3855601C04B20F2CF8DBEB
:106DF0000020F8730120C2E753544D333220494438
:106E00003D3D000025303278000000000D0A0000F2
:106E100074656D703D253031356C6C750D0A000060
:106E2000253031356C6C75002DE9F0438FB00121B0
:106E30003348FDF777FE00BF02213148FDF7E5FD3D
:106E40000028F9D02E48FDF7DCFD0646642E0ADA4C
:106E5000B6F5805F07DB2BA00AF0FEFE4FF0FF3097
:106E60000FB0BDE8F0832A482A49096840F821603C
:106E700028480068401C27490860092801DD0020D7
:106E80000860002406E0224850F8240005A941F8D3
:106E90002400641C0A2CF6DB002419E000204DF8C5
:106EA000240000250DE005A850F825005DF8241009
:106EB000884205DD05A850F825004DF824002F462E
:106EC0006D1C0A2DEFDB002005A941F82700641C8A
:106ED000042CE3DBDDE9010100EB01080298C8287E
:106EE00002DA4FF0FF30BBE74FF49A7108FB01F074
:106EF000C11700EB11514FEA21394846B0E70000B5
:106F00000024014056444143204F564552000000A2
:106F100018250020DC01002070B5114D11480088B3
:106F2000D8B1E81DFDF77EF904B2B4F5917F05DD17
:106F300001220DA1002007F03FFE70BD2146E81D93
:106F40000BF0E0FF0C48007820F00100401C0A49DB
:106F50000870002048700349088000BFEDE700007A
:106F6000A20600203C0000205541525432524543B5
:106F700056204F5645522100C02200200E4890F85E
:106F8000F9020E4931F8100038B14FF400700C4985
:106F9000486101200B4908600CE04FF4007008497B
:106FA00008610020074908600748007820F00100C8
:106FB00005490870704700007A1F002098400108BA
:106FC00000100140A8000020C022002030B58DB084
:106FD000244801F055FD05462348854204D1234944
:106FE000487808F005FE3AE02148854237D11D482F
:106FF000C08800EB400101EBC0011E4850F8213071
:107000001DA2322168460AF037FE00240DE0154823
:10701000C08800EB400101EBC001164800EB810085
:10702000801D005D19490855641C242CEFD30D48C0
:10703000C08800EB400101EBC0010E4850F8210070
:1070400013490860684603F03BF9012008F0D0FDC1
:107050000020104988704FF480700F4948610DB0CE
:1070600030BD0000702800202A04F400CC0200206B
:107070002A04EC004C09002041542B504F433D3072
:107080003930303030253038780D0A00880E002035
:107090007C000020D00700200010014008B502202D
:1070A0001A23A0220C210090002000F00DF90548C1
:1070B00000788023A0221B210090002003F062FDB5
:1070C00008BD0000A00300202DE9F05F04460D4636
:1070D00016461F46A02C01DA802D01DBBDE8F09F8B
:1070E000A019A02802DBC4F19F0086B2E81980280D
:1070F00002DBC5F17F0087B2E819401E83B2A019F8
:10710000401E82B22946204601F0B8F84FF0000830
:1071100018E005EB08001FFA80FA4FF000090BE0B9
:1071200004EB09001FFA80FB084800780AF0C2FB54
:1071300009F101001FFA80F9B145F1DB08F1010006
:107140001FFA80F8B845E4DB00BFC7E7A0030020C2
:107150002DE9FC5F04460D4616461F46B44201DC8D
:10716000BD4201DDBDE8FC9FA02E00DB9F26802FE5
:1071700000DB7F27301B401C80B20090781B401C36
:107180001FFA80FB05EB0B00401E83B200982044E1
:10719000401E82B22946204601F070F84FF00008E8
:1071A00029E005EB08001FFA80F94FF0000A1BE008
:1071B00004EB0A0080B20190B9F10D0F04DA104817
:1071C00000780AF077FB0BE0B9F11B0F04DA0D48E9
:1071D00000780AF06FFB03E00B4800780AF06AFBC6
:1071E0000AF101001FFA80FA00988245E0DB08F1FD
:1071F00001001FFA80F8D845D3DB00BFB2E70000DA
:107200009F0300209E030020A0030020F8B507463E
:107210000D4616461C4604B9F8BDBD4200DAFBE730
:10722000601EC4B200200090301983B22A46314655
:10723000384600F049F800BFEEE72DE9F84306466E
:107240000C4617461D46DDF82080BE4201DCAC42EC
:1072500001DDBDE8F8834346224639463046FFF754
:10726000D5FF43462A4639463046FFF7CFFF012077
:107270004346324629460090204600F00AF8012095
:1072800043463A4629460090204600F002F800BFE7
:10729000DFE72DE9F84305460E4617461C46DDF8A4
:1072A00020800CB9BDE8F883AE4200DAFAE7601E30
:1072B000C4B2381982B2334629463846CDF8008028
:1072C00000F002F800BFEDE72DE9FC5F04460D4633
:1072D00016461F46B44201DCBD4201DDBDE8FC9FFD
:1072E000A02C01DA802D00DBF8E7A02E00DB9F2622
:1072F000802F00DB7F27301B401C1FFA80FB781B90
:10730000401C1FFA80FA05EB0A00401E83B204EB12
:107310000B00401E82B22946204600F0AFFF4FF01E
:1073200000083DE005EB080080B2009000987F283F
:1073300001DD7F2000904FF000092BE004EB0900F5
:1073400080B2019001989F2801DD9F2001900C9848
:10735000012815D0022808D003280BD004280ED10C
:10736000114800780AF0A6FA0FE0104800780AF0F9
:10737000A1FA0AE00E4908780AF09CFA05E000BF7D
:107380000C4800780AF096FA00BF00BF09F101002E
:107390001FFA80F9D945D1DB08F101001FFA80F806
:1073A000D045BFDB00BF99E7A10300209E0300206A
:1073B000A60300209F03002010B511A000F0CAF919
:1073C00018B90FA110A00AF047FC17A000F0C2F9ED
:1073D00018B915A116A00AF03FFC1DA006F03EFA50
:1073E0001E4B4FF47F026FF07F418B2000F03EF880
:1073F000FFF754FE1AA20021084600F0E2F810BD83
:10740000485A4B313600000043616E27742066698C
:107410006E642074686520487A6B313646696C6505
:1074200028257329210D0A00485A4B3132000000EB
:1074300043616E27742066696E6420746865204815
:107440007A6B313246696C6528257329210D0A0053
:10745000616C6C7069632E626D700000FF64640083
:1074600077656C636F6D652E626D7000F0B50746D1
:107470000C4615461E463846FEF76AFB0949087059
:107480002046FEF765FB084908702846FEF760FBBA
:10749000064908703046FEF75BFB054908700AF0A4
:1074A00047F9F0BD9F030020A00300209E030020A9
:1074B000A10300202DE9F84F05460E4617469846D1
:1074C00008F00F0908F0F00AB9F1010F09D0B9F17D
:1074D000020F21D0B9F1030F39D0B9F1040F6CD1EB
:1074E00050E0002415E0012006EB040C1FFA8CF399
:1074F00005EB040C1FFA8CF2A6EB040C1FFA8CF1BE
:1075000005EB040C00901FFA8CF0FFF796FE601C50
:1075100084B2BC42E7DB51E0002415E0012006EB19
:10752000040C1FFA8CF3A5EB040C1FFA8CF2A6EBEB
:10753000040C1FFA8CF1A5EB040C00901FFA8CF0E0
:10754000FFF77BFE601C84B2BC42E7DB36E0002420
:1075500015E0012006EB040C1FFA8CF305EB040C7C
:107560001FFA8CF206EB040C1FFA8CF1A5EB040C4D
:1075700000901FFA8CF0FFF760FE601C84B2BC42E2
:10758000E7DB1BE0002415E00120A6EB040C1FFA4A
:107590008CF305EB040C1FFA8CF2A6EB040C1FFA1B
:1075A0008CF1A5EB040C00901FFA8CF0FFF745FE60
:1075B000601C84B2BC42E7DB00E000BF00BFBDE856
:1075C000F88F2DE9F04FFDB080460D4691464846B4
:1075D000FFF74AF883465846FFF762F88246BAF149
:1075E000000F02D17DB0BDE8F08F7CAB02221C21E0
:1075F000584604F073FF7BAB04221221584604F076
:107600006DFF7AAB04221621584604F067FF7B9881
:10761000A02802D87A98802800D9E3E779AB042221
:107620000A21584604F05AFF18207B990AF0BCFA48
:1076300006467A98471E7A982844401E83B27B9863
:107640004044401E82B22946404600F017FE002406
:1076500013E0799806FB070101AB3246584604F067
:107660003DFF01A800907B9882B2281981B20123C6
:10767000404603F0FFFB7F1E641C7A988442E8D3E7
:1076800000BFAFE72DE9FF4F85B0804692461F4609
:10769000DDF848B007F0F0000390039828B94FF0E8
:1076A0000C0901250C20049004E04FF0100901257D
:1076B000102004905446002625E020789F280EDDF7
:1076C000CDE9007B6378227808EB060188B2069941
:1076D00003F0AAFA06EB090086B2A41C13E0CDE978
:1076E000007B237808EB060188B20022069903F09C
:1076F0009BFA039818B906EBC50086B202E006EBC8
:10770000C50086B2641C20780028D6D109B0BDE837
:10771000F08F00000948C088084989880843074954
:1077200049880843054909880843054908800846EF
:10773000018804A00AF090FA00BFFEE7B80200201A
:10774000C00200200D0A5B4846483D253034785D74
:107750000D0A000070B505462C48406808B90020A5
:1077600070BD2BA12846FCF764FD58BB2A480021B8
:107770000160416081602846FEF776FF0446002CD8
:1077800001DA0020ECE710202349087048700978DE
:10779000214A527801FB02F0C11700EB5171C1F38D
:1077A000C7011D4A91701046446004EB440000EB91
:1077B000C4011648083000EB8100406A1146886019
:1077C0000120CDE715A12846FCF733FDD8B91548AF
:1077D00000210160416081602846FEF745FF0446B4
:1077E000002C01DA0020BBE70E48446004EB4400A3
:1077F00000EBC4010548083000EB8100406A0949EC
:1078000088600120ACE700BFAAE70000082F002035
:10781000485A4B3136000000F02A0020485A4B31BC
:1078200032000000FC2A002010B504460121C802E5
:1078300004F004FD7D2004F095FD08B104F01EFD68
:1078400045F2555000F028F8062000F019F8A0B2D3
:1078500000F01CF800F00CF800F002F810BD000079
:107860004CF6CC40014908607047000000300040F1
:107870004AF6AA2001490860704700000030004025
:1078800001494860704700000030004001498860AD
:107890007047000000300040014908607047000058
:1078A0000030004030B587B001A804F0B3FD434874
:1078B000407868B9424801780078401C404A10700E
:1078C00021B901223FA1002007F076F907B030BDB1
:1078D0004048007800B1F9E738480078C0F340002C
:1078E00000B9F3E73548007820F00200334908700A
:1078F000012239A1002007F05FF9022007F082F988
:107900002E480078C0F3800000B1DFE707F016FBD7
:1079100003AC01208DF80C008DF80D00BDF80400BB
:1079200080069DF8061040EA81509DF8071040EA55
:1079300041409DF8081040EA01309DF8091040EAE6
:1079400081109DF80A100843CDF80E002148B0F8C8
:107950009601ADF812001948D0F80A100822204606
:107960000CF0BAF81B4D08351448D0F80A0000F1A5
:1079700010014FF4C87228460CF0AEF80F4800789A
:1079800020F00100401C0D49087008464088401C4A
:10799000488008468088401C88800846D0F80A0045
:1079A000C1F806000846D0F806000F49C1F88C005F
:1079B000002002F09DFD00BF88E700004025002068
:1079C000000200205B534D535D496E76616C696423
:1079D00000000000302300205B534D535D53746F53
:1079E000726520534D5300007A1F002008B50E48E1
:1079F000007800B108BD0D480CF01CFB90B14FF4AD
:107A0000FA710A480CF02EFB0948007800900948EA
:107A10000078C0F30011084803780348027807A0F3
:107A20000AF01AF900BFE5E788020020A80200204A
:107A3000CC020020C022002093020020496E666F15
:107A40003A417574685B25645D2C47545B25645D21
:107A50002C4D495B25645D2C55495B25645D0D0A01
:107A6000000000000021016041608160C16001618F
:107A7000491E41617047000004480078FF2804DA7D
:107A800002480078401C01490870704747000020F8
:107A900010B553480068534A811A904262D017DCEF
:107AA000514AA0EB0201904268D00ADC4F490844D9
:107AB000002839D0B0F5401F76D0B0F5601F2BD12B
:107AC00062E0B1F5001F53D0B1F5401F7ED143E015
:107AD000474A881A914211D00BDCB1F5802F6CD047
:107AE00044480844002859D04349084400286DD12F
:107AF0002CE0182803D01E2868D11EE000BF012208
:107B00003EA1002007F058F800204449087044497D
:107B100088714448007800B158E043A002F0D0FBDF
:107B200000204549087051E0012244A1002007F0DF
:107B300043F800204049087048E0012244A1002099
:107B400007F03AF800203C4908703FE0012245A1C7
:107B5000002007F031F839E0012247A1002007F0AA
:107B60002BF833E001224BA1002007F025F82DE08F
:107B700001224FA1002007F01FF827E0012252A1A7
:107B8000002007F019F821E0012256A1002007F09B
:107B900013F800201249086018E005E0012258A1FE
:107BA000002007F009F811E001225CA1002007F095
:107BB00003F800200A49086008E001225EA10020C5
:107BC00006F0FAFF00206249087000BF00BF0448B9
:107BD00000686049884202D000201749087010BD33
:107BE000400000202A04F4002A04BC00D6FB83FFD6
:107BF000E0FF0700FCFBFBFF0408FCFF5B4B455963
:107C00005F5050542F4B45595F5050545F4D49437E
:107C10002052656C656173655D00000046000020C0
:107C2000D00700207E02002041542B504F433D30AE
:107C300043303030300D0A00450000205B4B455981
:107C40005F55502052656C656173655D00000000F2
:107C50005B4B45595F444F574E2052656C656173CD
:107C6000655D00005B4B45595F4F4B2052656C656D
:107C70006173655D000000005B4B45595F50414EEC
:107C8000454C5F4D454E552052656C656173655D91
:107C9000000000005B4B45595F50414E454C5F452D
:107CA0005849542052656C656173655D00000000A1
:107CB0005B4B45595F50414E454C5F5550205265D6
:107CC0006C656173655D00005B4B45595F50414ECB
:107CD000454C5F444F574E2052656C656173655D3E
:107CE000000000005B4B45595F455849545F444FC5
:107CF000574E5F47542052656C656173655D0000A7
:107D00005B4B45595F50315F50335F555044415490
:107D1000452052656C656173655D00005B4B45599C
:107D20005F4F4B5F444F574E5F4750532052656C37
:107D3000656173655D0000005B4B45595F4F5054B2
:107D4000494F4E2052656C656173655D000000000F
:107D5000820200202A04FC0010B5FEF7F5FC041E88
:107D600011D0012C0DD108480068401C064908605C
:107D700000F07EF8012000F059FA00200349088045
:107D800001E0FFF785FE10BD84020020A400002062
:107D900008B50121084604F061FA01213048FEF7D8
:107DA000EBF801211C2004F059FA48208DF803005B
:107DB00003208DF802000820ADF80000694629482C
:107DC000FEF74EF82020ADF8000069462648FEF781
:107DD00047F84020ADF8000069462348FEF740F818
:107DE0008020ADF8000069461F48FEF739F81020E2
:107DF000ADF8000069461C48FEF732F80820ADF8DF
:107E0000000069461848FEF72BF80420ADF8000082
:107E100069461548FEF724F80220ADF800006946CF
:107E20001048FEF71DF84FF48060ADF80000694679
:107E30000C48FEF715F82020ADF800006946094807
:107E4000FEF70EF810208DF803000001ADF80000D9
:107E500069460548FEF704F800200449087008BD8B
:107E60000002300000100140000C014045000020DD
:107E700000B589B079480068794A811A904270D07B
:107E800017DC784AA0EB020190426BD00ADC7649FD
:107E90000844002835D0B0F5401F74D0B0F5601FFD
:107EA0002ED1A6E0B1F5001F6ED0B1F5401FF7D17D
:107EB0006BE06E4A881A914211D00BDCB1F5802F2D
:107EC0007ED06B48084400287BD06A4908440028CB
:107ED000E6D148E0182803D01E28E1D129E000BFF0
:107EE000012065490870654988716548007810B9B6
:107EF00064A002F0E5F9012266A1002006F05CFE14
:107F0000A9E001205C4908705D48007858B96848CC
:107F10000078012807D15948007820B165A002F007
:107F2000CFF906F0F5FF012267A1002006F044FE1C
:107F300091E00120504908705148007858B95C48D8
:107F40000078012807D14D48007820B162A002F0E6
:107F5000B7F906F0DDFF012264A1002006F02CFE37
:107F600079E034E03FE0012265A1002006F024FE24
:107F70004F480078012805D16548007810B90420E1
:107F800007F036FE67E040E027E0012261A1002013
:107F900006F012FE5E480078C0B100205C4908700F
:107FA000624B63A21E2101A809F066FE01A802F03F
:107FB00087F964A26B21012006F0B8F8002201E0E5
:107FC00029E01CE001A9104606F0F6FD43E001227D
:107FD0005EA1002006F0F0FD3DE0012261A100203D
:107FE00006F0EAFD37E0012264A1002006F0E4FD7E
:107FF00031E0012267A1002006F0DEFD2BE0012226
:108000006BA1002006F0D8FD25E001226FA1002021
:1080100006F0D2FD1FE073480078401C71490870DB
:1080200008460078032810D10AF0B8FA6E480078A4
:10803000C0F3001048B11E480078012805D16B48F4
:108040000078012801D16A490870012269A1002045
:1080500006F0B2FD00BF00BF09B000BD4000002027
:108060002A04F4002A04BC00D6FB83FFE0FF0700CB
:10807000FCFBFBFF0408FCFF45000020D0070020AC
:108080007E02002041542B504F433D30423030306F
:10809000300D0A005B4B45595F5050542F4B4559EA
:1080A0005F5050545F4D49432050726573735D00BB
:1080B000CC02002041542B504F433D313030303002
:1080C0003030380D0A0000005B4B45595F55502099
:1080D00050726573735D000041542B504F433D3126
:1080E000303030303030370D0A0000005B4B4559DE
:1080F0005F444F574E2050726573735D000000005F
:108100005B4B45595F4F4B2050726573735D0000A8
:10811000800200205B4B45595F50414E454C5F4DFE
:10812000454E552050726573735D0000740E00203B
:1081300041542B504F433D30393030303025730D92
:108140000A000000B2CBB5A5000000005B4B45590A
:108150005F50414E454C5F455849542050726573FD
:10816000735D00005B4B45595F50414E454C5F5578
:10817000502050726573735D000000005B4B4559E1
:108180005F50414E454C5F444F574E2050726573CF
:10819000735D00005B4B45595F455849545F444F40
:1081A000574E5F47542050726573735D00000000A6
:1081B0005B4B45595F50315F50335F5550444154DC
:1081C000452050726573735D000000005B4B45599C
:1081D0005F4F4B5F444F574E5F475053205072657F
:1081E00073735D0082020020C022002092020020F2
:1081F000180200205B4B45595F4F5054494F4E20A9
:1082000050726573735D00000648016801F0FC015F
:1082100009040548826840F22A40024041EA02000F
:1082200070470000080C01400010014010B50446E2
:108230003CB980200749486141000748FDF7EDFE41
:1082400006E080200349086141000348FDF7E7FE8E
:1082500010BD000000100140000C014010B50446A4
:108260002146054804F074FB00BF8021024804F059
:1082700063FB0128F9D010BD003800402DE9F05F04
:1082800004460D4616461F46A046B146AA46BB46C2
:108290002A2000F0C7F94FEA282000F0D7F908F0AB
:1082A000FF0000F0D3F94FEA292000F0CFF909F0E0
:1082B000FF0000F0CBF92B2000F0B4F94FEA2A20A0
:1082C00000F0C4F90AF0FF0000F0C0F94FEA2B20DB
:1082D00000F0BCF90BF0FF0000F0B8F92C2000F022
:1082E000A1F9BDE8F09F00002DE9F0410E4800889B
:1082F00006120D4807787F239F2200210846FFF7CA
:10830000BDFF00240BE0002506E0304600F09EF99A
:10831000384600F09BF96D1CA02DF6DB641C802C08
:10832000F1DBBDE8F08100009803002010B500F0FB
:1083300003F980207F494861402008610120FDF752
:10834000C8F840207B4948610120FDF7C2F8402071
:10835000784908617820FDF7BCF8112000F062F937
:108360007820FDF7B6F8B12000F05CF9052000F0A8
:108370006DF93C2000F06AF93C2000F067F9B2206A
:1083800000F050F9052000F061F93C2000F05EF9A2
:108390003C2000F05BF9B32000F044F9052000F028
:1083A00055F93C2000F052F93C2000F04FF905202F
:1083B00000F04CF93C2000F049F93C2000F046F96F
:1083C000B42000F02FF9032000F040F9C02000F0A5
:1083D00029F9282000F03AF9082000F037F90420A4
:1083E00000F034F9C12000F01DF9C02000F02EF992
:1083F000C22000F017F90D2000F028F9002000F04D
:1084000025F9C32000F00EF98D2000F01FF92A2075
:1084100000F01CF9C42000F005F98D2000F016F9D9
:10842000EE2000F013F9C52000F0FCF81A2000F04F
:108430000DF9362000F0F6F8A02000F007F9E02052
:1084400000F0F0F8042000F001F9222000F0FEF81E
:10845000072000F0FBF80A2000F0F8F82E2000F0CA
:10846000F5F8302000F0F2F8252000F0EFF82A208F
:1084700000F0ECF8282000F0E9F8262000F0E6F8FB
:108480002E2000F0E3F83A2000F0E0F8002000F0A1
:10849000DDF8012000F0DAF8032000F0D7F813200F
:1084A00000F0D4F8E12000F0BDF8042000F0CEF890
:1084B000162000F0CBF8062000F0C8F80D2000F0E0
:1084C000C5F82D2000F0C2F8262000F0BFF82320C8
:1084D00000F0BCF8272000F0B9F8272000F0B6F82B
:1084E000252000F0B3F82D2000F0B0F83B2000F07C
:1084F000ADF8002000F0AAF8012000F0A7F8042051
:1085000000F0A4F8132000F0A1F83A2000F08AF857
:10851000052000F09BF8292000F084F84FF6FF7149
:10852000002000F0A7F8FFF7DFFE80200149086176
:1085300010BD00000010014000B587B001211820D7
:1085400003F08CFE03208DF81A0010208DF81B001C
:108550000121800203F072FE4FF48040ADF8180054
:1085600006A92D48FDF77CFC4FF480402A491031C4
:1085700008608010ADF8180006A92748FDF770FCC8
:108580004FF40050ADF8180018208DF81B0006A914
:108590002148FDF765FC4FF40040ADF8180006A92E
:1085A0001D48FDF75DFC4FF480501B4910310860F9
:1085B0004FF44040ADF804004FF48270ADF806006F
:1085C0000020ADF80800ADF80A00ADF80C00481521
:1085D000ADF80E000020ADF81000ADF81200072035
:1085E000ADF8140001A90D4804F0B4F901210B48BD
:1085F00004F096F910208DF81B00C020ADF818008B
:1086000006A90748FDF72CFC402005490861802099
:10861000086107B000BD0000000C014000380040B8
:108620000010014010B504464FF480400649086030
:10863000801008602046FFF711FE4FF48050024979
:10864000091F086010BD0000140C014010B504465D
:108650004FF48040064908608010091D08602046DC
:10866000FFF7FCFD4FF480500149086010BD000089
:10867000100C0140024A1080024A1180704700002D
:108680009A0300209803002008B50121084603F052
:10869000E5FD01211648FDF76FFC01213C2003F0A8
:1086A000DDFD10208DF8030003208DF802004FF44B
:1086B0000050ADF8000069460E48FDF7D1FB0420DC
:1086C000ADF8000069460C48FDF7CAFB4FF4807016
:1086D000ADF8000069460948FDF7C2FB4FF40050B1
:1086E00004490861042004491031086008BD0000F5
:1086F000000230000010014000140140000C014055
:1087000008B30021624A1160624A1170624A117016
:10871000624A1170FF21624A1170624A1170002191
:10872000614A1170614A1170614A1170FF21614AFA
:108730001170614A11704FF40051604A5161042177
:108740005F4A116070475F49097821B94FF40051C1
:108750005A4A516149E05C49097821B94FF4005106
:10876000564A116141E04E490978564A12789142C1
:1087700005D14C490978544A1278914219D0002108
:10878000444A1170484A11704E490978444A1170A0
:108790004D490978434A11704A4909784906090E3A
:1087A0003E4A11703F490978127802EB41013A4A7A
:1087B000117038490978491CC9B2364A1170364AD5
:1087C0001278914202DD0021324A11703149097854
:1087D000324A1278914204DA4FF40051374A11615B
:1087E00003E04FF40051354A51613849097819B90D
:1087F0000421334A116048E03549097821B9042140
:108800002F4A121F116040E02A4909782F4A127836
:10881000914205D1284909782D4A1278914219D000
:1088200000211C4A1170204A117028490978214AF8
:10883000117027490978204A11702449097849069E
:10884000090E1B4A11701C490978127802EB41018C
:10885000164A117014490978491CC9B2124A11709C
:10886000124A1278914202DD00210F4A11700E491E
:1088700009780F4A1278914204DA0421104A121F33
:10888000116002E004210E4A116000BF5AE70000A7
:108890006400002068000020690000206A000020B9
:1088A0006B0000206C0000206D0000206E00002096
:1088B0006F000020700000207100002000100140B7
:1088C0001414014058000020590000205A000020D4
:1088D0005B0000202DE9F0470446884691461E467D
:1088E000DDF820A0C4F80080002507E0206850F8DB
:1088F0002500077807B903E0681CC5B2C82DF5DB71
:1089000000BF681EC5B2681CA080052095FBF0F072
:1089100060816089052190FBF1F201FB120010B12A
:108920006089401C60810025C4F8D8600AE006B95F
:108930000AE0D4F8D80050F82500077807B903E01A
:10894000681CC5B2C82DF2DB00BFA4F8DC500025BE
:108950000EE0A088A84205DD1AF8051004F10D000C
:10896000415503E0002104F10D004155681CC5B2DA
:10897000C82DEEDB84F80C9000202081E08020469A
:1089800000F066F9BDE8F0872DE9F04704460F4690
:1089900016469846A4F83A710120A4F83C0100203C
:1089A000E08084F80C800025C4F8D8600DE006B99A
:1089B0000DE0D4F8D80050F8250090F80090B9F1F7
:1089C000000F00D103E0681CC5B2C82DEFDB00BF6B
:1089D000A4F8DC50642084F8380164220121204688
:1089E000FDF75EFFBDE8F0872DE9FF4106460F4623
:1089F0000A2E01DA012409E0642E01DA022405E0DE
:108A0000B6F57A7F01DA032400E004240A2F01DAA4
:108A1000012509E0642F01DA022505E0B7F57A7F28
:108A200001DA032500E00425334612A20B2101A838
:108A3000009709F021F960191049098888420AD085
:108A400060190E49088002201923A0220D210090F0
:108A50005020FEF739FC00206119891CC900C1F1C2
:108A6000A001009088B2012301AA0D21FEF70AFEA1
:108A7000BDE8FF8125647C2564000000B003002070
:108A800070B50446A08810B92748006870BD264814
:108A900000682649084408B3B0F5001F3DD1002105
:108AA000204600F030F9E08818B9A088401EE08028
:108AB00002E0E088401EE080257AE088052190FBF6
:108AC000F1F020812089A84203D0204600F0C0F8B0
:108AD00003E00121204600F016F921E000212046A4
:108AE00000F011F9E088401CE080E088A18888420D
:108AF00001DB0020E080257AE088052190FBF1F081
:108B000020812089A84203D0204600F0A1F803E08C
:108B10000121204600F0F7F802E003480068B5E7BD
:108B200000BF0020B2E7000040000020D6FB43FF5A
:108B300010B50446A08810B94348006810BD4248EB
:108B400000684249084400283CD0B0F5001F03D01B
:108B5000B0F5601F72D16DE0204600F00CF9B4F85A
:108B60003C01401EA4F83C01B4F83C0118B9B4F82B
:108B70003A01A4F83C01E08880B9B4F83A0105282C
:108B800008DD752200212046FDF78AFE012084F8C9
:108B90003E0106E0A088401EE08002E0E088401E22
:108BA000E08094F83E0118B1002084F83E0102E014
:108BB000204600F0E0F8B4F83A11B4F83C01FFF7B1
:108BC00013FF3EE0204600F0D6F8E088401CE0802D
:108BD000B4F83C01401CA4F83C01B4F83C01B4F8E2
:108BE0003A11884202DD0120A4F83C01E088A18806
:108BF00088420EDBB4F83A01052808DD6422002122
:108C00002046FDF74DFE012084F83E0101E00020E2
:108C1000E08094F83E0118B1002084F83E0102E0A3
:108C2000204600F0A8F8B4F83A11B4F83C01FFF778
:108C3000DBFE06E00448006880E7FFE702480068C2
:108C40007CE700BF002079E740000020D6FB43FF0F
:108C50002DE9F0410446A08808B9BDE8F081207AEA
:108C600000EB8000C7B23D4619E0A088A84210DCA6
:108C7000052095FBF0F100FB11501D2101EB0010C8
:108C80001FFA80F81023902241460020FEF71CFABC
:108C900003E02946204600F088F8681CC5B2781D1C
:108CA0008542E2DB0121204600F02DF88F26208945
:108CB000002808DD06F1080188B2032308221D21DF
:108CC000FEF7F8FB05E0082310221D213046FEF7D1
:108CD000FBF94FF06D0821896089401E814208DA56
:108CE00006F1080188B2042308224146FEF7E2FBA0
:108CF00007E0A8F1080081B2082310223046FEF7F1
:108D0000E3F900BFA9E72DE9F84304460E464FF00A
:108D10000008D4F8D80018B108F1100000F0FF08DE
:108D2000E088052190FBF1F201FB1200C7B21D2083
:108D300000EB0710C5B24EB1042005F10E038C22E2
:108D4000294600904046FEF7BFFA08E0032005F1EF
:108D50000E038C22294600904046FEF7B5FA009695
:108D6000E188206850F82120012329464046FEF77B
:108D700089FCBDE8F883F8B504460026D4F8D8008D
:108D800010B106F11000C6B2A5791D2000EB051048
:108D9000C7B201200090E188206850F8212001230B
:108DA00039463046FEF76EFCF8BD2DE9F0438BB036
:108DB00004460D46052095FBF0F100FB115087B2EB
:108DC00000261D2000EB07101FFA80F910238E22C9
:108DD00049463046FEF778F9142106A8FBF7EDF96D
:108DE000207B18B100208DF82B0009E0206850F896
:108DF0002510142206A8FBF709FA00208DF82B0095
:108E0000112206A901A806F021F8D4F8D800B0B1C3
:108E100004F10D0010F80580D4F8D80050F828208F
:108E200049463046FEF7CDFB002006F110010090C8
:108E300088B2012301AA4946FEF724FC07E000207E
:108E4000012301AA494600903046FEF71BFC0BB0F7
:108E5000BDE8F0832DE9F0438BB004460D460520B4
:108E600095FBF0F100FB11501FFA80F800271D2040
:108E700000EB08101FFA80F910238E22494638466D
:108E8000FEF722F9142106A8FBF797F9207B18B109
:108E900000208DF82B000CE005EBC50204F1DE008C
:108EA00000EB4201142206A8FBF7B0F900208DF870
:108EB0002B00112206A901A805F0C8FFD4F8D8009C
:108EC00058B305EBC50104F1DE0000EB4100407C26
:108ED000B4F8DC10884206DB012215A1002005F061
:108EE0006BFE002606E005EBC50104F1DE0000EB99
:108EF0004100467CD4F8D80050F826204946384630
:108F0000FEF75FFB002007F11001009088B20123FB
:108F100001AA4946FEF7B6FB07E00020012301AA9B
:108F2000494600903846FEF7ADFB0BB0BDE8F08334
:108F30004C4231002DE9F0410446A08808B9BDE853
:108F4000F081002512E0A088A84209DC1D2000EB7A
:108F500005171023902239460020FEF7B5F803E0EC
:108F600029462046FFF776FF681CC5B2052DEADBCF
:108F700094F83801752802D1A088401EE080204670
:108F8000FFF7F9FE8F26B4F83A01052808DD06F14F
:108F9000080188B2032308221D21FEF78BFA05E0A1
:108FA000082310221D213046FEF78EF86D27B4F8F5
:108FB0003A01052808DD06F1080188B204230822D9
:108FC0003946FEF777FA07E0A7F1080081B20823D7
:108FD00010223046FEF778F800BFB0E7F0B58FB04A
:108FE00005460126012705EB850000EB45111848D1
:108FF0000C18207810B1052817D106E06B1C15A2BB
:10900000322102A808F038FE12E0A07858B9B4F86E
:109010000300611D6B1C14A2CDE90010322102A8CF
:1090200008F02AFE00E0002702E00026002700BF2B
:1090300000BF2078401CC0B22070052801DD002050
:10904000207017B102A801F03BF930460FB0F0BD17
:10905000CB24002041542B54435053544154555376
:109060003D25640D0A00000041542B5443504F50DD
:10907000454E3D25642C25733A25640D0A000000F9
:109080002DE9F04190B0044620680E9060680F9082
:109090002088C0F3C507382F02DAC7F1380001E095
:1090A000C7F17800804642462849204600F062F821
:1090B0000026002518E004F11800E91C405C0206B7
:1090C00004F11800A91C405C42EA004204F11800B7
:1090D000691C405C42EA002004F11801495D084324
:1090E0004DF82600761C2D1D0E2EE4D3694604F1A2
:1090F000080006F04FF80026002521E004F10800E2
:1091000010F8261050304155503830F82600C0F382
:10911000072204F15800691C4254503850F82600C8
:10912000C0F3074204F15800A91C4254503850F8CB
:109130002600000E04F15801EA1C8854761C2D1DEF
:10914000042EDBD310B0BDE8F0810000A45201086A
:1091500000214160016005498160054AC260CA433F
:109160000261034AD2434261704700000123456710
:1091700089ABCDEF2DE9F04391B004460F4615467B
:109180002088C0F3C509206800EBC500216888422B
:1091900002D26068401C6060206800EBC50020605F
:1091A000606800EB5570606033E017F8012B4846AB
:1091B00009F1010904F118010A54B9F1400F28D14D
:1091C0004FF0000800261AE004F11800F11C405C82
:1091D000020604F11800B11C405C42EA004204F1AE
:1091E0001800711C405C42EA002004F11801895DFE
:1091F000084301A941F8280008F10108361DB8F11B
:10920000100FE1D301A904F1080005F0C3FF4FF0EE
:109210000009281EA5F10105C7D111B0BDE8F083F2
:1092200008B54FF4A06001F0FFFA25208DF800008A
:1092300001208DF801008DF802008DF803006846CA
:1092400001F0BAFA26208DF8000001208DF8010007
:109250008DF802008DF80300684601F0ADFA272072
:109260008DF8000001208DF801008DF802008DF8C6
:109270000300684601F0A0FA17208DF800000120D5
:109280008DF801008DF802008DF80300684601F0AA
:1092900093FA0E208DF8000001208DF801008DF862
:1092A00002008DF80300684601F086FA4FF4C060B2
:1092B00001F0BAFA03208DF8000001208DF80100BA
:1092C00000208DF8020001208DF80300684601F0AF
:1092D00073FA08BD70B50546002407E0285D0D2827
:1092E00002D10020285570BD601C84B22846FAF7D0
:1092F00099FFA042F2D800BFF5E7000030B585B075
:1093000004460D46012005F003FD234607A2142163
:10931000684608F0B1FC684600F0D2FF284600F02D
:10932000CFFF06A000F0CCFF05B030BD41542B4C60
:1093300053485454533D25642C220000220D0A004A
:1093400000BFFEE72DE9F04104460F4627600025E7
:1093500000BF206850F8250090F80080B8F1000F99
:1093600000D102E0681CC5B2F3E700BF681EC5B2B9
:10937000681C2071052095FBF0F0E071E079052173
:1093800090FBF1F201FB120010B1E079401CE0719A
:10939000124800681249884202D01248006980B120
:1093A000104802F001FFC6B2042E03DD0120A071B7
:1093B000667102E00020A071667100200949086111
:1093C00007E0064800680849884202D10020A071E1
:1093D0006071204600F05CF8BDE8F081400000209C
:1093E0002A04F400582800202A04EC0070B5044632
:1093F000254800682549084408B3B0F5001F3DD151
:109400000021204600F09DF8607918B92079401EAF
:10941000607102E06079401E6071A5796079052174
:1094200090FBF1F0A071A079A84203D0204600F093
:109430002FF803E00121204600F083F821E000210D
:10944000204600F07EF86079401C607160792179D7
:10945000884201DB00206071A5796079052190FBCD
:10946000F1F0A071A079A84203D0204600F010F8D6
:1094700003E00121204600F064F802E002480068A1
:1094800070BD00BF0020FBE740000020D6FB43FF7B
:109490002DE9F0410446A07900EB800000F0FF08C0
:1094A000454619E02079A84210DC052095FBF0F133
:1094B00000FB11501D2101EB001087B2781E81B214
:1094C000102378220020FDF7FFFD03E02946204607
:1094D00000F06FF8681CC5B208F105008542E1DBB9
:1094E0000121204600F02DF88C26A079002808DD07
:1094F00006F10A0188B2032308221D21FDF7DAFFD5
:1095000005E012231A461D213046FDF7DDFD6D27CB
:10951000A179E079401E814209DABA1E91B206F1C2
:109520000A0290B204230822FDF7C4FF07E0A7F166
:109530000A0081B2082313223046FDF7C5FDBDE8BD
:10954000F0812DE9F84F04460D464FF0000960798F
:10955000052190FBF1F201FB120000F0FF081D2035
:1095600000EB0810C6B26179206850F821703846C7
:10957000FDF7CEFB0FFA80FA4DB1042006F10E0381
:109580008C22314600904846FDF79EFE08E00320FD
:1095900006F10E038C22314600904846FDF794FEFA
:1095A00001233A46314648460095FEF76BF8BDE880
:1095B000F88FF8B505460C46052094FBF0F100FB4A
:1095C0001140C6B21D2000EB0610C7B2781E81B252
:1095D000122378221420FDF777FD002000902868E0
:1095E00050F82420012339460020FEF74BF8F8BD3F
:1095F00010B50B4800680B49884208D10A484088DA
:10960000012801DBFBF79CFF052006F0F1FA044876
:1096100000680649884202D1052006F0E9FA10BD2B
:10962000400000202A04EC00402500202A04F40019
:1096300038B50446ACB1FDF731FD012109A004F0B5
:10964000E3FD0BA004F0F8FE01236E229F21002011
:10965000FDF7DCFD0020012308A272210090FEF737
:1096600011F838BDCFFBCFA2C9BEB3FD000000008A
:10967000C8B7B6A8C9BEB3FD3F0000005B4D5DC8CA
:10968000B7B6A820205B455849545DC8A1CFFB0060
:109690002DE9F04104460F4615461E462780A57069
:1096A0003046FAF7BFFD84F87500102084F8770083
:1096B000002084F87400BDE8F0812DE9F84F0446DD
:1096C00089464FF0000A4E4694F802C094F877E0BD
:1096D0000CEB0E03B4F800C094F876E0F4441FFAE3
:1096E0008CF2A1782088FDF7EFFC142104F16000D2
:1096F000FAF763FD2088C0F19F0087B23846F9175A
:1097000007EB5171C1F3C70184F87410D0460025EE
:10971000AB4646E030789F2810DD94F87400401B7B
:10972000022808DB04F16000284431880180A81C6D
:10973000C5B2B61C11E04FF0010B0EE094F87400B6
:10974000401B012807DB317804F160004155681C9B
:10975000C5B2761C01E04FF0010BBBF1000F20D029
:109760004FF0000B002104F16000415500200090F3
:1097700094F802C04246531C03F0FF080CEB0211A0
:109780002088012304F16002FDF77CFF0AEB05004D
:109790001FFA80FA0025B8F1050F02DB5046BDE83C
:1097A000F88F30780028B5D1002104F160004155D0
:1097B0000020009094F802C04246531C03F0FF08BA
:1097C0000CEB02112088012304F16002FDF75AFF1F
:1097D0000020E4E710B5094800680949884204D12F
:1097E000FCF7ACFA052006F003FA044800680549C6
:1097F000884202D1052006F0FBF910BD4000002090
:109800002A04EC002A04F40038B50446ACB1FDF794
:1098100045FC012109A004F0F7FC0BA004F00CFEAC
:1098200001236E229F210020FDF7F0FC0020012380
:1098300009A272210090FDF725FF38BDCFFBCFA212
:10984000B8F1CABDBBAF0000C8B7B6A8C9BEB3FD6A
:10985000CBF9D3D0A3BF00005B4D5DC8B7B6A8203D
:10986000205B455849545DC8A1CFFB0010B5104896
:10987000FFF7BCFD04460F4884420ED10C484079E6
:1098800010B1012808D103E00A2006F0B1F903E085
:109890000B2006F0ADF900BF08E007480068074953
:1098A000884203D10649487806F0A2F910BD0000AD
:1098B000AC0000202A04EC00400000202A04F40040
:1098C000CC02002038B50446E4B1FDF7E7FB0121E6
:1098D0000DA004F099FC01236E229F210020FDF7CA
:1098E00095FC0C490C48FFF72DFD01236E229F21AA
:1098F0000020FDF78BFC0020012308A272210090BC
:10990000FDF7C0FE38BD0000CEC4B1BED1A1CFEE80
:1099100000000000F4010020AC0000205B4D5DC899
:10992000B7B6A820202020205B455849545DCDCBF8
:10993000B3F6000010B51C4800681C49884203D1EA
:10994000052006F055F92EE01748006818498842AE
:1099500029D0154800681749884224D11648FAF7DB
:1099600061FC1649098888421DD967239F22182166
:109970000020FDF7EDFB104B182208211048FFF7DF
:1099800087FE0D480D4A128881180D48FFF795FE95
:1099900004462CB10948008820440849088002E0A8
:1099A00000200649088010BD400000202A04F40071
:1099B0002A04EC002A04BC00E2250020F00100206B
:1099C0006A25002038B50446002C2DD00020174908
:1099D00008804FF4C8711648FAF7EFFBFDF75EFBFD
:1099E000012114A004F010FC114802F023FE104BDA
:1099F000182208211248FFF74BFE0D480B4A128827
:109A000081180F48FFF759FE0849088001236E228C
:109A10009F210020FDF7FAFB0020012309A27221FB
:109A20000090FDF72FFE38BD00BFFCE7F0010020DD
:109A3000E2250020CFFBCFA2D4C4B6C100000000B5
:109A40006A2500205BCFC25DB7ADD2B3205B45581D
:109A500049545DB7B5BBD80010B51248408810B165
:109A60001148FFF765F8114800681149084450B1E2
:109A7000B0F5002F03D0B0F5402F0FD10AE002203F
:109A800006F0B6F80BE00748408810B1092006F050
:109A9000AFF804E0082006F0ABF800E000BF00BF1C
:109AA00010BD00004025002070280020400000204C
:109AB000D6FB13FF18B10121034A516102E00121D5
:109AC000014A1161704700000010014008B50120F3
:109AD000ADF8000010208DF8030003208DF802007F
:109AE00069460348FCF7BCF90020FFF7E3FF08BD17
:109AF0000010014010B51C4C1C48007800B910BD86
:109B00002EE040F21E21A01C00F07AFD208020886B
:109B100000281BDD1648007800B121E00022A11CBE
:109B2000104605F049F8002012490872A0782B2849
:109B300002D0A0785E2808D1A01C01F03DFF0128CA
:109B400000D10DE0A01CFBF7A5F809E02088002853
:109B500005DA012208A1002005F02EF800E000E05F
:109B6000CFE700BF00BFCAE7121200209302002017
:109B700088020020D00700205175657565463100C8
:109B80002DE9F041B0B000260027594890F8DD01DA
:109B9000C0EB4011574800EB4105554890F8DD01F6
:109BA000C0EB4011534800EB410000F11F04DFF807
:109BB000488152A2642117A808F05EF84C4890F83A
:109BC000DF0120B950A117A8FAF702FB14E0494BB6
:109BD0001F3B51A2502103A808F04EF803A800F043
:109BE0006FFB444B1F3B52A2502103A808F044F8DE
:109BF00003A917A8FAF7ECFA002217A9104604F0F7
:109C0000DBFF4CA2642117A808F036F8287808B1C9
:109C1000207820B93CA117A8FAF7DAFA15E02B460C
:109C200047A2502103A8009408F026F803A800F0EA
:109C300047FB2B4648A2502103A8009408F01CF8CB
:109C400003A917A8FAF7C4FA0126012217A90020D0
:109C500004F0B2FF002E48D041A2642117A808F0FA
:109C60000BF8234890F89B00C0B1012802D00228CD
:109C700019D10EE03DA117A8FAF7AAFA1C48CDE9C0
:109C8000004590F89B303AA2502103A807F0F4FF5A
:109C900016E03DA117A8FAF79BFA00BF3CA117A850
:109CA000FAF796FA00BF3CA117A8FAF791FA104804
:109CB00090F89B303BA2502103A807F0DDFF00BFC6
:109CC00000BF012217A9002004F076FF03A800F0CE
:109CD000F7FA002203A9104604F06EFF00BF00BF90
:109CE000012235A1002004F067FF30B0BDE8F0810B
:109CF0007A1F002078210020121200204163636542
:109D00007373703A00000000756E737570706F7237
:109D1000742D456D7074790041542B4D495050524B
:109D20004F46494C453D312C222573220D0A000037
:109D3000257300002C4E616D652D506173733A00E0
:109D400041545E5050504346473D222573222C22F9
:109D50002573220D0A00000025732C2573000000D6
:109D6000415554482D4C4F47494E3A005041500000
:109D70004154245143504450503D312C25642C25EE
:109D8000732C25730D0A0000434841500000000069
:109D90004E4F4E450000000020446F206E6F7468E7
:109DA000696E67004154245143504450503D312C5A
:109DB00025640D0A00000000417574684C6F6769E6
:109DC0006E20446F6E65000010B586B00446152203
:109DD000E11D2748FAF7D8F90020254908750846FB
:109DE00000798DF81400084640798DF815000020A0
:109DF0008DF8160005A8FAF787FA0C2829D2DFE8B3
:109E000000F01106121D132807141E08281F00BF9A
:109E100000BF02201749087017A21421684607F0F6
:109E20002BFF1CE000BF00BF00BF012011490870DC
:109E300015A21421684607F01FFF10E000BF00BF05
:109E400000200C49087014A21421684607F014FF82
:109E500005E015A21421684607F00EFF00BF00BF01
:109E60006A46034914A007F0F7FE06B010BD0000D3
:109E700044140020900200204348494E415F554E53
:109E800049434F4D5D0000004348494E415F4D4FEF
:109E900042494C455D0000004348494E415F5445EE
:109EA0004C45434F4D5D0000554E4B4E4F572D498D
:109EB000434349445D00000049434349443A257304
:109EC0002025730D0A00000010B50446204602F05C
:109ED000F1FB122204F109010348FAF797F902494C
:109EE00002A007F0B9FE10BD32140020494D4549CB
:109EF0003A25730D0A0000002DE9F0410446724D29
:109F0000AE1C0027714800780D2818D2DFE800F059
:109F1000071827364958D7758896A5B6C800012C6A
:109F20000BD101226AA1002004F046FE6CA000F0D3
:109F3000C7F9012008F0CEFB01E04FF0FF37BEE08B
:109F4000012C05D0012268A1002004F035FE02E0BA
:109F5000304608F0CDF9022008F0BCFBAFE0012C40
:109F600005D0012265A1002004F026FE02E0304663
:109F700008F03CFA032008F0ADFBA0E0012C05D06E
:109F8000012263A1002004F017FE06E0304608F02D
:109F9000C5FAFBF7FBF800F049F9042008F09AFB3A
:109FA0008DE0012C05D001225DA1002004F004FE0B
:109FB00002E0304608F092FA052008F08BFB7EE0C4
:109FC000012C05D001225AA1002004F0F5FD10E07B
:109FD00006F10D00FAF798F941F65831884203D09E
:109FE000062008F077FB6AE0012255A1002004F06A
:109FF000E3FD072008F06EFB61E0012C07D0012291
:10A0000053A1002004F0D8FD02F062FF04E0012219
:10A0100053A1002004F0D0FD082008F05BFB4EE0C7
:10A02000012C02D06FF0010749E0012250A100206D
:10A0300004F0C2FD092008F04DFB40E0012C05D0E2
:10A0400001224EA1002004F0B7FD02E03046FFF7E8
:10A050003BFF0A2008F03EFB31E0012C05D0012235
:10A060004AA1002004F0A8FD04E03046FFF7ACFE52
:10A07000FCF7F0FB0B2008F02DFB20E0012C05D0B5
:10A08000012246A1002004F097FD03E02988304614
:10A0900000F022F9FFF774FD0C2008F01BFB0EE026
:10A0A000012C05D0012241A1002004F085FD04E02F
:10A0B000012243A1002004F07FFD012700BF00BF63
:10A0C0003846BDE8F0810000121200209602002000
:10A0D0004D6F64656D53746172742E2E2E000000F6
:10A0E000415445300D0A00004765744D6F64656D3D
:10A0F0004D6F64756C65206661696C004765744DD1
:10A100006F64656D566572206661696C00000000C1
:10A11000476574506F63566572206661696C000014
:10A12000476574506F63436F6465206661696C00B6
:10A1300053657420545473206661696C00000000FC
:10A140005365745454535370656564204F6B00001D
:10A1500052652D5365742053706B4D696300000088
:10A160005365742053706B4D6963204F6B00000082
:10A1700043617264205265616479000047657449E7
:10A180004D4549206661696C0000000047657449CF
:10A1900043434944206661696C0000004765745080
:10A1A0006F6350617261206661696C005365745021
:10A1B0006F63534D6F6465206661696C0000000039
:10A1C000536574506F63534D6F6465204F6B00008F
:10A1D00010B51348007810B11248007800B110BDD6
:10A1E0001148007818B9012003F078F916E00E48FC
:10A1F0008078002803DD032003F070F90EE00A48A0
:10A200000079002807DD08488079002803DD042054
:10A2100003F064F902E0022003F060F900BFDEE71A
:10A220009202002088020020D007002010B50848C4
:10A230000078012800D010BD06A000F041F800BF52
:10A2400000BF09A000F03CF800BF00BF00BFF2E76C
:10A250009100002041542B504F433D33303030307B
:10A2600030303130300D0A0041542B504F433D30D7
:10A2700033303030300D0A0008B501211C2001F0C8
:10A28000EDFF10208DF8030003208DF8020002205E
:10A29000ADF8000069460948FBF7E2FD0120ADF882
:10A2A000000069460548FBF7DBFD02200349103139
:10A2B00008600120091D086008BD0000000C014075
:10A2C00070B504462046F9F7ADFF85B22946204611
:10A2D00007F05AF970BD00002DE9F043A3B0044621
:10A2E0000D4600260027B0460021E81E21542146D5
:10A2F00004F10D00FAF76CFC05460020605519AA20
:10A3000042A12046FCF764FC05464148D0F81D30C8
:10A3100040A26421684607F0AFFC19A96846F9F726
:10A3200088FF00B1012619AA3BA12046FCF750FC8A
:10A33000054608F0A7F881464B4638A264216846D6
:10A3400007F09AFC19A96846F9F773FF00B10127D5
:10A3500019AA33A12046FCF73BFC0546314B2FA23E
:10A360006421684607F088FC19A96846F9F761FF7F
:10A3700008B14FF001085EB957B9B8F1000F07D125
:10A38000012229A1002004F017FC23B0BDE8F083CE
:10A3900028A0FFF795FF76B11D48D0F81D3029A2FF
:10A3A000282119A807F068FC694619A8FAF7C5FB27
:10A3B0006846FFF785FF7FB108F064F881464B4699
:10A3C00022A2282119A807F057FC694619A8FAF714
:10A3D000B4FB6846FFF774FFB8F1000F0CD0114BC7
:10A3E0001CA2282119A807F047FC694619A8FAF70A
:10A3F000A4FB6846FFF764FF18A0FFF761FF012286
:10A4000017A1002004F0D8FB00BFBEE7696400007C
:10A41000381F0020256C750069700000257300004E
:10A42000707764006A1F0020504F43207374696C7A
:10A430006C00000041542B504F433D3031303030E0
:10A440003000000069643D256C753B0069703D2556
:10A45000733B00007077643D25733B000D0A0000DC
:10A460005273745F504F43506172610070B58AB08F
:10A47000064626B1012E05D0022E09D105E005249D
:10A48000192507E00524372504E00524052501E00A
:10A490000AB070BD00BF234607A21E2102A8009586
:10A4A00007F0EAFB02A8FFF70BFF002202A9104603
:10A4B00004F082FB00BFEBE741542B5544503D258F
:10A4C000642C25640D0A000030B502460B4619467F
:10A4D000144607E008782578A84201D0012030BD55
:10A4E000491C641C08780028F4D100BFF7E700007D
:10A4F0002DE9F0470546002734480468002640F25D
:10A500003138DFF8CC90042032490861002C00DAA1
:10A5100055E031484068A04200D850E015B1002015
:10A5200009F094FB06EB080104EB440000EBC402C5
:10A530002948083000EB8200406A81420AD904EBC6
:10A54000440000EBC4012448083000EB8100406A5D
:10A55000871B00E04746FDF78BF904EB440101EB54
:10A56000C4021D49083101EB82000021FAF760FDA9
:10A5700004EB440101EBC4021749083101EB8200EE
:10A580004B463A46314600F029F804EB440101EB12
:10A59000C4021149083101EB820007F071F804EBA5
:10A5A000440101EBC4020C49083101EB8200012196
:10A5B000FAF73EFD15B1012009F048FB00BF042069
:10A5C000044948613846BDE8F08700009C0000203F
:10A5D0007A1F002000100140082F00202DE9F041D3
:10A5E00080460C4615461E4604482718AAB239462E
:10A5F000304609F071FABDE8F081000000F01F005C
:10A60000F8B505460B462B49888808B90020F8BDE7
:10A610004F88881D30F82700ADF800004F88881D4E
:10A6200000EB87004088ADF802000024002220E003
:10A63000B1F8D00000B920E0CE31D1F80A00CF88BF
:10A64000C65DC888401CC880C88831F8CE79B84239
:10A6500002DB0020A1F8D400B1F8D000401EA1F820
:10A66000D0009C4203DA2046671CBCB22E54501C1A
:10A6700082B2BDF800009042DADC00BF4888401C7E
:10A6800048804888322801DB002048808888401EA6
:10A690008880BDF80000904202D06FF00100B6E75C
:10A6A000BDF80000984202DD4FF0FF30AFE7BDF883
:10A6B0000000ACE75C1E002030B503460A46124895
:10A6C0000024048084804480002108E00025841D4B
:10A6D00004EB81046580841D24F82150491C322933
:10A6E000F4DBC0F8D830002104E00024D0F8D850C2
:10A6F0006C54491C9142F8DB20F8CE2F0024848052
:10A70000C4804480CE3830BD5C1E002070B5044645
:10A710000A4622498888322802DB4FF0FF3070BD9C
:10A72000B1F8D0001044B1F8CE50A84202DD6FF06D
:10A730000100F4E7B1F8D2500E88881D00EB8600C6
:10A7400045800D88881D20F82520002317E0E05C57
:10A75000D231D1F806500E88A8550888401C0880D0
:10A7600031F8D209B0F5206F02DB0020A1F8D20049
:10A77000B1F8D000401CA1F8D000581C83B293421D
:10A78000E5DB0888401C08800888322801DB0020AF
:10A7900008808888401C88800020C0E75C1E00205C
:10A7A00000B54FF420610248FFF786FF00BD0000AE
:10A7B0005C1400207047000070B5002100230F22B8
:10A7C000C47804B3154C246804F4E064C4F5E06470
:10A7D000210AC1F10403CA40447804FA03F18478E1
:10A7E0001440214309010E4C0678A155047804F069
:10A7F0001F050124AC4005786D11AD0005F1E02581
:10A80000C5F8004109E0047804F01F050124AC40BC
:10A81000044D0678761145F8264070BD0CED00E039
:10A8200000E400E080E100E002490143024A1160D7
:10A83000704700000000FA050CED00E02DE9F04142
:10A8400004460D4616461F462580A670142239463A
:10A85000E01CF9F7DBFCE01CF9F7E4FC6076607EB5
:10A86000C006000EA0761020E07600202076BDE81D
:10A87000F081000070B50446217EE01C455C16485E
:10A8800000681649084498B1B0F5001F03D0B0F530
:10A89000601F1ED11BE0392D02DA681CC5B200E032
:10A8A0003025217EE01C4554204600F019F810E0C8
:10A8B000217E607E401E814203DA207E401C20768D
:10A8C00001E000202076204600F00AF801E0022096
:10A8D00070BD00BF0020FBE740000020D6FB43FF17
:10A8E0002DE9FC410446A77894F81BC06744103F4B
:10A8F000BBB2278894F81AC06744BAB2A1782088FE
:10A90000FCF726FC207EC50000200090A17820885E
:10A910000123E21CFCF7B6FE2088284485B221887A
:10A92000681AC11700EB5171C1F3C706E01C805DC6
:10A930008DF8040000208DF8050001200090A1781A
:10A94000034601AA2846FCF79DFEBDE8FC810000F5
:10A950000EB50121084601F081FC04208DF80300AA
:10A9600003208DF802004FF40070ADF80000694636
:10A970000B48FBF775FA09210120FBF751FA4FF458
:10A980000070019000208DF8080008208DF8090063
:10A9900001208DF80A0001A8FAF79EFE0EBD000006
:10A9A000000C014010B51448FFF764FF134800681D
:10A9B0001349884216D1062212490F48C01CF9F7E4
:10A9C00046FC18B9122005F013F90BE00EA003F0B5
:10A9D00033FD322009F039FB01200E4908610620C1
:10A9E00005F006F9054800680B49884202D10620A7
:10A9F00005F0FEF810BD0000722700204000002086
:10AA00002A04EC0094000020C3DCC2EBB4EDCEF3CA
:10AA100000000000582800202A04F400F0B5A7B078
:10AA200000272E48FEF72CF806462D48864203D113
:10AA3000062005F0DDF84FE02A4886424CD1274831
:10AA4000847929480078012803D0022C01DBA01C5E
:10AA5000C4B2264890F89C00A0423AD0234880F81F
:10AA60009C4023A003F0E8FC0020FFF741FD07F025
:10AA700011FC07F007FD054607F0F2FB07461A48F0
:10AA80000078012807D12B461CA232211AA8009772
:10AA900007F0F2F808E01E480095D0F81D301DA21E
:10AAA00032211AA807F0E8F801A91AA8FAF745F820
:10AAB0001CA0FFF705FC01A8FFF702FC1DA0FFF793
:10AAC000FFFBFCF7D5FE142009F0BFFA1AA0FFF730
:10AAD000F7FB012005F08CF827B0F0BD70280020AE
:10AAE0002A04F4002A04EC00910000207A1F0020C0
:10AAF000C5E4D6C3CDEAB3C90000000069703D25A6
:10AB0000733B646F6D61696E3D25733B000000000F
:10AB1000381F002069643D256C643B69703D2573D6
:10AB20003B00000041542B504F433D30313030301A
:10AB3000300000000D0A000041542B504F433D30BF
:10AB400034303030300D0A0070470000014608688C
:10AB5000034A1268904201D8012070470020FCE7A8
:10AB6000AC030020024B1B6813440B6070470000CD
:10AB7000AC03002002490968491C014A1160704772
:10AB8000AC0300202DE9F84F05460C4616461F463B
:10AB9000A02D01DA802C01DBBDE8F88FA819A028D0
:10ABA00002DDC5F19F0086B2E019802802DDC4F104
:10ABB0007F0087B2FCF75CFE0A984FEA8009194BC8
:10ABC00013F809209C4609F101031CF803105B1CD3
:10ABD0001CF8030001F0E4FB8246E019401E83B23A
:10ABE000A819401E82B221462846FDF747FB4FF0C8
:10ABF000000813E004EB080000904FF0000B09E0A0
:10AC00004FEA2A20FDF722FD0AF0FF00FDF71EFDA6
:10AC10000BF1010BB345F3DB08F10108B845E9DBA3
:10AC200000BFB9E7082B00202DE9FF4F95B0239C0A
:10AC3000229800F0F0001090229800F00F000F9082
:10AC40004FF0000B179848BB109840B94FF0080917
:10AC50000C254FF0010A7E4FDFF8F88107E04FF036
:10AC6000080910254FF0010A7B4FDFF8F0810BE057
:10AC700098F800101898814200D109E008F1010805
:10AC80000BF101001FFA80FB98F800000028EFD1BB
:10AC900000BF0BFB0AF000FB057728E0109898B97D
:10ACA0004FF010090C254FF0020A01AF4FF00008D9
:10ACB0004FF0000B01AA109BDDE91701FBF70AFD1D
:10ACC000182814D0664F12E04FF0100910254FF0ED
:10ACD000020A07AF4FF000084FF0000B07AA109BC5
:10ACE000DDE91701FBF7F6FC202800D05C4F169831
:10ACF0002844802802DB19B0BDE8F08F159848443D
:10AD0000A02800DBF7E716982844401E83B2159868
:10AD10004844401E82B2DDE91501FDF7AFFA00207C
:10AD200013908EE013991698084486B20020149070
:10AD30007FE0DDE9140101EBC00080B2129017F84A
:10AD4000010B11904FF0000B6CE0802040FA0BF0EB
:10AD50001199084080B30D2E0ADA24B941480078D1
:10AD600006F0A8FD5AE04048007806F0A3FD55E043
:10AD70001B2E0ADA24B93B48007806F09BFD4DE013
:10AD80003A48007806F096FD48E06E2E09DA1CB9C4
:10AD9000002006F08FFD41E03248007806F08AFD81
:10ADA0003CE024B93048007806F084FD36E02D48B8
:10ADB000007806F07FFD31E0FFE70D2E0ADA24B9B6
:10ADC0002948007806F076FD28E02648007806F04D
:10ADD00071FD23E01B2E0ADA24B92448007806F01E
:10ADE00069FD1BE02048007806F064FD16E06E2E39
:10ADF0000ADA24B91B48007806F05CFD0EE01C4816
:10AE0000007806F057FD09E024B91648007806F0EE
:10AE100051FD03E01448007806F04CFD0BF10100F1
:10AE20001FFA80FBBBF1080F8FDB1498401C80B227
:10AE3000149014985045FFF67CAF1398401C80B2D4
:10AE400013901398A842FFF66DAF00BF53E70000C0
:10AE5000604E0108044E010890420108304201088A
:10AE600080480108A00300209F0300209E030020CB
:10AE7000A10300202DE9F04F87B0894616469A4677
:10AE8000109F002533E009EB0500059005FB06F057
:10AE90000690002428E004EB4400385C039004EBA7
:10AEA0004400401C385C049004EB4400801C17F8FC
:10AEB00000B04FEAEB0002900498801001900398D4
:10AEC000C01000900298C102019801EB4011009857
:10AED00008441FFA80F84FEA2820FDF7B7FB08F076
:10AEE000FF00FDF7B3FB641CB442D4DB6D1C554579
:10AEF000C9DB07B0BDE8F08F2DE9F04104460E46EE
:10AF000017469846234800682349884202D02348C0
:10AF1000006960B1214801F047F9C5B2042D01DD97
:10AF2000E56000E0E56000201C49086106E0194882
:10AF300000681B49884201D10020E060C4F800800D
:10AF40006660A7603520208233206082208A28280E
:10AF500008DD218AA1F1280000EBD071C1F34F0177
:10AF6000A18201E00020A082608A282808DD618A91
:10AF7000A1F1280000EBD071C1F34F01E18201E0A3
:10AF80000020E08200221146204600F053F8BDE880
:10AF9000F0810000400000202A04F400582800201E
:10AFA0002A04EC0010B504462048006820490844F3
:10AFB000E8B1B0F5001F06D0B0F5401F2CD0B0F5B9
:10AFC000601F2DD129E04FF0FF312046E26800F0EC
:10AFD00031F8E06818B1E068401EE06001E005204B
:10AFE000E06001212046E26800F024F818E04FF00C
:10AFF000FF312046E26800F01DF8E068052803D222
:10B00000E068401CE06001E00020E0600121204693
:10B01000E26800F00FF803E002E00020207600BFB5
:10B0200000BF0248008880B210BD00004000002030
:10B03000D6FB43FF2DE9F04786B006468946924687
:10B04000B9F1000F70D1FCF729F8F268716851F876
:10B0500022000D2103F0D8F8002784E04FF000080B
:10B060007CE0308A00FB08F0B18A4418708A78438B
:10B070001930F18A451807EB470000EB080394A14B
:10B0800001A8B26806F00CFE07EB47014144F068E6
:10B0900088424AD1A9B2A0B201AAFCF792FA0220D2
:10B0A000ABB204F1290C1FFA8CF2A5F1010C1FFAC6
:10B0B0008CF1A4F1010C00901FFA8CF0FCF704F95C
:10B0C000022005F1290C1FFA8CF304F1290C1FFA58
:10B0D0008CF205F1280C1FFA8CF1A4F1010C009000
:10B0E0001FFA8CF0FCF7F0F8022005F1280C1FFA8B
:10B0F0008CF3A2B2A9B2A4F1010C00901FFA8CF05B
:10B10000FCF7E2F8022005F1280C1FFA8CF304F199
:10B11000290C1FFA8CF2A9B204F1280C00901FFA36
:10B120008CF0FCF7D1F817E023E005F1290C1FFAA9
:10B130008CF304F1290C1FFA8CF2A5F1010C1FFA13
:10B140008CF1A4F1010C1FFA8CF0FCF701F8A9B204
:10B15000A0B201AAFCF735FA08F10108B8F1030F13
:10B16000FFF67FAF7F1C022FFFF678AF012030760D
:10B17000ABE0F268716851F822000D2103F044F849
:10B1800003209AFBF0F79AFBF0F100FB11A8308A3C
:10B1900000FB08F0B18A4418708A78431930F18AAC
:10B1A0004518B9F1000F44DD0220ABB204F1290CBF
:10B1B0001FFA8CF2A5F1010C1FFA8CF1A4F1010C1D
:10B1C00000901FFA8CF0FCF77FF8022005F1290CA3
:10B1D0001FFA8CF304F1290C1FFA8CF205F1280CEC
:10B1E0001FFA8CF1A4F1010C00901FFA8CF0FCF70F
:10B1F0006BF8022005F1280C1FFA8CF3A2B2A9B259
:10B20000A4F1010C00901FFA8CF0FCF75DF802200D
:10B2100005F1280C1FFA8CF304F1290C1FFA8CF2AB
:10B22000A9B204F1280C00901FFA8CF0FCF74CF83E
:10B230003BE0ABB204F1290C1FFA8CF2A5F1010C32
:10B240001FFA8CF1A4F1010C1FFA8CF0FBF780FFC0
:10B2500005F1290C1FFA8CF304F1290C1FFA8CF26A
:10B2600005F1280C1FFA8CF1A4F1010C1FFA8CF0E7
:10B27000FBF76EFF05F1280C1FFA8CF3A2B2A9B2FE
:10B28000A4F1010C1FFA8CF0FBF762FF05F1280C0A
:10B290001FFA8CF304F1290C1FFA8CF2A9B204F105
:10B2A000280C1FFA8CF0FBF753FF307E68B907EBD0
:10B2B000470000EB080306A101A8B26806F0F0FC05
:10B2C000A9B2A0B201AAFCF77CF906B0BDE8F087EC
:10B2D000257325642E626D70000000002DE9F04F8B
:10B2E000D9B0824600270020129011903822FC49E4
:10B2F00003A8F8F749FF00BF3846791C0FB203A92D
:10B3000051F8200000780028F6D1781E07B20025F9
:10B3100023E003A850F825900AF1030B0020579072
:10B32000589010E099F800009BF80010884202D075
:10B33000012057900BE009F101090BF1010B58981E
:10B34000401C00B2589099F800000028EAD100BFD4
:10B35000579800B903E0681C05B2BD42D9DB00BFB5
:10B36000BD4202D159B0BDE8F08F0D2D7ED2DFE88D
:10B3700005F007162494A8FEFDFCFBFAF9F8F70087
:10B380000122D8A1002003F017FC092002F0D6F812
:10B390000220F9F7A3FF0120D5490870EBE2012252
:10B3A000D4A1002003F008FC092002F0C7F8FAF746
:10B3B000BDFE0120F9F792FFDDE231AAD0A150468F
:10B3C000FBF706FC0446012C01DB282C05DB0122DF
:10B3D000CCA1002003F0F0FBCDE231A927A8F8F7BB
:10B3E00043FF31AACDA15046FBF7F2FB04460CB94E
:10B3F00000260BE0052C05DD0122CAA1002003F088
:10B40000DBFBB8E231A8F8F77FFF86B231AACCA106
:10B410005046FBF7DDFB0446012C01DB0A2C05DD61
:10B420000122C8A1002003F0C7FBA4E231A8F8F76D
:10B4300078FF8046CA48D0F81D00404504D0C8486F
:10B44000C0F81D8001201290C64890F89C00042886
:10B4500005D00420C34981F89C000120119027A940
:10B46000C148F8F7E6FE38B127A900E082E2BE48FD
:10B47000F8F7FAFE01201190B948D0F81D00BA4B38
:10B48000BAA29621CDE9006031A806F0F5FB0122B1
:10B4900031A9002003F090FB6DE206F0F3FFBB49F9
:10B4A0000290CDE90010AE48D0F81D30B8A2962128
:10B4B00031A806F0E1FB012231A9002003F07CFB5A
:10B4C00059E231AA8EA15046FBF782FB0446012CBB
:10B4D00001DB282C05DB0122BDA1002003F06CFB61
:10B4E00049E231A927A8F8F7BFFE31AA8BA150463F
:10B4F000FBF76EFB04460CB900260BE0052C05DDBE
:10B500000122B9A1002003F057FB34E231A8F8F77B
:10B51000FBFE86B2934890F89C00042805D00420D6
:10B52000904981F89C000120119027A98E4828306D
:10B53000F8F77FFE20B98B48B0F82E03B04209D04F
:10B5400027A989482830F8F78FFE8648A0F82E638F
:10B55000012011908348B0F82E03834B283307E075
:10B56000FBE1E9E1DCE1ADE056E048E01DE00BE0A5
:10B57000A4A29621009031A806F07EFB012231A9F9
:10B58000002003F019FBF6E17648B0F82E03764B65
:10B590002833A2A29621009031A806F06DFB01226B
:10B5A00031A9002003F008FBE5E131AAA1A1504632
:10B5B000FBF70EFB0446002C01DB1E2C05DD0122EF
:10B5C0009EA1002003F0F8FACCE624B900216548DA
:10B5D00080F8DF1104E031A96348A230F8F744FE97
:10B5E000614BA2339DA2962131A806F045FB0122B2
:10B5F00031A9002003F0E0FA01201190BBE15A4B81
:10B60000A2339BA2962131A806F036FB012231A974
:10B61000002003F0D1FAAEE131AA9AA15046FBF71F
:10B62000D7FA0446012C01DB1E2C05DD012297A16F
:10B63000002003F0C1FA95E631A91DA8F8F714FE21
:10B6400031AA9AA15046FBF7C3FA0446012C01DB4C
:10B650001E2C05DD012298A1002003F0ADFA81E641
:10B6600031A913A8F8F700FE13A81DAB9AA29621E2
:10B67000009031A806F000FB012231A9002003F060
:10B680009BFA9D480068002800DA74E19B491DA8D8
:10B69000F8F7CFFD30B999491F3113A8F8F7C9FD64
:10B6A00000B968E11DA99548F8F7DEFD13A9934894
:10B6B0001F30F8F7D9FD03202A4981F8DD01012068
:10B6C000119058E18D4B1F338C4A8DA131A806F0A3
:10B6D000E7FA012231A9002003F06EFA4BE10000E5
:10B6E000A841010847542B544D3A4F4B000000002D
:10B6F0007E02002047542B54473A4F4B0000000075
:10B700004950000047542B534D503A4641494C5B39
:10B71000495020496E76616C69645D00506F7274A7
:10B720000000000047542B534D503A4641494C5BB2
:10B73000506F727420496E76616C69645D00000020
:10B7400050534E0047542B534D503A4641494C5BA1
:10B7500050534E20496E76616C69645D00000000B4
:10B76000381F00207A1F0020B720002047542B5399
:10B770004D503A49503D25733B506F72743D2575CD
:10B780003B50534E3D256C75000000006A1F0020A1
:10B7900047542B524D503A50534E3D256C753B4DFE
:10B7A0004549443D25733B434E554D3D3030303087
:10B7B0003030303030303B55494D49443D303030E9
:10B7C000303030303030303B49503D25733B000045
:10B7D00047542B5347503A4641494C5B4950204906
:10B7E0006E76616C69645D0047542B5347503A464E
:10B7F00041494C5B506F727420496E76616C69648C
:10B800005D00000047542B5347503A49503D257383
:10B810003B506F72743D25753B00000047542B521E
:10B8200047503A49503D25733B504F52543D256493
:10B830003B000000416363657373700047542B53F2
:10B840004143433A4641494C5B41636365737370BE
:10B8500020496E76616C69645D00000047542B538B
:10B860004143433A416363657373703D25733B0005
:10B8700047542B524143433A416363657373703DB0
:10B8800025733B004163636F756E740047542B4111
:10B89000504E3A4641494C5B4163636F756E74206C
:10B8A000496E76616C69645D0000000050617373DD
:10B8B000776F72640000000047542B41504E3A46A7
:10B8C00041494C5B50617373776F726420496E76A7
:10B8D000616C69645D00000047542B41504E3A4151
:10B8E00063636F756E743D25733B50617373776F3F
:10B8F00072643D25733B00009C0000203222002032
:10B9000047542B5241504E3A4163636F756E743DFC
:10B9100025733B50617373776F72643D25733B00F1
:10B9200064224FF4601131A808F060F8012231A9B7
:10B93000002003F041F91EE01548B0F82F00144B29
:10B94000213314A29621009031A806F095F9012226
:10B9500031A9002003F030F90DE0124812A296211F
:10B96000036831A806F088F9012231A9002003F00C
:10B9700023F900BF00BF00BF129808B101F04EF8D4
:10B98000119810B10020FEF7B3FD00BFEAE40000FB
:10B99000381F002047542B5645523A25735F5625D1
:10B9A00064000000D801002047542B4241543A2043
:10B9B0002564205600000000F0B5BBB004464821C5
:10B9C0000BA8F8F7FAFB60784C2818D1A078532818
:10B9D00015D1E078482812D1207954280FD1607A07
:10B9E00045280CD10020FB49C8700846807818B95A
:10B9F0004FF48070F849486101203BB0F0BD607998
:10BA0000302827D1A079422824D1E07946280DD1C9
:10BA1000207A46280AD10020F049087003F086F900
:10BA20000A214FF47A7001F03BF911E0E0793028F7
:10BA30000ED1207A30280BD10120E6490871E74960
:10BA4000087003F073F90A214FF4FA7001F028F935
:10BA50000120D2E7607938287FD1A07942287CD1B3
:10BA6000E079302879D1207A312814D106F0C4FB4E
:10BA70000120D8490871D84948610020D54988700B
:10BA8000D648007818B94FF48070D3494861012036
:10BA9000D049087008E0207A302805D10020CD492F
:10BAA00008710120CC490861607A30281CD1A07A45
:10BAB000302819D1C948007801280AD10020C74987
:10BAC0000870C448807810B10020C24988700120F5
:10BAD00093E70020BF49887003F028F90A214FF44A
:10BAE000FA7001F0DDF835E0607A30281AD1A07ADA
:10BAF000312817D106F080FB0120FCF797FB0020CE
:10BB0000B74908800120B3490870887003F00EF926
:10BB1000B44890F8F802E8B10A214FF4FA7001F045
:10BB2000BFF817E0607A312814D1A07A332811D1F8
:10BB3000AA480078012802D10020A84908700120F5
:10BB4000A44981F8B00603F0F1F80A214FF47A70A5
:10BB500001F0A6F8012050E7FFE7607938286ED1A0
:10BB6000A0793228FBD1E0798DF87800207A8DF821
:10BB7000790000208DF87A001EA8F8F7C5FBC7B23F
:10BB800037B1012F7ED0022F70D0032F6FD1ADE0DF
:10BB90000020904981F8AF0608709348007820F0A3
:10BBA00010009149087091A266211EA806F064F861
:10BBB000607C422814D1A07C352811D1607E4328B6
:10BBC0000ED1A07E41280BD105208A4908700120A2
:10BBD000804981F8B30688A11EA8F8F7F9FA4BE06E
:10BBE000607C432816D1A07C452813D1607E432871
:10BBF00010D1A07E32280DD1764890F8B3060128E6
:10BC000003D00220734981F8B3067FA11EA8F8F77C
:10BC1000DFFA31E0607C432812D1A07C45280FD1A7
:10BC2000607E43280CD1A07E312809D105206949C6
:10BC300081F8B30677A11EA8F8F7CAFA1CE05EE007
:10BC4000607C432814D1A07C332811D1607E422827
:10BC50000ED1A07E37280BD106205E4981F8B306AD
:10BC60006FA11EA8F8F7B4FA06E00BE010E043E07D
:10BC70006EA11EA8F8F7ACFA01221EA9002002F05E
:10BC80009BFF39E001226CA1002002F095FF33E018
:10BC900004F11100F8F7C6FA801EC5B2242D00DBAE
:10BCA00024252A4604F111016648F8F76DFA0020B0
:10BCB0006449485547491531624803F075F800203A
:10BCC000607410221DA904F10900F8F7E5FA414952
:10BCD000086101225CA1002002F06EFF01205D4995
:10BCE000087003203B4981F8B30605E001225AA100
:10BCF000002002F061FF00BF00BF01207DE620466A
:10BD0000FAF74EFA08B1012077E66079382860D159
:10BD1000A07936285DD101202E4908701E203549B2
:10BD20000870207A30284DD104F11100F8F77AFA22
:10BD3000801EC5B2242D00DB24252A4604F1110102
:10BD400001A8F8F721FA002001A9485560741022D3
:10BD50001DA904F10900F8F79FFA1E49C863423192
:10BD600001A803F021F81B484078C8B93948007889
:10BD700030B901AB3BA266211EA805F07DFF0AE0A9
:10BD800000203449087001A82E4B37A2662100908C
:10BD90001EA805F071FF1EA90120FDF7AFFA11E002
:10BDA0003748007801280DD1002035490870094B2B
:10BDB000423334A266211EA805F05EFF1EA90120B1
:10BDC000FDF79CFA0020034981F8AF060120487076
:10BDD00013E65FE0D0070020001001408100002042
:10BDE000A40000207A1F0020C02200205B6D736732
:10BDF0005D0000007C020020D5CBBAC5D0C5CFA223
:10BE0000B4EDCEF300000000CEDECDF8C2E7C1AC49
:10BE1000BDD30000CEDEB7A8C1ACBDD3000000008A
:10BE2000C3BBD3D0B7FECEF1000000004E6F206C34
:10BE30006F67696E000000006C6F67696E20696E45
:10BE400067000000CC0F00206C6F67696E206F6B7D
:10BE500000000000800000206C6F676F757420691F
:10BE60006E6700002573000025733243443244316D
:10BE700042354337433242443243257300000000C9
:10BE80007D02002042444638433845423243257300
:10BE900000000000607938282BD1A079332828D100
:10BEA000E079302825D1207A302822D104F1110000
:10BEB00000F000FC04F11100F8F7B4F90646242E56
:10BEC00001DB242600E0761C8D4904F1110002F00C
:10BED0006BFF0020607410221DA904F10900F8F71F
:10BEE000DBF987497439C1F89C0000206074012097
:10BEF00083E5607938280AD1A079332807D1E07921
:10BF0000302804D1207A312801D1012075E56079EB
:10BF1000392804D1A079312801D101206DE560795B
:10BF2000302825D1A079452822D1002060743AA973
:10BF300004F10D0002F038FF9DF8E9008DF8E400EF
:10BF40009DF8EA008DF8E500BDF8E4006C4974390D
:10BF50008881012081F86C000846838969A26621E6
:10BF60001EA805F089FE01221EA9002002F024FE71
:10BF70006079382832D1A07934282FD12046FDF7B6
:10BF8000A9F904F109010120FDF7B8F9082260A11F
:10BF900004F10900F8F75BF928B901205849743910
:10BFA00081F8AF0618E008225CA104F10900F8F757
:10BFB0004EF928B900205249743981F8AF060BE0D8
:10BFC000102259A104F10900F8F741F920B9012024
:10BFD0004B49743981F8AF0601200EE560793228AB
:10BFE0006ED1A07931286BD12046FDF773F9444812
:10BFF000743890F86B0000EB400101EBC001404841
:10C000002C3000EB81000021C0F805104172607DEA
:10C0100070B920213A48743890F86B0000EB400268
:10C0200002EBC00236482C3000EB8200417110E078
:10C030003348743890F86B0000EB400202EBC0020A
:10C040002F482C3000EB8200411D04F1150002F056
:10C05000ABFE002060753AA904F10D0002F0A4FEC9
:10C060009DF8E8008DF8E3009DF8E9008DF8E20006
:10C070009DF8EA008DF8E1009DF8EB008DF8E000F6
:10C080001F48743890F86B0000EB400202EBC002CE
:10C090001B482C30389940F822100321A03890F822
:10C0A0006B0000EB400202EBC00215482C3000EBA5
:10C0B0008200017101201249743981F86A009CE400
:10C0C000607931281AD1E079302817D1A07B372840
:10C0D00002D0A07B382811D11848D4F8131041623F
:10C0E000D4F81710816204F11F00FDF7F3F804F192
:10C0F0001F010120FDF702F901207EE400BF7CE46E
:10C10000440800206F6E654C696E653A2564000036
:10C11000433144394341423100000000434443422B
:10C120004233463600000000424146344244443027
:10C13000423343394239413600000000500E00209E
:10C1400008B501211C2000F089F810208DF80300AB
:10C1500003208DF802000420ADF800006946034872
:10C16000F9F77EFE04200149486108BD0010014036
:10C1700010B50B48007800B910BD042009490861CA
:10C180000120FCF753F84FF40070064908610020C5
:10C1900005F0F0FF04200349486100BFFEE70000FE
:10C1A0007F0200200010014070B50446606900283D
:10C1B00005DA07A005F050FD4FF0FF3070BD606953
:10C1C00054F820506069401E60612846F6E7000080
:10C1D000737461636B20697320656D7074790D0AE7
:10C1E0000000000070B504460D466069042804D1C3
:10C1F00006A005F031FD012070BD6069401C606142
:10C20000606944F820500020F6E700007374616311
:10C210006B2066756C6C0D0A0000000029B1064A9F
:10C2200052690243044B5A6104E0034A5269824353
:10C23000014B5A61704700000010024029B1064AC4
:10C24000D2690243044BDA6104E0034AD2698243B3
:10C25000014BDA61704700000010024029B1064A24
:10C2600092690243044B9A6104E0034A9269824353
:10C27000014B9A6170470000001002400348406A79
:10C2800040F0807001494862704700000010024091
:10C2900030B500210022002400232D4D6D6805F0EB
:10C2A0000C0121B1042905D0082923D105E0294D2D
:10C2B000056022E0274D05601FE0254D6D6805F4FF
:10C2C0007012234D6D6805F48034022505EB92420F
:10C2D0001CB9214D554305600BE01D4D6D6805F4FB
:10C2E00000351DB11C4D5543056002E0194D554305
:10C2F000056002E0174D056000BF00BF144D6D687A
:10C3000005F0F0010909154D6B5C0568DD404560DD
:10C310000F4D6D6805F4E061090A104D6B5C4568CE
:10C32000DD4085600A4D6D6805F46051C90A0B4D0A
:10C330006B5C4568DD40C560054D6D6805F44041A6
:10C34000890B074D6B5CC568B5FBF3F5056130BD26
:10C3500000100240001BB700808D5B000000002031
:10C360001000002010B501460022002300204A11D1
:10C37000012A02D1094C236806E0022A02D1074CA7
:10C38000236A01E0054C636A01F01F020124944016
:10C390001C400CB1012000E0002010BD0010024044
:10C3A00070B50346DC108D10D610E00200EB45108E
:10C3B000304480B270BD00004FF4FA600449088038
:10C3C00001208870C870002008714871887170471A
:10C3D000040200200E488079401CC0B20C498871CC
:10C3E0003C2813DB0020887108464079401CC0B20D
:10C3F00048713C280ADB0020487108460079401C3F
:10C40000C0B20871182801DB0020087170470000D5
:10C41000040200200949098801800849897881704F
:10C420000649C978C17005490979017103494979FB
:10C43000417102498979817170470000040200202E
:10C4400038B5002407E01E481E4941F824000020AA
:10C450001D490855641C052CF5DD002416E004EB8D
:10C46000440000EBC401194800EB81000079401E34
:10C470001549085504EB440000EBC401134800EBD8
:10C480008100401D0F4941F82400641C0F48A0386A
:10C4900090F86B00A042E2DC0C48A038808928B9F3
:10C4A0000BA0084908600020074908550648094BB9
:10C4B0000022044900900848FCF70CFA38BD00003F
:10C4C0006C030020D82A00206D0300207008002093
:10C4D000BFD500005C030020702800202DE9F04744
:10C4E00004460D4617469846002C02DA0020BDE8A7
:10C4F000F08719484068A04201D80020F7E7E91901
:10C5000004EB440000EBC4021348083000EB820047
:10C51000406A81420AD904EB440000EBC4010E4892
:10C52000083000EB8100406A461B00E03E4604EB09
:10C53000440000EBC4010848083000EB8100806A29
:10C5400000EB050909F58059B2B24946404607F0AB
:10C550004DFA3046CBE70000082F0020F0B5054625
:10C560000B461646002700240DE0281900F051FA6A
:10C57000024638467F1C1A544FEA122C38467F1C5C
:10C5800003F800C0A41CB442EFDBF0BD10B50024DA
:10C59000FBF76EF932221C491C48FFF7DFFF1A48EF
:10C5A000D0F81D001A49884208D31748D0F81D104A
:10C5B0000022184B591A72EB020009DA1248D0F81F
:10C5C0001D1015A005F048FB00200F49C1F81D0003
:10C5D0000D48B0F82F0040F29511884204D008466B
:10C5E0000949A1F82F00012410A107482130F7F7CD
:10C5F00020FE28B10DA104482130F7F735FE0124B3
:10C600000CB100F00BFA10BD381F002000F8010833
:10C6100040420F0000EA56FA50534E20696E766190
:10C620006C69643A25780D0A0000000048533139DE
:10C63000314C00007FB504466D461C48C2881C483A
:10C6400000EB8200006800F110014FF4C872204630
:10C6500007F0CCF91548C288154800EB8200016844
:10C660000222284607F0C2F900208DF801000F4889
:10C67000C2880F4800EB820001680222284607F0BA
:10C680002BFA0B481638808870B109481638808814
:10C69000401E0749163988800846808820B9084618
:10C6A000007820F0010008707FBD00007028002095
:10C6B000562500200246114607E00D2801D00A2821
:10C6C00002D100230B7003E0491C08780028F4D144
:10C6D00000BF704710B504F009FD0120014981F841
:10C6E000B10610BDD00700202DE9F04786B0002626
:10C6F000784890F88B004E2802D0522812D10BE0D7
:10C700000120754948707348D0F88C00C1F80600C4
:10C71000012006B0BDE8F087012270A1002002F0E0
:10C720004BFA09E0012270A1002002F045FA002036
:10C73000694948700520ECE700BF002001236DA285
:10C740000D2100901A20FAF79DFF0120742380220A
:10C75000642100901D20FAF770FD4FF4407A4FF4E9
:10C76000FA284FEA1837C8F30B0008B1781C87B2D3
:10C7700000251BE00AEB050007F016F90A2095FBDF
:10C78000F0F100FB115008B1FBF772F86420684328
:10C7900090FBF7F0C6B2FF2006F11D02722366215E
:10C7A00000901D20FAF790FD681C85B2BD42E1DBC8
:10C7B0000020012353A20D2100901A20FAF762FFF6
:10C7C00073237F2265211E20FAF7C2FC0DF10809B0
:10C7D00000244DE000208DF808008DF80900ADF828
:10C7E0000E00CDF80A0044B94A4804904A48059022
:10C7F00039490498C1F80A0013E040F2E730844256
:10C8000005D1464804904FF44010059009E0601EA1
:10C810004FF4401101EB40200490601C01EB4020DC
:10C8200005904FF4401000EB44211022484607F0D9
:10C8300053F9142094FBF0F100FB114008B1FBF711
:10C8400017F80A2094FBF0F100FB114078B964203E
:10C8500060434FF47A7190FBF1F0C6B2012006F10B
:10C860001D020346722100906620FAF712FD641C37
:10C87000B4F57A7FAEDB4E20164981F88B004FF479
:10C880004010C1F88C000020FDF732FE4FF440103C
:10C890001149C1F8060000204880888008460078C9
:10C8A00020F0010008700846007820F002000870AF
:10C8B0000846007820F0040008700120487002F05B
:10C8C000A1F910224FF44011484607F08FF80020DC
:10C8D0001FE700007A1F0020402500205B534D53C6
:10C8E0005D526573657400005B534D535D52457234
:10C8F00072330000CFFBCFA2C4DAB4E6C5E4D6C3DE
:10C90000312F3200CFFBCFA2C4DAB4E6C5E4D6C3E0
:10C91000322F320000CE37000002300000CC37004A
:10C9200021B1028842F04002028004E002884FF602
:10C93000BF731A40028070470246002013890B40E3
:10C940000BB1012000E00020704701468889704744
:10C950008181704710B50022028802F441520B8891
:10C960004C8823438C882343CC8823430C8923435E
:10C970004C8923438C892343CC8923431A43028067
:10C98000838B4FF2FF74234083830B8A038210BD95
:10C9900010B5044600BF02210A48FFF7CDFF00286A
:10C9A000F9D021460748FFF7D3FF00BF0121054812
:10C9B000FFF7C2FF0028F9D00248FFF7C6FFC0B258
:10C9C00010BD00000030014001461CE000BF00BF68
:10C9D00000BF00BF00BF00BF00BF00BF00BF00BF5F
:10C9E00000BF00BF00BF00BF00BF00BF00BF00BF4F
:10C9F00000BF00BF00BF00BF00BF00BF00BF00BF3F
:10CA000000BF00BF00BF0A1EA1F1010399B2DDD132
:10CA100070470146088870477047000010B5042031
:10CA20000549086132220549054805F0E3F804206C
:10CA30000149486110BD000000100140381F00206E
:10CA400000F8010810B51948FCF71AF80446184810
:10CA500084421CD117A001F0EFFC1A4890F8DD01C8
:10CA60001249C98888420ED010488079154981F84A
:10CA7000DD010020FDF73CFDC82007F0E6FA0120AB
:10CA80001149087010E0062003F0B2F80CE00F48DE
:10CA9000844203D10E2003F0ABF805E00C48844239
:10CAA00002D1062003F0A4F810BD00007028002079
:10CAB0002A04EC00BCB4BDABD6D8C6F4B8FCD0C2D6
:10CAC0002E2E2E007A1F00207F0200202A047C00D8
:10CAD0002A04F40038B50446002C3CD01F480078E6
:10CAE000012809D01EA001F0A7FCC82007F0ADFA6C
:10CAF000062003F07DF838BD1C480078012809D1D4
:10CB00001BA001F099FCC82007F09FFA062003F053
:10CB10006FF8F0E7FAF7C2FA022119A001F074FBEE
:10CB20000120194991F8DD11184A50541046184B4C
:10CB30000022184900901848FBF7CCFE01236E2212
:10CB40009F210020FAF762FB0020012313A272212B
:10CB50000090FAF797FD00BFCDE700009C0300208E
:10CB6000BDFBD6B9D0DEB8C400000000C80000206C
:10CB7000C5E4D6C3CEC4BCFECEDE41504E0000009C
:10CB8000C9E8D6C341504E007A1F0020FC000020A7
:10CB9000E0000020CC000020702800205B4F4B5D9F
:10CBA000C7D0BBBB20202020205B50315DCFEAC71F
:10CBB000E900000010B51D4800681D49884212D1E7
:10CBC0001C480078401C1B490870084600781A4928
:10CBD0000978884202DB0020164908701548007861
:10CBE00001F02AF921E0114800681449884214D163
:10CBF0001048007818B9104800780E4908700D48A0
:10CC00000078002804DD0B480078401E09490870B0
:10CC10000848007801F010F907E004480068084966
:10CC2000884202D10D2002F0E3FF10BD4000002039
:10CC30002A04BC00EC000020C80000202A04DC000C
:10CC40002A04F40038B50446CCB1FAF727FA0221D9
:10CC50000BA001F0D9FA00200B49087008460078B3
:10CC600001F0EAF801236E229F210020FAF7CEFAA4
:10CC70000020012305A272210090FAF703FD38BDC0
:10CC800041504ECFEAC7E900EC00002020202020D0
:10CC900020202020205B455849545DB7B5BBD80003
:10CCA00070B505460C460B4890F8F80220B94FF4D1
:10CCB00080700949486170BD284605F0F1FF2146A2
:10CCC000002007F0A3F904F10801012007F09EF904
:10CCD00000BFF0E77A1F00200010014043185A00FF
:10CCE000FF2A00DD7047034B1870034B197000BF1B
:10CCF000F8E700005A0000205B00002000B589B072
:10CD00002948006829490844C0B1B0F5001F06D081
:10CD1000B0F5401F22D0B0F5601F41D13CE024485F
:10CD2000007818B902202249087004E020480078F1
:10CD3000401E1F490870F8F79BFA31E01C48007844
:10CD4000022803D100201A49087004E0184800782E
:10CD5000401C17490870F8F78BFA21E0154890F845
:10CD6000B40613490978884212D011480078114955
:10CD700081F8B4060E4802780FA101A804F090FFD4
:10CD800001A8FDF79DFA012211A1002001F014FF76
:10CD9000012002F02DFF03E0062002F029FF00BF72
:10CDA00000BF09B000BD000040000020D6FB43FFDB
:10CDB000ED000020D007002041542B504F433D345C
:10CDC00030303030303031253032780D0A000000FC
:10CDD00055706461746520636F6465747970650073
:10CDE00038B504460425012C22D1002021490880B1
:10CDF000FAF754F9012120A001F006FA01236E226E
:10CE00009F210020FAF702FA1E48007848B91EA0B8
:10CE100001F012FB322007F018F9062002F0E8FEBC
:10CE200006E01D4890F8B4061C490870F8F720FA8F
:10CE30001048008838B90020012319A272210090FF
:10CE4000FAF720FC0AE00B480088C82806D1002029
:10CE5000012319A272210090FAF714FC05480088FA
:10CE6000401C80B203490880B0F5C87F01DB002078
:10CE7000088038BD00010020B1E0C2EBC6F7C9E868
:10CE8000D6C3000095020020C4A3BFE9D4DDCEB410
:10CE9000C6F4B6AF00000000D0070020ED0000206F
:10CEA0005BC9CF5DD1A1D4F12020202020205BCF11
:10CEB000C25DD1A1D4F100005B4D5DB1A3B4E62009
:10CEC0002020205B455849545DCDCBB3F6000000CF
:10CED00000B58BB006A2282101A804F0CDFE0BA15D
:10CEE00001A8F7F775F901A8FDF7EAF90BB000BD45
:10CEF00061742B737973636D643D73746172745FD5
:10CF000070636D20766F6C756D6520003720370D6E
:10CF10000A00000010B5294800682949084450B1AA
:10CF2000B0F5001F06D0B0F5401F28D0B0F5601F47
:10CF300041D13CE000BF21480068224988420DD120
:10CF40002148807A062805DA1F48807A401C1E494D
:10CF500088720FE000201C4988720BE01A48807A22
:10CF600018B906201849887204E01748807A401ED4
:10CF7000154988721449887A00F0A0F81BE012481D
:10CF8000807A124991F8F912884209D00E48807AC5
:10CF90000E4981F8F902F9F7F1FF0120FDF7A8FA2F
:10CFA00001200B490861022002F022FE03E002206A
:10CFB00002F01EFE00BF00BF10BD000040000020B8
:10CFC000D6FB43FF2A04DC00C02200207A1F002089
:10CFD0005828002038B5044604B3FAF75FF8012159
:10CFE0001FA001F011F90020012320A23B21009095
:10CFF000FAF748FB0020F9F7D9F9214890F8F9022F
:10D0000020498872887A00F059F801236E229F2106
:10D010000020FAF7FBF800201B4908801A48008816
:10D0200038B90020012319A272210090FAF72AFBD7
:10D030000AE015480088C82806D10020012319A25B
:10D0400072210090FAF71EFB0F480088401C80B246
:10D050000D490880B0F5C87F01DB0020088038BD8D
:10D06000B1B1B6B7C9E8D6C300000000B1B1B6B7D8
:10D07000C9CFB4ABC9E8D6C33A202020C3EB000027
:10D080007A1F0020C0220020020100205BC9CF5D72
:10D09000D1A1D4F12020202020205BCFC25DD1A1DE
:10D0A000D4F100005B4D5DB1A3B4E6202020205BED
:10D0B000455849545DCDCBB3F60000007FB5054619
:10D0C000104830F815404B239F223B216420FAF78B
:10D0D0003FF844B9002001230BA23B2100906420BB
:10D0E000FAF7D0FA0DE0234609A20A2101A804F0BC
:10D0F000C3FD0020012301AA3B2100906420FAF720
:10D10000C1FA7FBD9840010820B9D8B1D5200000F0
:10D11000202530326420C3EB0000000038B50446FF
:10D120000C25012C1DD1F9F7B9FF01211EA001F03A
:10D130006BF800200090A8B201231EA23821FAF754
:10D14000A1FA1F4890F8F8021E49087005F098FAF5
:10D1500001236E229F210020FAF758F800201A4977
:10D1600008801948008838B90020012317A27221CD
:10D170000090FAF787FA0AE013480088C82806D119
:10D180000020012317A272210090FAF77BFA0E48C3
:10D190000088401C80B20C490880B0F5C87F01DBD4
:10D1A0000020088038BD0000CCE1CABED2F4C9E836
:10D1B000D6C30000202020BFAAB9D83A0000000042
:10D1C0007A1F0020EE000020040100205BC9CF5D23
:10D1D000D1A1D4F12020202020205BCFC25DD1A19D
:10D1E000D4F100005B4D5DB1A3B4E6202020205BAC
:10D1F000455849545DCDCBB3F600000010B51C482E
:10D2000000681C49084450B1B0F5001F06D0B0F5C5
:10D21000401F11D0B0F5601F28D123E000BF164891
:10D22000007818B901201449087002E00020124962
:10D23000087005F025FA19E0104890F8F8020E4938
:10D240000978884207D00C4800780C4981F8F80228
:10D250000120FDF74DF9012009490861062002F07F
:10D26000C7FC03E0062002F0C3FC00BF00BF10BDF6
:10D2700040000020D6FB43FFEE0000207A1F002074
:10D280005828002010B50424244800682449084484
:10D29000B8B1B0F5001F06D0B0F5401F22D0B0F5F0
:10D2A000601F39D134E01F480078401CC0B21D49CE
:10D2B0000870052801DB00200870022000F038F813
:10D2C0002AE018480078002805DD16480078401E3E
:10D2D0001449087002E0042012490870022000F08E
:10D2E00027F819E0104890F89A000E49097888420A
:10D2F00007D00C4800780C4981F89A000120FDF70E
:10D30000F7F8012009490861062002F071FC03E0EA
:10D31000062002F06DFC00BF00BF10BD40000020E1
:10D32000D6FB43FFEF0000207A1F00205828002082
:10D3300030B587B005460424012D48D14D4890F8FA
:10D340009A004D490870F9F7A9FE01214BA000F0A1
:10D350005BFF00200090A0B201234AA23821FAF717
:10D3600091F945480078042805D14AA20A2104A869
:10D3700004F082FC0BE03F4890303F49097800EB15
:10D380004100038845A20A2104A804F075FC00208E
:10D3900004F15001009088B2012304AA3821FAF761
:10D3A00071F9354803783FA2062102A804F064FC15
:10D3B000012202A9002001F0FFFB01236E229F2120
:10D3C0000020F9F723FF0020374908802FE0022DC5
:10D3D0002DD104F1500188B21023A0223821F9F791
:10D3E000B7FE25480078042805D12AA20A2104A8FE
:10D3F00004F042FC0BE01F4890301F49097800EB15
:10D400004100038825A20A2104A804F035FC00206D
:10D4100004F15001009088B2012304AA3821FAF7E0
:10D4200031F901236E229F210020F9F7EFFE1E48FB
:10D43000008838B9002001231CA272210090FAF75D
:10D4400021F90AE018480088C82806D100200123E5
:10D450001CA272210090FAF715F913480088401CAD
:10D4600080B211490880B0F5C87F01DB0020088038
:10D4700007B030BD7A1F0020EF0000204C4344C9A4
:10D48000E8D6C30020B1B3B9E2CAB1BCE43A202067
:10D4900020200000B3A3C1C1202020002533642038
:10D4A000C3EB000025336400060100205BC9CF5D9B
:10D4B000D1A1D4F12020202020205BCFC25DD1A1BA
:10D4C000D4F100005B4D5DB1A3B4E6202020205BC9
:10D4D000455849545DCDCBB3F600000010B5044665
:10D4E000052C27D2DFE804F0030A11181F000020E2
:10D4F00011490870012000F021F81BE001200E49BD
:10D500000870052000F01AF814E002200A4908709B
:10D51000062000F013F80DE00320074908700420EE
:10D5200000F00CF806E0042003490870012000F028
:10D5300005F800BF00BF10BD5D00002010B5044617
:10D540000A2C60D2DFE804F0050E172029323B4494
:10D550004D560021084600F015FA00210846FFF755
:10D56000BDFB50E00021012000F00CFA002108462C
:10D57000FFF7B4FB47E00121084600F003FA002161
:10D580000846FFF7ABFB3EE00A21012000F0FAF964
:10D5900000210846FFF7A2FB35E00021084600F015
:10D5A000F1F900210120FFF799FB2CE0002108464A
:10D5B00000F0E8F901210846FFF790FB23E0002185
:10D5C000084600F0DFF90A210120FFF787FB1AE087
:10D5D0000021012000F0D6F900210120FFF77EFB99
:10D5E00011E00121084600F0CDF901210846FFF7BE
:10D5F00075FB08E00A21012000F0C4F90A2101208E
:10D60000FFF76CFB00BF00BF10BD000010B5FFF7B7
:10D610006BF8044601F0F6FA012202A1002001F0A5
:10D62000CBFA10BD5B534D535D4F6B0010B52248D4
:10D63000006822490844B8B1B0F5001F06D0B0F523
:10D64000401F22D0B0F5601F34D12FE01C48007875
:10D65000401CC0B21A490870042801DB0020087081
:10D66000022000F033F825E015480078002805DD99
:10D6700013480078401E1249087002E00320104948
:10D680000870022000F022F814E00D4800780D49DF
:10D6900081F8F6020120FCF72BFFF9F7DBF80120F7
:10D6A00009490861062002F0A3FA03E0062002F00F
:10D6B0009FFA00BF00BF10BD40000020D6FB43FF13
:10D6C000B40000207A1F002058280020F0B589B04F
:10D6D000054600260C24012D43D1F9F7DFFC01217A
:10D6E00043A000F091FD00200090A0B2012343A2CE
:10D6F0003821F9F7C7FF45480068F8F7D3FD07461A
:10D700003B4643A2142101A804F0B6FA0020009081
:10D71000A0B2012301AA5621F9F7B4FF3E4890F8C0
:10D72000F6023E4951F820303DA20A2106A804F035
:10D73000A3FA06A8F6F776FDC6B2012004F150015F
:10D74000009088B2012306AA3821F9F79BFF012334
:10D750006E229F210020F9F759FD002031490880F1
:10D7600023E0022D21D100200690079008902B483D
:10D770002D49097850F8213029A20A2106A804F081
:10D780007BFA06A8F6F74EFDC6B2012004F150015F
:10D79000009088B2012306AA3821F9F773FF01230C
:10D7A0006E229F210020F9F731FD1E48008838B90C
:10D7B000002001231DA272210090F9F763FF0AE007
:10D7C00018480088C82806D1002001231DA2722114
:10D7D0000090F9F757FF13480088401C80B21149A8
:10D7E0000880B0F5C87F01DB0020088009B0F0BDDB
:10D7F000CDF8C2E7C9E8D6C30000000020CDF8C2CA
:10D80000E7D1A1D4F13A202020200000C40200205A
:10D810004D4F44453A2573007A1F0020B800002080
:10D820002573000070010020B40000205BC9CF5DAB
:10D83000D1A1D4F12020202020205BCFC25DD1A136
:10D84000D4F100005B4D5DB1A3B4E6202020205B45
:10D85000455849545DCDCBB3F6000000F8B50446F9
:10D860002046F8F701FF06463046F8F719FF05464F
:10D8700005B9F8BD6B4602221C213046FEF72EFE8C
:10D88000BDF80000082800D0F3E7044B4FF4806295
:10D8900036213046FEF722FE00BFEAE7082B0020C3
:10D8A00010B51248FBF7ECF804461148844215D134
:10D8B0000E48C0880F4991F83013884207D00B48B2
:10D8C00080790C4981F830030120FCF711FE01201A
:10D8D00009490861062002F08BF905E007488442F7
:10D8E00002D1062002F084F910BD0000702800204B
:10D8F0002A04EC007A1F0020582800202A04F40093
:10D900001CB504460020019004B3F9F7C7FB0221BF
:10D910000FA000F079FC0120104991F8301301AA02
:10D92000505401A80E4B00220E4900900E48FAF701
:10D93000D1FF01236E229F210020F9F767FC002010
:10D9400001230AA272210090F9F79CFE1CBD000081
:10D95000C4A3CABDC9E8D6C3000000007A1F0020D6
:10D96000E000002074010020702800205B4F4B5D18
:10D97000C7D0BBBB2020205B455849545DCDCBB3FD
:10D98000F600000043185A00FF2A00DD7047034BE1
:10D990001870034B197000BFF8E700005800002012
:10D9A0005900002010B52448FBF720FD0446234809
:10D9B000844239D12048407909282AD2DFE800F092
:10D9C00005090D1115191D2125000D2002F010F972
:10D9D0001FE0102002F00CF91BE0112002F008F902
:10D9E00017E0132002F004F913E0172002F000F909
:10D9F0000FE0182002F0FCF80BE0152002F0F8F818
:10DA000007E0192002F0F4F803E01A2002F0F0F821
:10DA100000BF00BF0848407908280BDC0648417960
:10DA20000748FEF7DFFB05E00648844202D10220EA
:10DA300002F0DEF810BD0000AC0000202A04EC006B
:10DA4000582800202A04F40010B51848FBF718F8ED
:10DA500004461748844221D1164890F8F70213492A
:10DA6000C988884213D011488079124981F8F70299
:10DA7000084690F8F702012803D10FA0FCF720FC1C
:10DA800002E016A0FCF71CFC0120FCF731FD012090
:10DA90001B490861062002F0ABF805E019488442F2
:10DAA00002D1062002F0A4F810BD0000702800206A
:10DAB0002A04EC007A1F002061742B737973636D64
:10DAC000643D73746172745F70636D20766F6C7502
:10DAD0006D65203720370D0A0000000061742B733C
:10DAE0007973636D643D73746172745F70636D20EC
:10DAF000766F6C756D65203720350D0A00000000CB
:10DB0000582800202A04F4001CB504460020019087
:10DB100004B3F9F7C3FA02210FA000F075FB01204E
:10DB2000104991F8F71201AA505401A80E4B002297
:10DB30000E4900900E48FAF7CDFE01236E229F2178
:10DB40000020F9F763FB002001230AA27221009054
:10DB5000F9F798FD1CBD0000B3A1BEB0C4A3CABDB7
:10DB6000000000007A1F0020E00000208401002057
:10DB7000702800205B4F4B5DC7D0BBBB2020205BD3
:10DB8000455849545DCDCBB3F600000010B500F008
:10DB900001F810BD0CB500200190009033480068DA
:10DBA00040F480303149086000BF3048006800F41C
:10DBB000003000900198401C0190009820B94FF669
:10DBC000FF7101988842F0D12848006800F40030C5
:10DBD00010B10120009001E0002000900098012881
:10DBE00043D12348006840F01000214908600846EE
:10DBF000006820F0030008600846006840F001005B
:10DC000008601A48406819494860084640684860FA
:10DC10000846406840F4806048600846406820F448
:10DC20007C1048600846406840F410204860084670
:10DC3000006840F08070086000BF0C48006800F089
:10DC400000700028F9D00948406820F00300074917
:10DC500048600846406840F00200486000BF034842
:10DC6000406800F00C000828F9D10CBD00100240FB
:10DC70000020024010B50D480078022814D10C484D
:10DC800000680C49884206D10320084908700AA0A0
:10DC9000FCF716FB07E0064800680A49884202D1F3
:10DCA000062001F0A5FF00BF00BF10BDF40000205A
:10DCB000400000202A04EC0041542B464F54413DC3
:10DCC000310D0A002A04F40010B58CB00446002C73
:10DCD0002AD0F9F7E3F9012133A000F095FA36A034
:10DCE000F8F780F801236E229F210020F9F78EFAC1
:10DCF0000020012334A272210090F9F7C3FC4FF0F9
:10DD0000FF303749086000203649087036A0FCF71C
:10DD1000D7FAC821374806F0A5F90020012336A21A
:10DD200072210090F9F7AEFC2E48007810B101285E
:10DD300036D12DE02F4806F07DF9F0B12848006873
:10DD400050B901202749087031A0F8F74BF8962107
:10DD5000284806F087F91AE021480068002816DDF7
:10DD60001F482FA1026802A803F09AFF02A8F8F743
:10DD700039F802201B49087009E001201949087090
:10DD80002AA0F8F72FF896211A4806F06BF907E059
:10DD9000184806F04FF910B1012001F029FF00BF2B
:10DDA00000BF0CB010BD0000C9FDBCB6B6D4BDB2FA
:10DDB000B0E6B1BE00000000D5FDD4DABCECB2E2A2
:10DDC000B0E6B1BE000000005B4D5DC9FDBCB620F1
:10DDD0002020205B455849545DCDCBB3F6000000B0
:10DDE000F0000020F400002041542B464F54413FE6
:10DDF0000D0A0000F80000205B4D5DC8B7B6A820F2
:10DE00002020205B455849545DCDCBB3F60000007F
:10DE1000C3BBD3D0BFC9B8FCD0C2B0E6B1BE00000E
:10DE2000B8FCD0C2B5BD562564203F00BCECB2E2C0
:10DE3000B3ACCAB1000000002DE9F04196B08046B5
:10DE400000261B250E2467239F2229460020F9F770
:10DE50007FF953485349097850F8213052A22821BC
:10DE60000CA803F009FF00203246761C0090102019
:10DE700000FB025101230CAA1846F9F703FC49499B
:10DE80000978C1EB4112494901EB4200F6F7CAF9A2
:10DE9000C7B244480078C0EB4012444800EB42014E
:10DEA000224602A8F6F770F9002002A9085502AB35
:10DEB0003FA228210CA803F0DFFE00203246761C8A
:10DEC0000090102000FB025101230CAA1846F9F71C
:10DED000D9FBA74217DD33480078C0EB4012334826
:10DEE00000EB420001190CA8F6F7BEF900200090E3
:10DEF0003046721CD6B2102202FB005101230CAA3C
:10DF00001846F9F7BFFB27490978C1EB41122749A9
:10DF100001EB420101F11F00F6F784F9C7B2214875
:10DF20000078C0EB4012214800EB420000F11F01D5
:10DF3000224602A8F6F728F9002002A9085502ABEC
:10DF40001DA228210CA803F097FE00200090304667
:10DF5000721CD6B2102202FB005101230CAA1846F3
:10DF6000F9F790FBA74218DD0E480078C0EB40128D
:10DF70000E4800EB42001F3001190CA8F6F774F9A7
:10DF8000002000903046721CD6B2102202FB0051D5
:10DF900001230CAA1846F9F775FB16B0BDE8F0810D
:10DFA000CC000020EC00002025733A0078210020EE
:10DFB0004E616D653A257300506173733A257300A5
:10DFC00038B505468024B5F5AA7F20DA524806F018
:10DFD00031F800B938BD50214F4806F043F84F489A
:10DFE000007840B9A0B24EA20121F9F7EAFA012067
:10DFF0004A4908708EE000204849087004F1150174
:10E000008AB2A0B20D230021F9F7A2F882E0B5F59B
:10E01000B17F0FDCA0B242A20121F9F7D2FA0320AE
:10E02000009004F1100082B2032308211846F9F78A
:10E0300030F96FE0B5F5BB7F19DCA0B238A2012141
:10E04000F9F7BFFA0320009004F10C0082B2032319
:10E0500008211846F9F71DF90320009004F110007B
:10E0600082B2032308211846F9F713F952E0B5F5F7
:10E07000C87F23DAA0B22AA20121F9F7A2FA03206D
:10E08000009004F1080082B2032308211846F9F732
:10E0900000F90320009004F10C0082B20323082150
:10E0A0001846F9F7F6F80320009004F1100082B248
:10E0B000032308211846F9F7ECF82BE0A0B218A2C8
:10E0C0000121F9F77EFA03200090201D82B203237C
:10E0D00008211846F9F7DDF80320009004F1080044
:10E0E00082B2032308211846F9F7D3F803200090E1
:10E0F00004F10C0082B2032308211846F9F7C9F88D
:10E100000320009004F1100082B203230821184676
:10E11000F9F7BFF800BF5DE7380300203C0300209B
:10E1200056424154312E626D70000000F8B504462D
:10E130000D4616463046F8F7EBFD074605F114008C
:10E1400083B2E019083082B229462046F9F700F878
:10E150000120AA1C91B2221D009090B201233246E8
:10E16000F9F790FAF8BD000030B58BB004460D46C3
:10E1700022480078322190FBF1F201FB120088BBAB
:10E1800024221F491F48F6F778F850B928221C4965
:10E190001C48F6F772F820B91948743890F8B006A0
:10E1A00088B105F1100083B29F2229460020F8F7BC
:10E1B000CFFF282212491348F5F7E6FF0020104947
:10E1C000743981F8B00624220E4902A800F03EFE00
:10E1D000002004F13001009088B20123084A29464A
:10E1E000F9F750FA05480078401CC0B2034908709E
:10E1F000C82801DB002008700BB030BD3E030020B2
:10E2000044080020F4290020F8B504460D462046B5
:10E21000F8F77EFD06460D250020C6F1A00707EBA6
:10E22000D7710090C1F34F00012322462946F9F728
:10E2300029FAF8BD10B50B23322200212D20F8F762
:10E2400087FF1C48007800F0010030B90B234B22F7
:10E2500000212D20F8F77CFF2AE016480078C0F353
:10E26000400080B913480078C0F3001028B912A20A
:10E2700000212D20F9F7A5F91AE012A200212D2086
:10E28000F9F79FF914E00B480078C0F3001028B9A3
:10E2900009A200212D20F9F794F904E009A2002138
:10E2A0002D20F9F78EF90AA200213720F9F789F914
:10E2B00010BD0000C0220020475053312E626D7007
:10E2C00000000000475053412E626D7000000000B6
:10E2D000475053322E626D7000000000F0B58DB0D3
:10E2E00006460D4614463CA207CA01AB07C30027E9
:10E2F0003C480078401CC0B23A490870062800DA51
:10E3000014B10020374908703648007803283ADAFB
:10E31000354890F8AF0670B9344933484230F5F7C4
:10E3200088FF00B99CB124222F4942312F48F5F7CC
:10E330002BFF01270BE02D4901A8F5F77AFF00B963
:10E340002CB1092201A92948F5F71EFF0127002F4A
:10E350003FD005F1100083B29F2229463046F8F7DE
:10E36000F7FE2422214904A800F070FD00201023AC
:10E3700004AA294600903046F9F784F901201A4989
:10E3800081F8B00625E0194917481530F5F751FF17
:10E3900000B9F4B12422144915311448F5F7F4FEFC
:10E3A00005F1100083B29F2229463046F8F7D0FECF
:10E3B00024220E4904A800F049FD0020102304AADD
:10E3C000294600903046F9F75DF90120064981F8A9
:10E3D000B0060DB0F0BD0000B5A5BAF4C4A3CABD27
:10E3E000000000003F030020D0070020182A002072
:10E3F00000B587B002A8FDF74BFF0398009004A07A
:10E40000DDE90423029903F027FC07B000BD0000FA
:10E41000535953434C4B3D25642C50434C4B313D99
:10E4200025642C50434C4B323D25642C48434C4BC7
:10E430003D25640D0A000000F0B593B00546402468
:10E4400004F11403A4F1140081B29F220020F8F714
:10E450007FFE012004F112030090A4F1120081B2AA
:10E460009D220220F8F7E9FE1222294601A800F0B9
:10E47000EDFC01A8F8F74CFC86B2C6F1A00000EB59
:10E48000D071C1F34F0700200090A4F1080081B2C1
:10E49000012301AA3846F9F7F5F813B0F0BD0000E2
:10E4A00038B50446002534B11948007800F0010061
:10E4B000B0B1012514E01648007800F001001549BC
:10E4C0000978884200D138BD1148007800F0010079
:10E4D000104908700E48007800F0010000B10125D5
:10E4E000012D02D0022D0FD105E00BA203213C200B
:10E4F000F9F767F809E0002001230AA20321009040
:10E500003C20F9F7BFF800E000BF00BF00BFDAE72A
:10E5100040250020F20100204D61696C312E626DB2
:10E52000700000002020000038B504464248007802
:10E53000012805D141A202210020F9F742F804E0A8
:10E5400042A202210020F9F73CF8012C01DB632CE8
:10E5500006D10B23152203210720F8F7F9FD69E006
:10E56000082C0EDA0320022307220A21009009203A
:10E57000F8F78FFE0B23152203211846F8F7E8FD64
:10E5800058E0102C16DA0320022307220A210090FB
:10E590000920F8F77EFE032002230A22114600908C
:10E5A0000720F8F776FE0B23152203210F20F8F73A
:10E5B000CFFD3FE0162C1EDA0320022307220A219A
:10E5C00000900920F8F765FE032002230A22114675
:10E5D00000900720F8F75DFE032002230D220A2198
:10E5E00000900520F8F755FE0B2315220321132078
:10E5F000F8F7AEFD1EE00320022307220A21009057
:10E600000920F8F746FE032002230A221146009053
:10E610000720F8F73EFE032002230D220A21009076
:10E620000520F8F736FE0320022310220A2100906D
:10E63000F8F72FFE38BD0000D501002053696E6742
:10E640006C654F4B2E626D700000000053696E6761
:10E650006C652E626D70000038B505464248006852
:10E6600042490968884207D0404800683E4908602E
:10E670000846006800F0E2F83D4800683D49096836
:10E68000884205D13C4800783C49097888420BD043
:10E690003A480078384908703648006834490860BC
:10E6A00034480068FFF740FF35480078642808DAEE
:10E6B0004FF4B4703349086031480078401C304949
:10E6C0000870314800682F490968884204D12D48F4
:10E6D0000068B0F5AA7F07DA2A4800682A4908606E
:10E6E00028480068FFF76CFC0020FFF7D9FE274898
:10E6F0000078C0F340002549097801F0010140EAA3
:10E70000012022490978C1F3001140EA8104204820
:10E710000088A04203D01E480480FFF78BFD2846E6
:10E7200000F040F81B4890F8AF061B4991F9001023
:10E73000884217D0174890F8AF0640B216490870C3
:10E740000846007830B90E231E226E217920F8F792
:10E75000BBFC07E00020012310A26E21009079206D
:10E76000F8F790FF38BD0000F8020020C802002032
:10E77000EC0200208C020020F6020020D5010020CF
:10E78000E8020020D8010020F0020020C022002072
:10E79000F4020020D0070020FC020020B9D2B6CF3E
:10E7A0000000000010B58CB004461C48407808B941
:10E7B0000CB010BD0AA8FDF72DFE9DF82E001849DB
:10E7C0000978884200D13CB39DF82E0014490870A6
:10E7D000087800EBD0714910A0EB410151B19DF8D0
:10E7E0002D0000909DF82C300EA21E2102A803F0EF
:10E7F00043FA09E09DF82D0000909DF82C300CA202
:10E800001E2102A803F038FA0020012302AA0146C3
:10E8100000905020F8F736FF00BFC9E7D00700206E
:10E820003D030020253032643A2530326400000078
:10E8300025303264202530326400000038B50446AB
:10E84000022C01D0032C08D10020012313A2014681
:10E8500000901820F8F716FF1FE0042C03D0052CB9
:10E8600001D0082C08D1002001230DA20146009000
:10E870001820F8F707FF10E0092C08D10020012329
:10E8800008A2014600901820F8F7FCFE05E00B23D3
:10E890002D2200211820F8F75BFC38BD324700001C
:10E8A000334700003447000070B588B005460C4679
:10E8B000002655B18548007838B100208449A1F878
:10E8C00068008449087081490870824800780628E9
:10E8D00023D2DFE800F003233894C0D67EA0FFF7F0
:10E8E000ABFD7B487FA21E21C36B684603F0C4F9D1
:10E8F0006846FBF7E5FC00226946104600F05CF92B
:10E900000020734981F86C0088814FF4FA717A48CD
:10E9100005F0A8FB01206F490870D4E0764805F0A7
:10E9200089FB18B96A4890F86C0058B1684880892A
:10E93000002804DC0020664981F86B00B7E0022063
:10E9400064490870BFE06248B0F86800604989898E
:10E95000884212DB5E48B0F8683068A21E21684623
:10E9600003F08AF901226946002000F025F9584891
:10E970008089401E5649A1F86800012C16D15448E0
:10E98000B0F868005F490880514880890988401ABA
:10E99000052803DB05205C4908701DE04C48007B1E
:10E9A00058490978401A5849087015E04848B0F8A5
:10E9B0006800052807DA0020524908804448007B97
:10E9C0005149087008E04248B0F86800401F4D49BE
:10E9D000088005204C4908704B480078052802DB68
:10E9E0000520494908700020394981F86B004548E5
:10E9F00000884649088003203649087063E0414892
:10EA0000008841490978084440490988884203DC64
:10EA100005203049087056E000202D4981F86A0031
:10EA20003A4803880088401C384A108038A21E21CA
:10EA3000684603F021F96846FBF742FC002269466C
:10EA4000104600F0B9F8C8212B4805F00BFB042054
:10EA50002049087037E01E4890F86A0048B11C4809
:10EA600090F86B00401C1A4981F86B00032019498B
:10EA70000870214805F0DEFA10B10520154908702C
:10EA800021E0012C09D11248B0F868001E4909782C
:10EA900008440F49A1F8680008E00D48B0F8680084
:10EAA00019490978401A0A49A1F8680000BF0120F5
:10EAB0000649087060239F2228210020F8F748FBB0
:10EAC000012008B070BD00BF3046FAE78400002086
:10EAD000D007002085000020C7EBC9D4BAF22E2E43
:10EAE0002E00000041542B504F433D304530303014
:10EAF00030253038780D0A00880000206F76657266
:10EB00003A2564008E000020900000208C00002038
:10EB100041542B504F433D3130303030303231256D
:10EB20003034780D0A00000001221CA1002000F002
:10EB300043F84FF400501C49486104201B49086009
:10EB40008001194948610120086180204861022044
:10EB5000174908600120091D086040021249086138
:10EB600040F6B830F8F760FE002144F21C00FDF7D3
:10EB700075FB00214FF4C020FDF760FB00210D481C
:10EB8000F5F734FF00210120FDF748FB05E04FF4C5
:10EB90007A7005F05AFAF8F76BFEF8E7536C656582
:10EBA00070696E67000000000010014014140140FD
:10EBB000100C0140002401402DE9F04105460E46AD
:10EBC0001746012D01D1BDE8F0810C48007800B155
:10EBD000F9E73046F5F726FB0446B4F5807F01DD02
:10EBE0004FF480742146304602F06AFA1FB10221C8
:10EBF00003A002F065FA00BFE5E700002C0000204A
:10EC00000D0A00002DE9FF410546022D01DDBDE89A
:10EC1000FF81002D5FD0012D2FD100202F4948808A
:10EC200088806F460846D0F80660E8464FF47A744C
:10EC300021E010223146384604F0D8FE9DF800004D
:10EC4000012812D125484088401C244948809DF85D
:10EC50000100012809D108468088401C88800846A8
:10EC6000007820F00100401C0870601E84B204B9D6
:10EC700002E0D8F80C60DCE72DE0022D2BD16F46C6
:10EC80001648D0F80660E8464FF47A7421E0102266
:10EC90003146384604F0AAFE9DF8000018B90F4826
:10ECA000C0F80A6016E0601E84B28CB90B48007888
:10ECB00020F00400001D09490870012208A100206D
:10ECC000FFF77AFF00F032F808A0FBF7F9FA01E04D
:10ECD000029EDCE700BF00BF99E70000402500204E
:10ECE0005B534D535D46756C6C00000041542B4CDA
:10ECF00053485454533D312C2243464642434641E7
:10ED0000324432443143324641220D0A00000000B1
:10ED100010B5044614B100F009F803E04FF4807018
:10ED20000149486110BD00000010014030B5114894
:10ED300090F8F70208B9032400E0042400250FE04E
:10ED40004FF480700C4908610520FDF73DFE4FF43B
:10ED50008070094948610520FDF736FE681CC5B280
:10ED6000A542EDDB4FF48070034908610520FDF7F3
:10ED70002BFE30BD7A1F00200010014008B54FF473
:10ED80008070ADF8000010208DF8030003208DF88E
:10ED9000020069460348F7F763F80020FFF7B8FF61
:10EDA00008BD000000100140F8B506460D4630468B
:10EDB000F5F738FA00F0010000B1F8BD40E000249A
:10EDC00029E016F8010B0DF804001DF804003028A6
:10EDD0000ADB1DF80400392806DC1DF80400303871
:10EDE000C0B20DF8040014E01DF8040041280ADB4D
:10EDF0001DF80400462806DC1DF804003738C0B2B0
:10EE00000DF8040005E01DF804005738C0B20DF8F5
:10EE10000400601CC4B2022CD3DB9DF80000000784
:10EE2000000E8DF800009DF8000000F0F0008DF855
:10EE300000009DF800009DF80110084305F8010B43
:10EE400030780028BBD1287000BFB6E72DE9F04725
:10EE50000646884614464046F5F7E4F98146002107
:10EE6000601E3154621E41463046F5F7CFF9601EF0
:10EE700048451CDC052C1ADD2E21A01E3154E01E55
:10EE800031543546002707E028789F2802DDAD1C65
:10EE9000BF1C01E06D1C7F1C201FB842F4DCB8428F
:10EEA00005D128789F2802DD2E21201F3154BDE88E
:10EEB000F087000010B50D480078B0B10C4800781C
:10EEC000401CC0B20A49087005280EDB09480078CA
:10EED000012803D108A26B21FFF728F9002003497C
:10EEE0000870012206A1FFF767FE10BD8002002016
:10EEF00081020020CC020020B2CBB5A500000000AA
:10EF00005175697447726F757053656C000000002D
:10EF100010B506A26B210120FFF708F90120054971
:10EF2000087000200449087010BD0000C8B7B6A8DA
:10EF300000000000800200208102002010B5E6B031
:10EF4000084CA4F1080090F89801022806D140F27C
:10EF50008D12214601A8F5F717F900E000BF00BFA8
:10EF600066B010BD3823002010B505F011F804F08C
:10EF700083FC05F015F810BD10B51248006840F08C
:10EF8000010010490860084640680F4908400D49D3
:10EF90004860084600680D4908400A49086008466C
:10EFA000006820F4802008600846406820F4FE00D5
:10EFB00048604FF41F008860FEF7E8FD04480549EB
:10EFC000086010BD001002400000FFF8FFFFF6FED1
:10EFD0000040000808ED00E021B1028842F0010283
:10EFE000028004E002884FF6FE731A4002807047E8
:10EFF00031B1B0F8442042F40042A0F8442005E0CA
:10F00000B0F84420C2F30E02A0F84420704700007C
:10F0100070B5002400220023058C4FF6EF763540B2
:10F020000584028C8388048B48F6FF752C404FF6CC
:10F03000FF452C400D884FF6FF7606EA05252C4348
:10F040004FF6DF752A400D8906EA05152A434D88DB
:10F0500006EA05152A43154DA84202D0144DA842D0
:10F060001DD14FF67F752A404D894FF6FF7606EA8F
:10F0700005152A434FF6BF752A408D8806EA051507
:10F080002A434FF6FF352B404FF2FF752B408D89F9
:10F0900006EA85052B43CD8906EA85052B43838047
:10F0A0000483CD880587028470BD0000002C0140D8
:10F0B00000340140002202881D4B98420ED01D4BA7
:10F0C00098420BD0B0F1804F08D01B4B984205D02E
:10F0D0001A4B984202D01A4B984204D14FF68F73C4
:10F0E0001A404B881A43174B984207D0164B984248
:10F0F00004D04FF6FF431A40CB881A4302808B8816
:10F1000083850B8803850A4B98420BD0094B9842A4
:10F1100008D00E4B984205D00D4B984202D00D4BB3
:10F12000984201D10B7A0386012383827047000045
:10F13000002C014000340140000400400008004061
:10F14000000C00400010004000140040004001404E
:10F15000004401400048014010B570210648F5F711
:10F160002CF8064890F8F902054A32F8101005A06C
:10F1700002F072FD10BD0000C02200207A1F0020A6
:10F180009840010847707374696D653D25640D0AE8
:10F1900000000000F0B505460C4628686968AA68BA
:10F1A000EB6801EA020623EA01073E4327683E4472
:10F1B000FE4F3E443044C60146EA5060084400EA2F
:10F1C000010622EA00073E4367683E44F84F3E448A
:10F1D00033441E0346EA1353034403EA000621EABC
:10F1E00003073E43A7683E44F24F3E443244560470
:10F1F00046EAD2321A4402EA030620EA02073E43F4
:10F20000E7683E44EC4F3E4431448E0546EA912186
:10F21000114401EA020623EA01073E4327693E44FE
:10F22000E64F3E443044C60146EA5060084400EAD6
:10F23000010622EA00073E4367693E44E04F3E4430
:10F2400033441E0346EA1353034403EA000621EA4B
:10F2500003073E43A7693E44DA4F3E443244560416
:10F2600046EAD2321A4402EA030620EA02073E4383
:10F27000E7693E44D44F3E4431448E0546EA91212D
:10F28000114401EA020623EA01073E43276A3E448D
:10F29000CE4F3E443044C60146EA5060084400EA7E
:10F2A000010622EA00073E43676A3E44C84F3E44D7
:10F2B00033441E0346EA1353034403EA000621EADB
:10F2C00003073E43A76A3E44A6F524464F3E324418
:10F2D000560446EAD2321A4402EA030620EA02073A
:10F2E0003E43E76A3E44BB4F3E4431448E0546EA06
:10F2F0009121114401EA020623EA01073E43276BEC
:10F300003E44B54F3E443044C60146EA506008448E
:10F3100000EA010622EA00073E43676B3E44AF4F16
:10F320003E4433441E0346EA1353034403EA0006F3
:10F3300021EA03073E43A76B3E44A94F3E443244B3
:10F34000560446EAD2321A4402EA030620EA0207C9
:10F350003E43E76B3E44A34F3E4431448E0546EAAC
:10F360009121114401EA030622EA03073E4367683C
:10F370003E449D4F3E443044460146EAD060084436
:10F3800000EA020621EA02073E43A7693E44974F7E
:10F390003E4433445E0246EAD353034403EA010683
:10F3A00020EA01073E43E76A3E44914F3E4432441F
:10F3B000960346EA92421A4402EA000623EA00074C
:10F3C0003E4327683E448B4F3E4431440E0546EA97
:10F3D0001131114401EA030622EA03073E4367693B
:10F3E0003E44854F3E443044460146EAD0600844DE
:10F3F00000EA020621EA02073E43A76A3E447F4F25
:10F400003E4433445E0246EAD353034403EA010612
:10F4100020EA01073E43E76B3E44794F3E443244C5
:10F42000960346EA92421A4402EA000623EA0007DB
:10F430003E4327693E44734F3E4431440E0546EA3D
:10F440001131114401EA030622EA03073E43676AC9
:10F450003E446D4F3E443044460146EAD060084485
:10F4600000EA020621EA02073E43A76B3E44674FCB
:10F470003E4433445E0246EAD353034403EA0106A2
:10F4800020EA01073E43E7683E44614F3E44324470
:10F49000960346EA92421A4402EA000623EA00076B
:10F4A0003E43276A3E445B4F3E4431440E0546EAE4
:10F4B0001131114401EA030622EA03073E43676B58
:10F4C0003E44554F3E443044460146EAD06008442D
:10F4D00000EA020621EA02073E43A7683E444F4F76
:10F4E0003E4433445E0246EAD353034403EA010632
:10F4F00020EA01073E43E7693E44494F3E44324417
:10F50000960346EA92421A4402EA000623EA0007FA
:10F510003E43276B3E44434F3E4431440E0546EA8A
:10F520001131114481EA02065E4067693E443E4F54
:10F530003E443044060146EA1070084480EA010661
:10F540005640276A3E44394F3E443344DE0246EA81
:10F550005353034483EA00064E40E76A3E44344F67
:10F560003E443244160446EA12421A4482EA030632
:10F570004640A76B3E442F4F3E443144CE0546EAF9
:10F580005121114481EA02065E4067683E442A4FD9
:10F590003E443044060146EA1070084480EA010601
:10F5A000564027693E44254F3E4449E078A46AD737
:10F5B00056B7C7E8DB702024EECEBDC1AF0F7CF597
:10F5C0002AC68747134630A8019546FDD89880691A
:10F5D000AFF7448BBED75C892211906B937198FD75
:10F5E0008E4379A62108B44962251EF640B340C077
:10F5F000515A5E26AAC7B6E95D102FD653144402AD
:10F6000081E6A1D8C8FBD3E7E6CDE121D60737C311
:10F61000870DD5F4ED145A4505E9E3A9F8A3EFFCED
:10F62000D9026F678A4C2A8D4239FAFF81F67187B9
:10F6300022619D6D0C38E5FD44EABEA4A9CFDE4BE6
:10F640003344DE0246EA5353034483EA00064E4045
:10F65000E7693E449F4F3E443244160446EA124254
:10F660001A4482EA03064640A76A3E449A4F3E4443
:10F670003144CE0546EA5121114481EA02065E403A
:10F68000676B3E44954F3E443044060146EA107095
:10F69000084480EA0106564027683E44904F3E44A5
:10F6A0003344DE0246EA5353034483EA00064E40E5
:10F6B000E7683E448B4F3E443244160446EA124209
:10F6C0001A4482EA03064640A7693E44864F3E44F8
:10F6D0003144CE0546EA5121114481EA02065E40DA
:10F6E000676A3E44814F3E443044060146EA10704A
:10F6F000084480EA01065640276B3E447C4F3E4456
:10F700003344DE0246EA5353034483EA00064E4084
:10F71000E76B3E44774F3E443244160446EA1242B9
:10F720001A4482EA03064640A7683E44724F3E44AC
:10F730003144CE0546EA5121114461EA03065640A0
:10F7400027683E446D4F3E443044860146EA90604F
:10F75000084460EA02064E40E7693E44684F3E4472
:10F7600033449E0246EA9353034463EA010646404B
:10F77000A76B3E44634F3E443244D60346EA5242AE
:10F780001A4462EA00065E4067693E445E4F3E44AA
:10F7900031444E0546EAD121114461EA0306564040
:10F7A000276B3E44594F3E443044860146EA906000
:10F7B000084460EA02064E40E7683E44544F3E4427
:10F7C00033449E0246EA9353034463EA01064640EB
:10F7D000A76A3E444F4F3E443244D60346EA524263
:10F7E0001A4462EA00065E4067683E444A4F3E445F
:10F7F00031444E0546EAD121114461EA03065640E0
:10F80000276A3E44454F3E443044860146EA9060B4
:10F81000084460EA02064E40E76B3E44404F3E44D7
:10F8200033449E0246EA9353034463EA010646408A
:10F83000A7693E443B4F3E443244D60346EA524217
:10F840001A4462EA00065E40676B3E44364F3E440F
:10F8500031444E0546EAD121114461EA030656407F
:10F8600027693E44314F3E443044860146EA906069
:10F87000084460EA02064E40E76A3E442C4F3E448C
:10F8800033449E0246EA9353034463EA010646402A
:10F89000A7683E44274F3E443244D60346EA5242CC
:10F8A0001A4462EA00065E40676A3E44224F3E44C4
:10F8B00031444E0546EAD12111442E6806442E609B
:10F8C0006E680E446E60AE681644AE60EE681E440C
:10F8D000EE60F0BD604BBBF670BCBFBEC67E9B2821
:10F8E000FA27A1EA8530EFD4051D880439D0D4D990
:10F8F000E599DBE6F87CA21F6556ACC4442229F4E6
:10F9000097FF2A43A72394AB39A093FCC3595B65A7
:10F9100092CC0C8F7DF4EFFFD15D84854F7EA86F74
:10F92000E0E62CFE144301A3A111084E827E53F79A
:10F9300035F23ABDBBD2D72A91D386EB08B540F257
:10F940002551354801F056FA002852D0324801F0CE
:10F950000DFBC0B2009040F225512F4801F019FA7A
:10F960002E480078022805D19DF800102C4801F09F
:10F9700002FB3EE029480078012805D19DF80010DF
:10F98000284801F0F8FA34E02448007858BB2648AB
:10F99000008828B10020254908802549087008BD45
:10F9A0009DF80010214802880088401C1F4B1880D9
:10F9B0001F4881541F4800780D281AD19DF8000077
:10F9C0000A2816D11A48007847280DD118484078DF
:10F9D000542809D11846008813490880002014498A
:10F9E0001A461288885404E0002010490880104903
:10F9F00008709DF800000F4908700821064801F0C2
:10FA0000ECF9012806D1044801F0B0FA08210248B7
:10FA100001F0B6F900BFC2E7003801402C00002019
:10FA20000044004000480040300000202E0000202C
:10FA3000BC0300203E00002008B540F225512548B7
:10FA400001F0D8F9B0B3234801F090FAC0B20090A9
:10FA50002148007802280AD19DF800101F4801F0C3
:10FA60008AFA40F225511B4801F093F908BD1C4861
:10FA7000008840F21E21884217DA9DF800001949DB
:10FA8000194A1288885418480088401C80B21649C8
:10FA9000088040F21E21884202DB002012490880C3
:10FAA0000F480088401C0E49088040F22551094843
:10FAB00001F06FF90821074801F08FF9012806D1FC
:10FAC000044801F053FA0821024801F059F900BF37
:10FAD000CCE70000004400402C000020003801402A
:10FAE00034000020840400203600002038B50024B3
:10FAF00040F22551374801F07DF900285CD03548A7
:10FB000001F034FAC0B2009033480078012805D1E2
:10FB10009DF80010314801F02EFA44E0304800888A
:10FB200000283DD19DF800002E492F4A12888854A4
:10FB300008460078242803D000202B49088004E0E0
:10FB400029480088401C2849088027480088B0F5CB
:10FB5000957F02DD002024490880244800780D2884
:10FB600021D19DF800000A281DD11E484078472861
:10FB700012D11C48C07852280ED11A484079432827
:10FB80000AD1002118480088401E164A1154164810
:10FB900000881349088006E000201349088002E02D
:10FBA00000201149088040F225510A4801F0F1F87F
:10FBB0009DF800000D4908700821064801F00DF974
:10FBC000012806D1034801F0D1F90821014801F0CC
:10FBD000D7F838BD004800402C0000200038014014
:10FBE0003C000020A20600203A0000203F00002038
:10FBF00003498978024A51701146887070470000A5
:10FC0000CC02002030B589B005467A48007810B1A2
:10FC100001281BD10FE07848007858B977A0FEF78B
:10FC20000BFC32217A4804F01DFA0120714908705A
:10FC300009B030BD0AE0764804F0FCF928B1002094
:10FC40006C4908700120FFF7D3FFF1E700BF002DDA
:10FC50007DD00020684981F86D006EA0FEF7ECFBB6
:10FC6000002071490880F7F719FA0D216FA0FEF7FF
:10FC7000CBFA002407E07048704941F824000020C6
:10FC80006F490855641C1E2CF5DD5B486DA21E21D2
:10FC9000036F01A801F0F0FF002201A91046FEF752
:10FCA0008BFF00244BE004EB440000EBC4016848E8
:10FCB00050F821005049C96B88423FD1E4B3234634
:10FCC00064A21E2101A801F0D7FF012201A9002092
:10FCD000FEF772FF4848D0F87C1104EB440000EBBB
:10FCE000C4025B4840F8221004EB440101EBC4025B
:10FCF000014601EB8201881D24225549891DF4F734
:10FD000043FA3D48B0F8801104EB440000EBC40214
:10FD10004F4800EB820081803748C06B3649C1F8FC
:10FD20007C012422423101F5A070F4F72DFA32480B
:10FD3000B0F84010A0F880112F48046F641C2E48C2
:10FD4000006FA04201DD1E2CADDB00241AE02EE086
:10FD500004EB440000EBC4013D4850F82100264963
:10FD6000C96B884202D101203549085504EB440093
:10FD700000EBC401364800EB8100801D2F4941F89B
:10FD80002400641C1C48006FA04201DD1E2CDFDB38
:10FD90002B48334B0022294900903248F8F79AFD4E
:10FDA00001236E229F210020F7F730FA40E71E481A
:10FDB000008838B9002001232BA272210090F7F7A8
:10FDC00061FC0AE018480088C82806D100200123F9
:10FDD0002BA272210090F7F755FC13480088401CB5
:10FDE00080B211490880B0F5C87F01DB002008808F
:10FDF00000BF1DE740030020D00700202020C7EBF4
:10FE0000CFC8B5C7C2BC2E2E2E2020200000000077
:10FE100044030020D5FDD4DABBF1C8A12CC7EBC93F
:10FE2000D4BAF22E2E2E000048030020C8BAD7E91B
:10FE3000D1A1D4F100000000580300203C2A00208A
:10FE4000B82A0020476E756D3D25640D0A0000003C
:10FE50004C090020693A25642A2A2A2A0000000059
:10FE60004C030020702800205BC9CF5DD1A1D4F1E4
:10FE70002020202020205BCFC25DD1A1D4F1000042
:10FE80005B4D5DC8B7B6A8202020205B455849547B
:10FE90005DCDCBB3F6000000F0B591B0064612255B
:10FEA00046B10020AF490870F7F7F8F80121AEA07D
:10FEB000FEF7AAF902272024AE480068AE4988421E
:10FEC00006D0AC480068AD49884201D0002E7DD0F4
:10FED0000020A8490860A348007818B1A14800781C
:10FEE00002285ED17F239F2221460020F7F730F9B8
:10FEF000A34BA4A2322101A801F0BEFE00200123E1
:10FF000001AA214600903846F7F7BCFB601984B27D
:10FF10009B482138D0F81D309DA2322101A801F064
:10FF2000ABFE0020012301AA214600903846F7F7D6
:10FF3000A9FB601984B292482138B0F82F3098A2FA
:10FF4000322101A801F098FE0020012301AA2146D8
:10FF500000903846F7F796FB601984B2002394A20C
:10FF6000322101A801F088FE0020012301AA2146C8
:10FF700000903846F7F786FB601984B28F4890A24C
:10FF80003221036801A801F077FE0020012301AAB5
:10FF9000214600903846F7F775FB0120714908703B
:10FFA000DDE0704800780128FAD17F239F222146A6
:10FFB0000020F7F7CDF8864886A23221036801A811
:10FFC00001F05AFE0020012301AA00E06AE0214668
:10FFD00000903846F7F756FB601984B200208DF880
:10FFE000380067482138D0F81D107E4A0EA8F6F771
:10FFF00061F90EAB7CA2322101A801F03DFE002088
:020000040801F1
:10000000012301AA214600903846F7F73BFB60190F
:1000100084B20020302377A23221009001A801F0A1
:100020002BFE0020012301AA214600903846F7F755
:1000300029FB601984B23222002101A8F4F7B6F836
:100040007148007828B971A2322101A801F014FE8C
:100050001CE06D480078012805D170A2322101A86A
:1000600001F00AFE12E068480078022805D170A26B
:10007000322101A801F000FE08E06348007803285F
:1000800004D170A2322101A801F0F6FD0020012365
:1000900001AA214600903846F7F7F4FA02203149C8
:1000A00008705CE0334800686B49884257D10020F3
:1000B000304908602B480078012803D0294800788F
:1000C00002284CD17F239F2221460020F7F740F8D9
:1000D0000020012361A2214600903846F7F7D2FAAA
:1000E000601984B2604B61A2322101A801F0C4FD05
:1000F0000020012301AA214600903846F7F7C2FAF2
:10010000601984B20020012359A22146009038468C
:10011000F7F7B8FA601984B2584B54A2322101A8FB
:1001200001F0AAFD0020012301AA214600903846D3
:10013000F7F7A8FA601984B25148B0F82E3351A2EB
:10014000322101A801F098FD0020012301AA2146D7
:1001500000903846F7F796FA00200249087011B06F
:10016000F0BD000090010020D6D5B6CBD0C5CFA2FF
:1001700000000000400000202A04DC002A04BC002B
:10018000591F0020D6D5B6CBD0CDBAC53A257300BD
:10019000D6D5B6CBB1E0C2EB3A256C7500000000B5
:1001A000D3A6D3C3B0E6B1BE3A5625640000000022
:1001B000C4DAB2BFB0E6B1BE3A25640074000020D4
:1001C000C4A3BFE9B0E6B1BE3A4C2564000000000C
:1001D00078000020B6D4BDB2B0E6B1BE3A56256470
:1001E000000000006A1F0020D0A3D1E9C2EB3A252D
:1001F000730000004D4355D6F7C6B53A25642E2549
:1002000064204D687A00000091020020C4A3BFE979
:10021000C0E0D0CD3ACEB4D6AA000000C4A3BFE956
:10022000C0E0D0CD3AB5A5B5E7D0C5B0E600000036
:10023000C4A3BFE9C0E0D0CD3AD2C6B6AFC1AACD03
:10024000A8B0E600C4A3BFE9C0E0D0CD3AC8ABCDAA
:10025000F8CDA8B0E60000002A04AC00BDBBBBBBD3
:10026000B7FECEF1C6F73A0008280020257300003B
:10027000B1B1B6B7B7FECEF1C6F73A0030280020CC
:100280007A1F0020504F52543A25640038B5044676
:10029000002C25D0F6F702FF0020012311A20D212A
:1002A0000090F7F7EFF912484088012807DB104863
:1002B000418800230F4A1048F8F766FB03E000214D
:1002C0000846F8F791FB002001230CA27221009050
:1002D000F7F7D8F901236E229F210020F6F796FF49
:1002E00038BD00002020CEC4B1BECFFBCFA200009D
:1002F00040250020E4010020702800205B4D5DB205
:10030000E9D4C4202020202020205B535DD1A1CF40
:10031000EE00000030B587B00546B5B1F6F7BEFE79
:100320000D21B8A0FDF770FF00200123BAA26E21B5
:1003300000901846F7F7A6F94FF0FF30B84908606B
:100340000020B849086007B030BDB748007808B948
:10035000002424E0B448807838B9B348807920B9C3
:1003600001240020B149086019E0AF48807828B91D
:10037000AD488079002801DD022410E0AA48807889
:1003800000280CDD0324A948006840B90120A749D2
:1003900008602B239F221B210020F6F7D9FE34B1E1
:1003A000012C14D0022C26D0032C76D14AE09C4894
:1003B000006884420AD069239F222E210020F6F78C
:1003C000C7FE9BA22E211E20F7F7FBF865E094489C
:1003D000006884420ED069239F222E210020F6F768
:1003E000B7FE93A22E211E20F7F7EBF801208E49CD
:1003F00081F8B00651E08A480068844205D069233C
:100400009F222E210020F6F7A3FE8648006828B917
:100410008AA22F213420F7F7D4F812E0814800682F
:10042000642805D188A22F213420F7F7CAF808E004
:100430007C480068C82804D186A22F213420F7F711
:10044000C0F82AE076480068844205D069239F22DC
:100450002E210020F6F77CFE7248006828B980A2A1
:100460002F213620F7F7ADF812E06E4800686428B7
:1004700005D17EA22F213620F7F7A3F808E06948BE
:100480000068C82804D17DA22F213620F7F799F8FB
:100490001B210020FDF768FE00BF00BF002C1CDD03
:1004A0006048006838B15F480068642803D05D4840
:1004B0000068C8280AD1032C08D059480068844233
:1004C00005D001221B210020FDF708FF84E0002257
:1004D0001B211046FDF702FF7EE02022142102A816
:1004E000F3F764FE092269A102A8F3F74DFE4D4817
:1004F000006838B90020012302AA1B210090F7F7F9
:10050000C1F81EE04748006864280AD12E208DF803
:1005100011000020012302AA1B210090F7F7B2F876
:100520000FE040480068C8280BD12E208DF811003C
:100530008DF812000020012302AA1B210090F7F77A
:10054000A1F8394890F8B30653490978884203D195
:1005500033480068401CB0BB334890F8B3064E499E
:10056000087008460078012805D14CA2142102A881
:1005700001F082FB29E048480078022805D14BA20F
:10058000142102A801F078FB1FE0434800780428FA
:1005900005D14AA2142102A801F06EFB15E03E48E5
:1005A0000078052805D149A2142102A801F064FBB6
:1005B0000BE039480078062806D147A2142102A88A
:1005C00001F05AFB01E007E007E00020012302AA46
:1005D0001B210090F7F756F800BF12480068401C36
:1005E00010490860B0F5967F01DB002008600C48D8
:1005F0000068844204D00A48046000200949086069
:1006000000BFA0E6B9ABCDF8BCAFC8BAB6D4BDB296
:10061000CFB5CDB300000000B2CBB5A500000000FF
:100620000003002004030020D0070020DC0200208B
:100630006C6F676F2E626D70000000005069636B15
:1006400075702E626D7000005069636B7570312E8D
:10065000626D70005069636B7570322E626D700050
:10066000737065616B65722E626D70007370656189
:100670006B6572312E626D700000000073706561F1
:100680006B6572322E626D7000000000D5FDD4DA09
:10069000B5C7C2BD2E00000008030020D5CBBAC5E7
:1006A000D0C5CFA2B4EDCEF300000000CEDECDF871
:1006B000C2E7C1ACBDD3202000000000C7EBB2E50B
:1006C000BFA820202020202000000000CEDEB7A8F8
:1006D000C1ACBDD300000000C3BBD3D0B7FECEF188
:1006E0000000000010B504462CB103A304A2064983
:1006F0000648FAF701FC10BDD6F7B2CBB5A500004D
:1007000050616C61636500007C030020B02900200B
:10071000F8B50546002600BF701CC0B20646224947
:1007200051F8200000780028F6D1002D3AD0F6F7D5
:10073000B5FC0D211DA0FDF767FD1F4800780128BD
:1007400015D0002407E0184850F824001B4941F850
:100750002400601CC4B2062CF5DB134850F82600B8
:10076000164941F824001648F8F7ECFD03E00E495D
:100770001348F8F7E7FD0020012312A27221009030
:100780001846F6F77FFF0020012310A27221009087
:100790007D20F6F777FF01236E229F210020F6F7D8
:1007A00035FDF8BD00BFFCE70C030020CFB5CDB38D
:1007B000C9E8D6C30000000091000020CC29002029
:1007C000AC000020C8B7B6A800000000B7B5BBD881
:1007D00000000000F8B50646002E58D0F6F75EFC83
:1007E00002212CA0FDF710FD01236E229F21002085
:1007F000F6F70CFD0020012329A272210090F6F7E4
:1008000041FF2D4890F89C502C480078012803D0D7
:10081000022D01DBA81EC5B2002409E0AC4203D1C1
:1008200001202749085502E0002025490855641C8D
:10083000042CF3DD21480078012808D12048214B01
:100840000022214900902148F8F744F81EE00024D6
:1008500006E01D4850F824001D4941F82400641C9E
:10086000022CF6DB184802692046641C184941F83E
:100870002020154842692046641C41F82020104879
:10088000104B002200901148F8F724F8F8BD00BF83
:10089000FCE70000B7FECEF1C6F7C1D0B1ED000015
:1008A0005B4D5DC8B7B6A820202020205B45584985
:1008B000545DCDCBB3F600007A1F002091000020DC
:1008C000B801002094010020A00100207028002021
:1008D000AC22002038B50446DCB1F6F7DFFB01217D
:1008E0000CA0FDF791FC0EA3382211460E48F9F733
:1008F000A5FF0D48F9F7F4FF01236822A02100208D
:10090000F6F784FC0020012308A272210090F6F77C
:10091000B9FE38BDC3DCC2EBD1E9D6A400000000AB
:100920003030303030300000722700205BC9CF5D9E
:10093000BCD3D6B52020202020205BCFC25DD2C6FC
:10094000B6AF000038B5044624B100203449087021
:10095000344908803248007820B1012817D0022895
:1009600032D11CE03048007850B930A0FDF764FD6A
:100970003221334803F076FB01202949087005E055
:10098000002000F073FE0220254908701CE02C486E
:1009900003F050FB10B10120FFF72AF914E001F039
:1009A00055FC80B1F6F77AFB0D2126A0FDF72CFC53
:1009B000FBF746FD01236E229F210020F6F726FC5F
:1009C00003201749087000BF00BF154800780328AE
:1009D00000D038BD1348008838B9002001231CA27C
:1009E00072210090F6F74EFE0AE00E480088C828F3
:1009F00006D1002001231CA272210090F6F742FECE
:100A000008480088401C80B206490880B0F5C87FBD
:100A100001DB0020088000F075FF00BFD9E700006F
:100A20007303002078030020D00700202020C7EBAC
:100A3000CFC8B5C7C2BC2E2E2E202020000000003B
:100A400074030020D3C3BBA7D1A1D4F100000000E0
:100A50005BC9CF5DD1A1D4F12020202020205BCF25
:100A6000C25DD1A1D4F100005B4D5DB5A5BAF42003
:100A70002020205B455849545DCDCBB3F6000000E3
:100A800000B504480021016081800120FFF7B0F823
:100A900000BD0000CC02002010B501F0E1FD00B95E
:100AA00010BD5C48007800B1FAE75B4800781B286D
:100AB00071D2DFE800F0AB0E2967646A6D717B7E4E
:100AC0008481AB878A8D90939996AB9CAB9FA2A5AE
:100AD000A800524800685249084418B1B0F5002FE8
:100AE00010D106E04F48007810B90220FFF780F8D7
:100AF00008E04D4890F8AF06012802D14BA0F9F765
:100B0000DFFB00BF00BF82E04C48FAF74BFA044617
:100B10004248006842494942884227D14748C06854
:100B200006281CD2DFE800F003070B0F1317042080
:100B3000FFF75EF813E00320FFF75AF80FE00520F7
:100B4000FFF756F80BE00620FFF752F807E00F20FA
:100B5000FFF74EF803E00720FFF74AF800BF00BF99
:100B60003648C1683648FBF73DFB07E02B48006874
:100B70003449884202D10120FFF73AF847E0F6F7FE
:100B800025FA44E000F0E4FE41E0F8F765FF3EE0BE
:100B9000FCF708FF3BE039E020480068294988421B
:100BA00003D11D494878FFF723F830E0F8F75EFEDF
:100BB0002DE0F8F7BFFE2AE0F8F70CFE27E0F8F783
:100BC00017FD24E0FBF73EFF21E0FBF7F3FF1EE0FB
:100BD000FCF7A0F91BE0FCF755FB18E0FCF726FD3D
:100BE00015E0F9F7DFFE12E0F9F718FF0FE0FCF768
:100BF00085F80CE0FCF702FB09E0FCF725FF06E0B6
:100C0000FCF74EFE03E0FDF735F800E000BF00BF43
:100C100000BF45E77E020020CC02002040000020FB
:100C2000D6FB13FF80020020D007002041542B5038
:100C30004F433D3530303030300D0A00B0290020B0
:100C4000582800202A04F40010B5002444480078F5
:100C500043498978884207D0414800784049487024
:100C600008468078087001243D4800781B2872D21D
:100C7000DFE800F0710E15191D2125292D31393DB0
:100C8000354145494D515955715D716165696D0039
:100C90003448F6F7E7FE2046FFF73CFB5BE02046D2
:100CA000FFF720FD57E02046FFF74CFE53E02046BB
:100CB000FEF7A8FF4FE02046FFF7E8FA4BE020469A
:100CC000FFF726FD47E02046FFF7E6F843E0204621
:100CD000F8F7F8FD3FE02046F8F774FE3BE02046C9
:100CE000F4F752FA37E02046F8F7A2FC33E020464A
:100CF000F8F78AFD2FE02046FBF7ECFE2BE02046BC
:100D0000FBF7A0FF27E02046FCF764F923E020462C
:100D1000FCF70EFB1FE02046FCF7D8FC1BE020464A
:100D2000FFF7D8FD17E02046FFF754FD13E02046FB
:100D3000FCF756F80FE02046FCF7F0F90BE02046F0
:100D4000FCF7E2FE07E02046FCF7DAFD03E0204670
:100D5000FCF7BAFF00BF00BF0120FDF77DFC10BD0E
:100D6000CC0200205828002010B5FEF7E7FD10BD8A
:100D700010B5FEF761FE10BD10B5FEF7B7FE10BD51
:100D800001F40072B2F5007F00D100BFCA430280B7
:100D9000704710B50022002340F66A14A14200D12A
:100DA00000BF0A1201249440A3B2DC43048010BDAA
:100DB00021B1828942F40052828104E082894DF699
:100DC000FF731A40828170471AB1838A0B43838272
:100DD00002E0838A8B438382704702460020B1F58C
:100DE000007F00D100BF13880B400BB1012000E051
:100DF0000020704770B50246002400230025002023
:100E000040F66A16B14200D100BFC1F3421501F0AD
:100E10001F03012606FA03F3012D02D19689334000
:100E200006E0022D02D1168A334001E0968A334053
:100E30000C12012606FA04F41688344013B10CB1E2
:100E4000012000E0002070BDF0B50346002400261C
:100E50000025002040F66A17B94200D100BF1846AD
:100E6000C1F3421401F01F06012707FA06F5012C11
:100E700001D10C3004E0022C01D1103000E014301C
:100E80001AB107682F43076002E00768AF430760A5
:100E9000F0BD00002DE9F04786B005460E4600245F
:100EA000A24600BFA1460027B08900B100BF2F466F
:100EB0002C8A4CF6FF700440F08804432C82AC89E5
:100EC0004EF6F3100440B088318908437189084315
:100ED0000443AC81AC8A4FF6FF400440B089044320
:100EE000AC8201A8FBF7D4F91F48874202D1DDF894
:100EF00010A001E0DDF80CA0A88900F4004040B18A
:100F00000AEBCA0000EB0A1031684900B0FBF1F8A7
:100F100007E00AEBCA0000EB0A1031688900B0FB59
:100F2000F1F86420B8FBF0F004012009642101FB12
:100F30001089A88900F4004040B1322000EBC900BC
:100F4000B0FBF1F000F00700044308E0322000EBB2
:100F500009106421B0FBF1F000F00F0004432C8174
:100F600006B0BDE8F08700000038014001468888DF
:100F7000C0F308007047C1F3080282807047000088
:100F800000B587B0012144F20400FBF767F94FF484
:100F90000070ADF8140018208DF8170003208DF8AC
:100FA000160005A92548F4F75BFF4FF48060ADF803
:100FB000140004208DF8170003208DF8160005A9F1
:100FC0001E48F4F74DFF4FF4E13001900020ADF8DA
:100FD0000800ADF80A00ADF80C00ADF810000C20C8
:100FE000ADF80E0001A91648FFF754FF012114487F
:100FF000FFF7DEFE4FF4E060F9F716FC25208DF8D0
:10100000180000208DF819008DF81A0001208DF8C5
:101010001B0006A8F9F7D0FB40210948FFF7B0FEF6
:10102000002240F227710648FFF70EFF002240F22F
:1010300025510348FFF708FF07B000BD0008014035
:10104000003801401FB504464FF4E1300090002005
:10105000ADF80400ADF80600ADF80800ADF80C00DE
:101060000820ADF80A00A4B1BDF80A0040F0040061
:10107000ADF80A0069461148FFF70CFF01210F483F
:10108000FFF796FE012240F225510C48FFF7DCFEE7
:1010900013E069460948FFF7FDFE01210748FFF705
:1010A00087FE002240F224410448FFF7CDFE0022D3
:1010B00040F225510148FFF7C7FE1FBD003801402F
:1010C00070B505460E4600240BE0295D0648FFF783
:1010D00052FF00BF40210448FFF77FFE0028F9D0EF
:1010E000641CB442F1DB70BD0038014000B585B02E
:1010F00001210420FBF7B2F801214804FBF79EF818
:101100000820ADF8100048208DF8130003208DF85A
:10111000120004A92948F4F7A3FE0420ADF810003A
:1011200018208DF8130004A92448F4F799FE4FF411
:10113000E13000900020ADF80400ADF80600ADF8F5
:101140000800ADF80C000C20ADF80A0069461C48F8
:10115000FFF7A0FE40211A48FFF712FE002240F2DE
:1011600027711748FFF770FE012240F225511448FD
:10117000FFF76AFE002240F224411148FFF764FEA7
:10118000012228210E48FFF75FFE012260210C4852
:10119000FFF75AFE01210A48FFF70AFE002009491D
:1011A000088009490880094908800949088040F2F7
:1011B0001E210848F3F701F805B000BD0008014002
:1011C000004400403200002034000020360000209F
:1011D00038000020840400202DE9F04788B0CC4876
:1011E0000088082802DA08B0BDE8F087C8480088FF
:1011F000B0F5077F18DD002240F22551C548FFF702
:1012000023FE0020C4490880C1490880C3490880E2
:10121000012240F22551BF48FFF716FE0122C0A16E
:101220001046FDF7C9FCDEE7B9480688042E00DA4F
:10123000D9E7102E01DA354600E01025B7480788B7
:1012400000240DE0BA48C05D03A90855781C80B29F
:10125000074640F21E21884200DD0027601C84B250
:10126000AC42EFDBB3A103A8F9F72EF900287DD03B
:10127000AA48078800240EE0AD48C05D0A2800D1C6
:101280000BE0781C80B2074640F21E21884200DB4A
:101290000027601C84B2B442EEDB00BFB44266DAC1
:1012A000601C85B2B5F5077F41DAA54805800024AA
:1012B00015E09F4899490988415CA148801C015567
:1012C00096480088401C80B29449088040F21E2154
:1012D000884202DB002091490880601C84B2AC4245
:1012E000E7DB00219648801C0155002240F2255181
:1012F0008848FFF7A9FD86480088401B844908807C
:10130000012240F225518348FFF79EFD8C4800885A
:10131000401C8B49088008460188801CF9F7F6F9C3
:1013200020B1012287A10020FDF746FC5BE784483D
:10133000058000241DE07E487849098810F8019056
:10134000B4F5077F03DA7E48801C00F804907348E8
:101350000088401C80B27149088040F21E218842FA
:1013600002DB00206D490880601C01E025E023E0DD
:1013700084B2AC42DFDB0021714880F81F120022EA
:1013800040F225516348FFF75FFD61480088401B2C
:101390005F490880012240F225515E48FFF754FD65
:1013A00067480188801CF9F7B1F920B1012269A1D1
:1013B0000020FDF701FC16E715E7102E00DA12E712
:1013C000564807884FF0000AD046002425E05848C8
:1013D00010F80790B9F12C0F08D1BAF1010F04DA17
:1013E0000AF1010000F0FF0A0DE018E0BAF1010F68
:1013F00009D1B8F1040F06DA4046411C1FFA81F802
:1014000001A901F80090781C80B2074640F21E2125
:10141000884200DB0027601C84B2B442D7DB00BFE7
:10142000B44200DBDFE6002001A901F8080001A8B2
:10143000F2F76AFF85B20A2D02DA4FF001080CE0DC
:10144000642D02DA4FF0020807E0B5F57A7F02DA80
:101450004FF0030801E04FF0040805EB08000E30E0
:1014600085B2AE4200DABEE6B5F5077F41DA344810
:101470000580002415E02E4828490988415C304841
:10148000801C015525480088401C80B223490880F3
:1014900040F21E21884202DB002020490880601CA7
:1014A00084B2AC42E7DB00212548801C01550022B4
:1014B00040F225511748FFF7C7FC15480088401B2C
:1014C00013490880012240F225511248FFF7BCFC65
:1014D0001B480088401C1A49088008460188801C67
:1014E000F9F714F988B101221EA10020FDF764FB71
:1014F0000BE023461FA2142103A800F0BDFB01222C
:1015000003A91046FDF758FB6DE600BF6BE600002F
:101510003400002000440040360000203800002045
:101520005B527832427566204F7665725D0000002E
:10153000840400202B5443505245435600000000C1
:10154000F20F00204D51756575652046756C6C3144
:10155000000000004D51756575652046756C6C3254
:10156000000000004D51756575652046756C6C3343
:101570000000000041744D7367427566204F766528
:1015800072205B25755D000070B505460E4600248F
:101590000BE0295D0648FFF7EEFC00BF4021044840
:1015A000FFF71BFC0028F9D0641CB442F1DB70BDCE
:1015B0000044004000B585B001210820FAF74EFE36
:1015C00001218804FAF73AFE4FF40060ADF81000EC
:1015D00048208DF8130003208DF8120004A91E483E
:1015E000F4F73EFC4FF4165000900020ADF80400D4
:1015F000ADF80600ADF80800ADF80C000420ADF819
:101600000A0069461548FFF745FC40211348FFF7DB
:10161000B7FB002240F227711048FFF715FC0122AA
:1016200040F225510D48FFF70FFC002240F2244103
:101630000A48FFF709FC01210848FFF7B9FB002021
:1016400007490880074908804FF496710648F2F769
:10165000B4FD05B000BD0000000C01400048004092
:101660003A0000203C000020A206002003494870F8
:101670000021024A9170012111707047350200204B
:101680002DE9F0419AB00646274DDFF8A080746A34
:101690006846F7F75DFD1EE0B4F5806F10D94FF492
:1016A00080624146284602F0A1F94FF48062294643
:1016B0006846F7F75FFD08F58068A4F580640AE0E6
:1016C000A2B24146284602F091F9224629466846D0
:1016D000F7F750FD0024002CDED16846F7F7D0FC68
:1016E0002F4630224FF4FF11284602F07FF91022D6
:1016F00016A907F11400F2F7AAFD58B1102216A995
:1017000007F11400F2F740FD30224FF4FF11284694
:1017100002F0E2F9102216A906F11400F2F734FDE6
:101720001AB0BDE8F0810000A837002000F01F00CB
:101730002DE9F041DFF8C0C09CF800C04FEA8C00F2
:10174000DFF8B8C01CF80070E04600F1010C18F892
:101750000C6000F1020C18F80C50E910B210FB10EC
:101760004FEAC12C0CEB421C9C441FFA8CF4DFF8AE
:1017700090C0ACF80040DFF88CC09CF800C04FEA85
:101780008C00C4461CF8007000F1010C18F80C60C5
:1017900000F1020C18F80C50E910B210FB104FEADF
:1017A000C12C0CEB421C9C441FFA8CF4DFF858C08F
:1017B000ACF80040DFF854C09CF800C04FEA8C0041
:1017C000C4461CF8007000F1010C18F80C6000F120
:1017D000020C18F80C50E910B210FB104FEAC12CA3
:1017E0000CEB421C9C441FFA8CF4DFF824C0ACF8CC
:1017F0000040BDE8F08100009F030020082B00207E
:10180000A4030020A0030020A60300209E030020C4
:10181000A203002010B500210022632803D0002875
:1018200006DB1F2804DC204B204C247843F82400DE
:101830001E4B1B78012B36D11B4B1B68002B05DB85
:10184000194B1B681F2B01DC01210CE0164B5B6858
:10185000002B05DB144B5B681F2B01DC012202E02F
:101860006323134C236079B172B10F4B1B680E4C8C
:101870006468A34204DD0C4B1B680D4C23600EE032
:1018800063230B4C23600AE021B1074B1B68084C13
:10189000236004E01AB1044B5B68054C23606323AA
:1018A000014C2360636010BDAC0200209802002050
:1018B0008C0200202DE9F84F0546AC000F4810F8C7
:1018C00004900146601C11F80080A01C0F5C4FEAD8
:1018D000E70A4FEAA80B4FEAE90000904FEACA2056
:1018E00000EB4B110098084486B23012F6F7AEFEBA
:1018F000F0B2F6F7ABFEBDE8F88F0000082B002031
:1019000000BFFEE710B510480078012802D0022879
:1019100017D10BE000F09AFC38B1FAF791FD0120E5
:101920000A4908700020084908700AE000F08EFC9F
:1019300030B1FAF785FD00200449087002490870AB
:1019400000BF00BF10BD0000E0020020E102002047
:1019500010B58EB04D480078002865D14C48C0883D
:1019600010BB4C4800684C4988421DD14B48B0F828
:101970006800052807DB4948B0F86800401F474960
:10198000A1F8680009E04548B0F8680028B9434864
:101990008089401E4149A1F868000120FFF766FEDA
:1019A00001203A49087029E03948C088401C38496C
:1019B0008988884222D137480068394988421DD138
:1019C0003848007840B13548B0F868003049898817
:1019D00008443249A1F868003048B0F86800401C5B
:1019E0002E498989884203DB00202C49A1F8680030
:1019F0000220FFF73BFE0220244908702448F7F735
:101A00003FF80446234800682749884206D1002051
:101A1000244908700220FEF7EBF833E023488442A3
:101A200030D11E48808900B92DE01948C08800EBEC
:101A3000400101EBC0011948A03050F821301CA230
:101A4000322101A800F018F901A8F8F739FC104874
:101A5000C08800EB400101EBC0011048A03000EB52
:101A60008100431D17A2322101A800F005F90122CF
:101A700001A90020FDF7A0F80120FEF7B9F8002029
:101A80000249087000BF00BF0EB010BDE002002088
:101A900070280020400000202A04DC00D00700202D
:101AA0002A04BC00E10200202A04F4002A04EC000D
:101AB00041542B504F433D30413030303025303889
:101AC000780D0A00BAF4BDD03A25730010B586B07F
:101AD00000F036F810211848F4F7A1FA0020ADF80C
:101AE00004004FF48270ADF806000020ADF8080045
:101AF0000220ADF80A000120ADF80C004002ADF85C
:101B00000E000020ADF81000ADF812000720ADF86F
:101B1000140001A90948FAF71DFF01210748FAF747
:101B2000FFFE4FF47A70F3F7E6FC01F08DFF0446F8
:101B3000012006B010BD0000000801400030014047
:101B400008B501210420FAF789FB01210803FAF7FF
:101B500085FB2020ADF8000003208DF8020018203E
:101B60008DF8030069460F48F4F77AF98020ADF844
:101B7000000069460B48F4F773F94020ADF8000007
:101B800004208DF8030069460648F4F769F910202F
:101B9000ADF800008DF8030069460248F4F760F9DB
:101BA00008BD00000008014010B502460846012AA1
:101BB00005D1CB1DDC1703EB5474E01012E0042AAE
:101BC00004D14B1C03EBD37460100BE0102A01D13D
:101BD000480007E0182A02D101EB410002E0202A68
:101BE00000D1880000E0401C00F00303002BFAD174
:101BF00010BD00002DE9F04705460E469046B5F1B0
:101C0000006F02D31348854201D3BDE8F087C5F3C6
:101C1000090000B1F9E7F3F73DFE2846F3F7D0FDE0
:101C20000746042F00D0F0E700240CE0315D601C73
:101C3000305C01EB00201FFA80F928194946F3F7C0
:101C400009FEA01C84B24445F0DBF3F7F9FD00BFA8
:101C5000DBE70000000002080FB4054B10B503A934
:101C6000044A029800F044F810BC5DF814FB000030
:101C700029220108B40300200FB41CB50A46521EE5
:101C8000CDE9000207A9054B6A46069800F030F836
:101C9000009A002111701CBC5DF814FB532101084F
:101CA0000FB4084B10B504A902AA039800F020F85D
:101CB000044602A9002000F057FA204610BC5DF847
:101CC00014FB00006921010800487047B803002098
:101CD00002E008C8121F08C1002AFAD170477047F5
:101CE000002001E001C1121F002AFBD17047000053
:101CF0002DE9FF4F8DB00F460546002606E025284A
:101D00000BD0DDE90F1290476D1C761C2878002857
:101D1000F5D111B03046BDE8F08F0024A246A146AF
:101D20000122EC4900E0044315F8013F203B02FA90
:101D300003F00842F7D128782A2810D06FF02F023C
:101D40002878A0F13001092914D80AEB8A0102EBA6
:101D5000410144F0020400EB010A6D1CF0E701CFE1
:101D60005FEA000A03D544F40054CAF1000A44F0C3
:101D700002046D1C28782E2817D115F8010F44F0A5
:101D800004042A280ED06FF02F022878A0F1300129
:101D900009290AD809EB890102EB410100EB01098D
:101DA0006D1CF2E757F8049B6D1C28786C280FD047
:101DB00006DC4C2817D068280DD06A2814D104E01E
:101DC000742810D07A280FD10DE044F400140AE0F2
:101DD00044F4801401E044F440146978814202D153
:101DE00004F580146D1C6D1C2A786E2A1FD00CDC43
:101DF000632A31D004DC002A8BD0582A11D1A3E009
:101E0000642A68D0692A0CD165E0732A2ED004DCDC
:101E10006F2A73D0702A04D19BE0752A6FD0782A7C
:101E20006ED01046DDE90F129047761C50E1C4F3E6
:101E30000250022806D0032809D0042801CF09D077
:101E4000066045E101CFF117C0E9006140E101CF33
:101E500006803DE106703BE117F8040B8DF80000A9
:101E600000208DF80100EB46012003E057F804BB89
:101E70004FF0FF3061074FF0000102D40DE008F190
:101E80000101884649450FDA8045F8DB1BF8081048
:101E90000029F4D108E008F1010188468142FADB0B
:101EA0001BF808100029F6D1DDE90F23AAEB080082
:101EB0008146214600F036F9304400EB080604E084
:101EC000DDE90F121BF8010B9047B8F10108F7D2BA
:101ED00021464846F7E00A21C4F302534FF0000BB5
:101EE0000891022B04D001CFC117032B09D00AE0BF
:101EF000FF1D27F00707F7E8020108E032E01FE0C6
:101F000020E000B2C117042B01D140B2C117031E5B
:101F100071F1000307DA4FF0000CD0EB0C006CEB12
:101F200001012D2302E0230504D52B238DF8243055
:101F3000012303E0E30701D02023F7E7984658E0A8
:101F40000A2110E010210EE010204FF0000B089045
:101F50000CE010214FF0000B44F004044FF008098E
:101F6000089103E008214FF0000B0891C4F30253DD
:101F7000022B04D001CF0021032B06D006E0FF1D69
:101F800027F00707F7E8020103E080B2042B00D135
:101F9000C0B24FF0000823072BD5702A07D0DDF818
:101FA00020C08CF0100C5CEA0B0C05D00EE0402336
:101FB0008DF82430012308E050EA010306D03023D5
:101FC0008DF824308DF8252002239846DDF820C0B6
:101FD0008CF0080C5CEA0B0C0BD150EA010301D128
:101FE000630706D530238DF824304FF00108A9F19E
:101FF0000109582A04D038A20B9208AA0A920BE0D1
:102000003AA2F9E75B46089AF2F74AFB0B9B9B5C06
:102010000A9A521E0A92137050EA0102F2D10A98EB
:10202000ADEB000000F1200B600702D524F48034F2
:1020300001E04FF00109D94502DDA9EB0B0000E0FA
:10204000002000EB0B0141440890AAEB010AE003D9
:1020500006D4DDE90F232146504600F063F806441C
:102060004FF0000908E009A911F80900DDE90F1295
:10207000904709F10109761CC145F4DBE0030CD55A
:10208000DDE90F232146504600F04CF8064404E0F9
:10209000DDE90F1230209047761C0899481E089001
:1020A0000029F5DC08E00A980A990078491C0A9191
:1020B000DDE90F129047761CBBF10001ABF1010B7B
:1020C000F1DC21465046DDE90F2300F019F8064403
:1020D0006D1C1BE6092801003031323334353637A8
:1020E0003839616263646566000000003031323364
:1020F0003435363738394142434445460000000004
:102100002DE9F041044600251E461746880404D4F4
:1021100005E039462020B0476D1C641EF9D52846DD
:10212000BDE8F0812DE9F041044600251E469046A9
:10213000C80301D5302700E02027880404D505E036
:1021400041463846B0476D1C641EF9D52846BDE8A7
:10215000F0814A68002A06D00A68531C0B60107090
:102160004868401E486070470A68531C0B60107036
:102170007047000070B504462646012210A10020D9
:10218000FCF71AFD12A0F8F79BF816B1012E08D142
:1021900003E013A0FCF750F904E014A0FCF74CF99D
:1021A00000E070BD00BF062506E0F5F761FB642086
:1021B00001F04BFF681E05B2002DF6DA00BFF0E714
:1021C00054727920746F205077724F666600000059
:1021D0004154245143505752444E0D0A0000000010
:1021E000D5FDD4DAB9D8BBFA00000000B5CDD1B91D
:1021F000B9D8BBFA0000000010B5C821054801F0AD
:1022000031FF012004490870012204A10020FCF7DD
:10221000D3FC10BD300200203402002053656E64F0
:1022200020656E61626C650070B504460D46E1B2D2
:102230000548FEF7A0FE00BF40210348FEF7CDFD94
:102240000028F9D0204670BD0038014003490878C5
:10225000097811B10021014A11707047380200203D
:1022600000200A4991F89C1005290CD2DFE801F002
:10227000030405070A0006E005E0054803E00448FA
:10228000283000E000BF00BF704700007A1F002028
:102290000721002010B50024114890F89C00052863
:1022A0000ED2DFE800F0030608090A000C4CC53422
:1022B00006E00C4C04E003E002E00A4C503400BF9E
:1022C00000BF1CB900200849087003E021460648F9
:1022D000F1F7CAFF012005490870204610BD000033
:1022E0007A1F00208F20002030280020A00000202E
:1022F00010B504461BA12046F8F7E6F820B11EA150
:102300002046F8F7E1F818B901202049087022E0CA
:102310001FA12046F8F7D8F820B122A12046F8F7EF
:10232000D3F818B902201949087014E022A12046F8
:10233000F8F7CAF820B124A12046F8F7C5F818B973
:1023400003201249087006E000201049087023A1FC
:102350002046FFF7A5FC002221461046FCF72CFC86
:1023600010BD00004D6F64656C3A2055393530372B
:10237000435F53584E5400004D6F64656C3A2055CE
:1023800039353037432053584E5400009102002015
:102390004D6F64656C3A205539353037435F53587B
:1023A0004E4D00004D6F64656C3A2055393530371D
:1023B000432053584E4D00004D6F64656C3A2055D4
:1023C00039353037430000004D6F64656C3A205555
:1023D0003935303743205633000000004D6F6465B7
:1023E0006C3A4E6F6E650D0A00000000FEB50446A3
:1023F000002221461046FCF7DFFB0026002530E0D6
:10240000605D5F282BD1701CC6B2012E08D1E81C7C
:10241000205C8DF80000281D205C8DF801001EE076
:10242000032E1CD1A81C205C8DF80200E81C205C47
:102430008DF80300281D205C8DF80400681D205CC9
:102440008DF8050000208DF806006846F1F75CFF66
:10245000074908600846016806A0FFF7FDFB681CF5
:1024600005B22046F1F7DEFEA842C9D8FEBD000045
:10247000740000204D6F64656D5665723A25640DD9
:102480000A00000010B50024104890F89C000528B0
:1024900010D2DFE800F00306090B0D000B4C9D3451
:1024A00008E00A4CED3405E0094C03E0084C01E07B
:1024B000084C00BF00BF28210748F1F77EFE2146E7
:1024C0000548F1F7D1FE204610BD00007A1F00201C
:1024D00084400108B72000200828002010B50446D9
:1024E000A07B302804D10020074981F8B40603E01E
:1024F0000120054981F8B406034890F8B41603A0FA
:10250000FFF7AAFB10BD0000D0070020506F634307
:102510006F64653A25640D0A000000002DE9F04162
:102520008CB004462046F1F77DFE8046002700254A
:1025300026E0605D0D2817D1002002A9C85502A829
:10254000F1F7E2FE064633460FA2282102A80094C6
:10255000FFF792FB002202A91046FCF72DFB0E4864
:1025600006600CB0BDE8F081605D302807DB605D7F
:10257000392804DC625D38467F1C02A90A546D1CB0
:102580004545D6DB00BFECE7504F437665723A25F0
:10259000643C2D3E257300007800002010B501201A
:1025A0000249087001F066FD10BD000043020020E2
:1025B00070B5ADF5936D0546302229460DF58D6059
:1025C00001F014FA2549DDF89404884203D0012073
:1025D0000DF5936D70BDDDF88C04B0F5805F01D909
:1025E0000220F5E705F58056DDF88C440DF5806096
:1025F000F6F7AEFD20E0B4F5806F11D94FF480629C
:102600003146684601F0F2F94FF4806269460DF5F3
:102610008060F6F7AFFD06F58066A4F580640BE0F8
:10262000A2B23146684601F0E1F9224669460DF54D
:102630008060F6F79FFD0024002CDCD10DF5806052
:10264000F6F71EFD10220DF27C410DF58B60F1F7BF
:10265000FEFD08B10320BBE70020B9E7311B2008CD
:102660000648006838B1054801780068401E034AF2
:102670001060C8B270470020FCE700008402002010
:1026800030B587B00C240E48007820B90DA102A8FF
:10269000FFF706FB03E00DA102A8FFF701FB02A86C
:1026A000F1F7C0FD0546012004F14001009088B219
:1026B000012302AA3821F4F7E5FF07B030BD00007E
:1026C000EE000020B9D8B1D500000000B4F2BFAAD6
:1026D0000000000010B504460A20734908707348D2
:1026E000047073A21E217348FFF7C6FA6F48007882
:1026F0000D281FD2DFE800F0071F2F3F4F5F6073E8
:102700008595A5B5C5003C206749087001226AA1DE
:102710000020FCF751FA6CA232216D48FFF7ACFAA9
:102720006CA21E216C48FFF7A7FA6CA21E2161481B
:10273000FFF7A2FAB5E001226BA10020FCF73CFAFA
:102740006EA232216248FFF797FA6EA21E216248FC
:10275000FFF792FAA5E001226CA10020FCF72CFA09
:102760006FA232215A48FFF787FA70A21E215A48F9
:10277000FFF782FA95E0012270A10020FCF71CFA15
:1027800072A232215248FFF777FA74A21E215248F2
:10279000FFF772FA85E0012273A10020FCF70CFA22
:1027A00075A232214A48FFF767FA78A21E214A48EB
:1027B000FFF762FA75E000BF012278A10020FCF764
:1027C000FBF97AA0F7F77CFD7FA232214048FFF7A2
:1027D00053FA82A21E214048FFF74EFA61E001221F
:1027E00082A10020FCF7E8F9FAF772FB82A23221FD
:1027F0003748FFF741FA88A21E213748FFF73CFA15
:102800004FE0012285A10020FCF7D6F987A23221F2
:102810002F48FFF731FA88A21E212F48FFF72CFA24
:102820003FE0012288A10020FCF7C6F989A23221ED
:102830002748FFF721FA8BA21E212748FFF71CFA31
:102840002FE001228AA10020FCF7B6F98BA23221E9
:102850001F48FFF711FA8CA21E211F48FFF70CFA40
:102860001FE001228AA10020FCF7A6F98CA23221E8
:102870001748FFF701FA8EA21E211748FFF7FCF94F
:102880000FE001228CA10020FCF796F98EA23221E4
:102890000F48FFF7F1F991A21E210F48FFF7ECF95D
:1028A00000BF00BF10BD000097020020960200206C
:1028B00040234000EA270020576169744D6F64652A
:1028C0006D52756E2E2E0000415445300D0A0000E9
:1028D0009A2700204F4B0000CC2700202B504F435D
:1028E0003A535441525400004765744D6F64656D0E
:1028F0004D6F64756C652E2E000000004154490D2B
:102900000A0000004D6F64656C3A00004765744D25
:102910006F64656D56657273696F6E2E2E000000D0
:1029200041542B4C435453570D0A0000496E6E65B9
:102930007256657273696F6E3A0000004765745095
:102940006F6356657273696F6E2E2E0041542B5063
:102950004F435F5645523F0D0A0000002B504F4336
:102960005F5645523A000000476574506F63436FED
:1029700064652E2E0000000041542B504F433D341F
:10298000303030303030300D0A0000002B504F43D3
:102990003A343030303030303030000053657454C9
:1029A000545353706565642E2E00000041542B4C27
:1029B000534854545353504545443D2D312C3730E2
:1029C00030300D0A0000000041542B4C5348545441
:1029D0005353504545443F0D0A0000002B4C5348CB
:1029E00054545353504545443A00000053657453C2
:1029F000706B4D69632E2E0061742B737973636D58
:102A0000643D73746172745F70636D20766F6C7572
:102A10006D650D0A000000003720370047657443DC
:102A20006172645374617475732E2E0041542B438C
:102A300050494E3F0D0A00002B4350494E3A205258
:102A40004541445900000000476574494D45492EF1
:102A50002E00000041542B4C5348494D45490D0A66
:102A6000000000002B4C5348494D45493A000000F6
:102A700047657449434349442E2E000041542B4975
:102A8000434349440D0A00005E534349443A000061
:102A9000476574504F43506172612E2E0000000054
:102AA00041542B504F433D3032303030300D0A000E
:102AB0002B504F433A303200536574506F63534D7F
:102AC0006F64652E2E00000041542B504F433D3162
:102AD000303030303032300D0A0000002B504F4380
:102AE0003A313030303030303000000038B54FF4FB
:102AF000FA70F4F799FEF9F75FFCFEF741FA4E48D9
:102B000000686422B0FBF2F1B1F1807F01D30120B3
:102B10001DE021F07F40401E4FF0E0225061501731
:102B20000F22002807DA13071D0E444B00F00F0494
:102B3000241F1D5503E013071C0E414B1C5400BFFE
:102B400000204FF0E022906107201061002020B1AA
:102B50003CA0FFF781F800BFFEE7FEF7C7FAFEF7DB
:102B600029FDF7F789FBF9F7EBFAFEF7AFFFF2F76C
:102B7000B0FEF5F70DF9FCF701F9F6F7A7FFF1F74D
:102B8000EDFEF5F781FDF5F7D1FBF4F715FCF2F753
:102B9000E3FAF6F745FBF4F76BFE00F0D1F8FBF72C
:102BA00027FCF7F7D5FEFCF7D7FAF3F7BFFAFDF7E6
:102BB00067FFFCF7BBF84FF4807028494861F9F7CC
:102BC000E5FCF4F7DBF92648B0F82F20022300F1EA
:102BD000210124A0FFF740F82148D0F81D1027A0BC
:102BE000FFF73AF82848F4F7C5F8012803D1264939
:102BF00026A0FFF731F8002027490880FAF706FDE4
:102C00002648408810B93C202449488001200C23E4
:102C1000A022002100900846F4F756FB02201A2358
:102C2000A0220D2100900020F4F74EFB00F04EFB97
:102C300000F0ECFD002038BD1800002018ED00E089
:102C400000E400E05379735469636B5F436F6E6611
:102C50006967206572720D0A0000000000100140D3
:102C6000381F00200D0A25735F5625642E25642029
:102C700053746172742E2E2E0D0A000050534E3A7A
:102C8000256C750D0A0000006A1F002068617264DF
:102C900049443A25730D0A00A40000207A1F002041
:102CA000F0B587B0054641F2BF2605FB06F0224984
:102CB00091FBF0F084B2204604EBD0714F1001215B
:102CC0000820F9F7BBFA0020ADF81600ADF8106047
:102CD000ADF812008DF81800601E80B2ADF8140037
:102CE00004A91648FCF7E6F9ADF806707020ADF8B7
:102CF00000000120ADF802000420ADF8040002201D
:102D0000ADF808000020ADF80A004FF48070ADF86F
:102D10000C000020ADF80E00ADF8067069460748BB
:102D2000FCF776F901210548FCF756F90121034823
:102D3000FCF75EF907B0F0BD006CDC02000C00404F
:102D400070B5002536A0F3F78FFC374908600846B8
:102D50000068002804DA32A134A0FEF77DFF70BDC0
:102D600031480068F3F79CFC0446B4F54C7F04D866
:102D70002BA132A0FEF770FFF1E7364B40F2313263
:102D8000002129480068F9F7A9FB0420324908709E
:102D9000304890F89C00042804DD00202D4981F87B
:102DA0009C0001252B4890F8DD01032804DD00205C
:102DB000284981F8DD010125264890F89A00052868
:102DC00004DB0020234981F89A000125214890F86E
:102DD000F902072804DB00201E4981F8F9020125C9
:102DE0001C4890F83003032804DB0020194981F8BF
:102DF000300301251748007818B9012015490870DB
:102E00000125FFF747FA15491248853002680A6024
:102E10008088888015B10020F7F76AFB00BF9EE725
:102E20007379732E696E69009C0000202573206EF3
:102E30006F7420666F756E640D0A00002573205351
:102E400059535F434F4E464947206C656E2065726B
:102E5000720D0A007A1F0020C80000209400002094
:102E600010B5F4F709FEFCF725F8134890F89A100E
:102E7000903000EB4100008800281BDD0F480088DF
:102E8000401C81B20D4801800B4890F89A20903088
:102E900000EB4200008881420CDB002007490880DB
:102EA0000748407818B90120F5F7C0F902E0002082
:102EB000F5F7BCF910BD00007A1F0020A400002027
:102EC000D007002010B50948007800B910BD0848A7
:102ED00001F0B0F800B9F9E70020044908700122B8
:102EE00004A1FBF769FE00BFF0E7000034020020F8
:102EF0003002002053656E642064697361626C6502
:102F0000000000002DE9F34FA3B0814600201E9081
:102F10001F90209021901C901D9040210CA8F1F74B
:102F20004CF90020089009900A900B90002600258B
:102F300000240690059000BF0CA840F8269024E0DD
:102F400019F804002C281CD108A905988855059863
:102F500018B900200CA941F8260000200590701C2B
:102F6000C6B209EB0400401C0CA941F826000CA8CD
:102F700050F8260040782A2806D1012008A9885553
:102F800002E00598401C0590641C24988442D7D325
:102F90000C9858B39DF820201EA80C99F1F736F92B
:102FA0001CAA06211EA800F0BBFF9DF8700000F0CF
:102FB0000F0A9DF8700000F0F00007900AF1080A6F
:102FC000BAF10A0F07DBAAF10A0000F0FF0A07981E
:102FD0001030C0B20790079840EA0A00B6498873DB
:102FE0009DF87100C8739DF8720008740D98E0B1E7
:102FF00000201E901F90209021909DF821201EA857
:103000000D99F1F703F99DF87800412807D1AA48F6
:10301000007820F00200801CA749087005E0A6484F
:10302000007820F00200A4490870A3480078C0F39B
:10303000400010B925B0BDE8F08F0E98002843D0AD
:1030400000201E901F90209021901C901D909DF8B4
:1030500022200DF179000E99F1F7D8F830208DF883
:103060007800052504E01EA9681C085C48556D1C05
:10307000082DF8DB00208DF880001CAA08211EA86E
:1030800000F04EFF00201E901F90209021900F987E
:10309000D0B19DF823201EA80F99F1F7B7F89DF83D
:1030A0007800854981F86C009DF873009DF87210D6
:1030B00040EA01209DF8711040EA01409DF870102F
:1030C00040EA01607C4988611098E0B300201E90BE
:1030D0001F90209021901C901D909DF824201EA8E8
:1030E0001099F1F793F8052504E01EA9681C085C07
:1030F00048556D1C082DF8DB00208DF880001CAAB7
:1031000008211EA800F00CFF1198E0B100201E90CD
:103110001F90209021909DF825201EA81199F1F76D
:1031200075F89DF87800644981F86D009DF873008A
:103130009DF8721040EA01209DF8711040EA0140AC
:103140009DF8701000E003E040EA01605A494861D0
:10315000129800285ED000201E901F902090219091
:103160009DF826201EA81299F1F750F8002405E0DA
:103170001EA8005D2E2800D104E0641C9DF82600E6
:10318000A042F5DC00BF9DF82600001B401E069003
:103190001EA8F1F7B9F80390F1F758FA07468846E8
:1031A0000698002814DD1EAA611C515CA1F13000B4
:1031B000F1F74CFA414A424BCDE90001F1F765F9CC
:1031C0003A464346CDE90201F1F7B8F8074688468A
:1031D0003C4A3D4B38464146F1F757F9CDE90201EB
:1031E000F1F745FA1FFA80FB64209BFBF0F0000228
:1031F0000A219BFBF1F10A2291FBF2F302FB13116E
:1032000040EA011011469BFBF1F201FB12B10843A9
:103210002949C861139878B300201E901F90209010
:1032200021909DF827201EA81399F0F7EFFF1EA804
:10323000F1F76AF880B204904FF4B471049890FBEF
:10324000F1F201FB120080B204906421049890FB1B
:10325000F1F001020A22049890FBF2F090FBF2F3E5
:1032600002FB130041EA0010049991FBF2F302FB08
:1032700013110843104908621498D8B100201E9019
:103280001F90209021901C901D909DF828201EA832
:103290001499F0F7BBFF1CAA06211EA800F040FEFF
:1032A0009DF87000044948739DF8710008739DF8FB
:1032B0007200C87200BFBDE6C02200209A99999999
:1032C0009999B93F6F1283C0CAA1FD3F10B50C4850
:1032D000F7F73AFC00200B4908800B4908800B499E
:1032E00008800B4908800B4908800B4908800B496E
:1032F00008800B4908800B4908800B49088010BDE5
:1033000050020020540200205602002058020020E3
:103310005A0200205C0200205E02002060020020B1
:1033200062020020640200206602002070B504469C
:103330000125208810B1272820D117E01DE0F2F7E1
:10334000FBFEF8F715FFF2F7A1F8F4F705FDF6F725
:103350003FFFFFF7B7FDF4F7A5FA01220A490B4832
:10336000F7F700FC00BF2720208000BF0648F7F7D2
:10337000EDFB08B9002070BD00BFE0E700BF0025ED
:10338000002020800320F6E76C020020500200207D
:1033900070B50446F2F746FE0125208810B13628A4
:1033A00014D10BE011E0F3F7B7FD32220A490B48C4
:1033B000F7F7D8FB00BF3620208000BF0648F7F79C
:1033C000C5FB08B9002070BD00BFECE700BF0025B9
:1033D000002020800320F6E7C801002050020020D2
:1033E00070B504460125208810B1502815D10CE095
:1033F00012E00020F5F784F90F220B490B48F7F78C
:10340000B1FB00BF5020208000BF0748F7F79EFBAC
:1034100008B9002070BD00BFEBE700BF0025002009
:1034200020800320F6E700007802002050020020F0
:1034300070B504460125208810B1422814D10BE054
:1034400011E0F6F757FB01220A490B48F7F78AFB10
:1034500000BF4220208000BF0648F7F777FB08B97D
:10346000002070BD00BFECE700BF002500202080D9
:103470000320F6E774020020500200202DE9F041FD
:103480000446804E01272088E22847D003DC40B163
:10349000DE2870D12AE0FA286ED0B0F5897FF8D105
:1034A000E1E0E8E000BF012277A10020FBF784FB08
:1034B0004FF4D7617848F0F780FE0120FAF70EF854
:1034C0000420764908610020754908707549086034
:1034D000F7F766F90220744908606422734974485A
:1034E000F7F740FB00BFDE20208000BF6F48F7F7F2
:1034F0002DFB10B90020BDE8F08100BF02206A4911
:10350000091D08600120091F086064226749684896
:10351000F7F728FB00BFE220208000BF6348F7F7E1
:1035200015FB08B90020E6E700BF01205E49091D30
:1035300008600020FFF7CEF84FF400715A481038A9
:10354000F2F762FD012802D15A49087002E0042016
:103550005249486101205249087000BF0020564975
:1035600008705649088041E05548F6F7A9FE192031
:10357000544908802BE07FE022E05348007800B1F6
:1035800056E040F21E21B01CF7F73AF880B23080C6
:1035900068B14E49B01CF6F797FF20B14C49B01CFA
:1035A000F6F792FF98B901204349087026E00222FD
:1035B0003E493F48F7F7D6FA00BFFA20208000BF07
:1035C0003A48F7F7C3FA08B9002094E700BF3D482E
:1035D00001880088401E00B23A4A10800029CCD1F0
:1035E00036480088401C00B2344908803348B0F99E
:1035F0000000384909788842B6DB00BF2E480078C1
:10360000F6F77AFC054605B9A8E7002D0FDA681C25
:1036100038B9012230A10020FBF7CEFAF2F7A6F864
:1036200005E0A81C18B904201B4981F8B30600BFA7
:1036300004201A49486101202E4908702E4908705B
:1036400018E0154890F8B10600B12CE700201249A7
:103650000872642215491648F7F784FA00BF4FF440
:103660008970208000BF1148F7F770FA08B9002070
:1036700041E700BFE5E715E700BF002700202080F5
:10368000032038E7121200204D6F64656D496E69A2
:10369000742E2E2E00000000D007002000100140E4
:1036A0009502002078000020100C01409C020020B0
:1036B000500200207F020020A1020020A202002070
:1036C0009A270020A402002088020020CC27002096
:1036D000EA270020970200204D6F64656D496E69EE
:1036E0007454696D656F7574204754204D6F64651F
:1036F00000000000930200209202002070B50446F2
:103700000125208810B10A2814D10BE011E0FDF743
:1037100063FD01220A490B48F7F724FA00BF0A208B
:10372000208000BF0648F7F711FA08B9002070BDE5
:1037300000BFECE700BF0025002020800320F6E753
:10374000B40200205002002070B5044601252088F4
:1037500010B136281AD111E017E0F8F73BFEF1F767
:10376000DDFCFFF77DFBF2F757FA64220A490B48AC
:10377000F7F7F8F900BF3620208000BF0648F7F7BA
:10378000E5F908B9002070BD00BFE6E700BF0025DD
:10379000002020800320F6E7700200205002002065
:1037A00070B504461548007820B100F029FB0020D0
:1037B000124908700125208810B12A2817D10EE07F
:1037C00014E00F48007808B900F042FB32220D499E
:1037D0000D48F7F7C7F900BF2A20208000BF09482D
:1037E000F7F7B4F908B9002070BD00BFE9E700BFE2
:1037F0000025002020800320F6E70000D0010020F3
:1038000088020020CC010020500200201FE0F4F7C5
:10381000EDF80F48FFF78AFD0E48FFF795FF0E48B9
:10382000FFF706FE0D48FFF769FF0D48FFF726FE7C
:103830000C48FFF7D5FD0C48FFF7B2FF0B48FFF728
:10384000A7FD0B4800F088F80A4800F01DF8DEE7F5
:103850005402002056020020580200205A02002084
:103860005C0200205E020020600200206202002054
:10387000640200206602002010B50248F7F77AF9CA
:1038800010BD00005002002070B5044601252088BC
:1038900010B1852852D149E04FE02B48007800282C
:1038A0003BD02948407820B1012813D0022833D1D9
:1038B00021E02548807858B901210846FAF7F4FF3D
:1038C00028B101202149087000201F49087000BF5D
:1038D00000BF21E01C48807858B900210846FAF75B
:1038E000E3FF28B10120194908700020164908702B
:1038F00000BF00BF10E01448807858B901210020B3
:10390000FAF7D2FF28B101201049087000200E49B3
:10391000087000BF00BF00BF00BF01220C490D4866
:10392000F7F720F900BF8520208000BF0848F7F78F
:103930000DF908B9002070BD00BFAEE700BF00253B
:10394000002020800320F6E7350200203802002006
:103950003C0200205002002070B50446012520885A
:1039600010B1152816D10DE013E0FDF76DF9FDF744
:1039700093F801220A490B48F7F7F4F800BF152025
:10398000208000BF0648F7F7E1F808B9002070BDB5
:1039900000BFEAE700BF0025002020800320F6E7F3
:1039A000E40200205002002010B50446240300F079
:1039B000EDF800F087F810210B48F2F72EFB2020DD
:1039C000F8F7E6FFC4F30740F8F7E2FFC4F3072077
:1039D000F8F7DEFFE0B2F8F7DBFF10210248F2F75C
:1039E0001EFB00F06FF810BD000801402DE9F0410A
:1039F00005460C46174610211248F2F70EFB0B2025
:103A0000F8F7C6FFC4F30740F8F7C2FFC4F3072076
:103A1000F8F7BEFFE0B2F8F7BBFFFF20F8F7B8FFFA
:103A20002870002605E0FF20F8F7B2FFA855701CAB
:103A300086B2BE42F7DB10210248F2F7F0FABDE889
:103A4000F0810000000801402DE9F041002400252C
:103A50000026002710210F48F2F7DFFA9F20F8F721
:103A600097FFFF20F8F794FF0546FF20F8F790FF37
:103A70000646FF20F8F78CFF074610210548F2F7AD
:103A8000CEFA280440EA062040EA07042046BDE8B2
:103A9000F08100000008014010B500241021084802
:103AA000F2F7BBFA0520F8F773FFFF20F8F770FF75
:103AB000044610210248F2F7B2FA204610BD000079
:103AC0000008014010B500BFFFF7E6FF00F001005D
:103AD0000028F9D110BD00002DE9F04781460F46BE
:103AE00016464FEA1738C7F30B0ACAF58054A642A8
:103AF00000DC344644E04FEA08314FF4805222485B
:103B0000FFF774FF002508E00AEB05001E49085C7A
:103B1000FF2800D003E0681C85B2A542F4DB00BF9B
:103B2000A54216DA4046FFF73FFF002507E019F8E7
:103B3000050005EB0A01144A5054681C85B2A542E1
:103B4000F5DB4FEA08314FF480520F4800F02EF8B1
:103B500004E022463946484600F028F8A64200D143
:103B60000FE008F101084FF0000AA1442744301B80
:103B700086B2B6F5805F02DD4FF4805400E0344633
:103B8000B9E700BFBDE8F087A83B002010B51021C1
:103B90000548F2F742FA0620F8F7FAFE102102482B
:103BA000F2F73DFA10BD0000000801402DE9F04198
:103BB00007460E461446F0B2C0F58075AC4200DCF4
:103BC000254612E02A463146384600F013F8AC424A
:103BD00000D10BE02F442E44601B84B2B4F5807FEB
:103BE00002DD4FF4807500E02546EBE700BFBDE83D
:103BF000F08100002DE9F04106460C461746FFF71C
:103C0000C5FF10211048F2F708FA0220F8F7C0FEAD
:103C1000C4F30740F8F7BCFEC4F30720F8F7B8FE7A
:103C2000E0B2F8F7B5FE002504E0705DF8F7B0FEED
:103C3000681C85B2BD42F8DB10210348F2F7EFF9AA
:103C4000FFF740FFBDE8F0810008014010B50446D1
:103C50001CB904A0FAF7F0FB02E005A0FAF7ECFBB0
:103C600010BD0000D5FDD4DAC9E8D6C300000000BD
:103C7000C9E8D6C3CDEAB3C90000000030B589B0A9
:103C8000002416E004EB840000EB44110B480D18EF
:103C9000687860B1A87850B1631C09A21E2101A800
:103CA000FDF7EAFF01A8F6F70BFB0020A870601CE7
:103CB000C4B2022CE6DB09B030BD0000CB240020EA
:103CC00041542B544350434C4F53453D25640D0AFA
:103CD0000000000010B500242A4800780B282DD2DF
:103CE000DFE800F0060A112C182C1C2C20242800D8
:103CF00025A0F6F7E5FA21E027A0F6F7E1FA012082
:103D0000284908701AE028A0F6F7DAFA00202549B9
:103D1000087013E027A0F6F7D3FA0FE029A0F6F712
:103D2000CFFA0BE02BA0F6F7CBFA07E02CA0F6F7C2
:103D3000C7FA03E02DA0F6F7C3FA00BF00BF114891
:103D40000078401CC0B20F4908700A2801DB00202F
:103D500008702948007802280DD1284800782649A3
:103D60000978884201D0FFF789FF2348007823496A
:103D70000870012010BD20480078204908702046B6
:103D8000F8E70000D101002041542B504F435F5011
:103D900050503F0D0A00000041542B434353510D36
:103DA0000A0000009802002041542B4353510D0A91
:103DB0000000000041542B4D4F444F445245583FA2
:103DC0000D0A000041545E535953494E464F0D0AA7
:103DD0000000000041542B5544503F0D0A000000E4
:103DE00041542B474749503F0D0A000041542B478F
:103DF0005049503F0D0A0000D5010020D20100209B
:103E000010B54B210148F0F7D8F910BDCA240020A5
:103E10002DE9F04105460E461746681E00F0FF08E2
:103E2000B8F1020F01DBBDE8F08108EB880000EB80
:103E3000481106480C18607800B9F4E7D4F81D2042
:103E400039463046904700BFEDE70000CB24002004
:103E50002DE9F0414FF00008FFF73CFF08B1BDE845
:103E6000F081002521E00DB9002701E01348077813
:103E70003C4615E004EB840000EB44110F48401C65
:103E80000E18707850B125B9D6F819102046884719
:103E900004E02046F5F7A2F800B103E0601CC4B2CC
:103EA000022CE7DB00BF681CC5B2022DDBDB022C55
:103EB00002DB00200149087000BFD0E7CA240020BF
:103EC0002DE9F04107460D469046A7F13100C6B2F4
:103ED000022E01DBBDE8F08106EB860000EB461107
:103EE0000E480C18607800B9F4E7B8F1000F09D15A
:103EF000312D02D10120A0700DE0302D0BD100201A
:103F0000A07008E00020A070D4F8210018B1D4F807
:103F100021103046884700BFDCE70000CB2400209A
:103F20002DE9FE4104460B460020009001900290CE
:103F300000271E460021002507E0605C00F00F0806
:103F400028466D1C0DF80080491CB142F5DB0020AD
:103F5000E054002110E01DF80100000701F1010C00
:103F60001DF80CC04CEA1060BC4607F1010808F0CF
:103F7000FF0702F80C00891CA942ECDB0020D0549A
:103F8000BDE8FE810148006870470000680200201B
:103F900002480068401C0149086070476802002020
:103FA00070B5002526E005EB4500144901EB4004FF
:103FB0002078E8B16088401C80B26080A188884287
:103FC00016DB15B1012D10D10BE000210C48FBF7D9
:103FD00003F80C48807818B94FF480700A4948619A
:103FE00003E001200849486100BF00BF00202070A5
:103FF000681CC5B2022DD6DB70BD00008E270020E4
:10400000000C0040D00700200010014010B502460F
:10401000022A00DB10BD02EB4203054C04EB430017
:104020000023438081800123037000BFF2E700007A
:104030008E27002000B50146FFF7A4FF0A689042D2
:1040400001D9012000BD0020FCE770B50446FFF750
:1040500099FF051901E0F3F70BFCFFF793FFA84266
:10406000F9D370BD00B50246FFF78CFF084410601D
:1040700000BD000010B50248F8F7CCF910BD0000F3
:1040800046020020312E312E312E31000B0F0A0551
:10409000021907051119010505000A000F001E008D
:1040A0003C0078002C01000068596364C8CCAAA7C2
:1040B000A2ABA56E6A568A57F4BBFEFA26212D29BB
:1040C0000D093E3A37320A07F7F2FBF5FFF61C18E6
:1040D0001314F1FDF90C9F089A97929B959F121B60
:1040E000152C2823F92A2722242E67252F98FC75C2
:1040F000F8F33C3833340304050F06017A77726213
:104100006B83848EC4CB8782353F364F3D399C9874
:104110009394424F4641818D4D49717D7996919D91
:1041200099C3C41DCECA7F767C7873747E7B751E5E
:104130001A171F16111D47195DC7C2CBC5CFD1DD98
:10414000D94C48C6C1CD61C9D78CFD88A1ADA9B1F4
:10415000BDB98B858F4B4586DCD8D3D4DED2DBD579
:10416000DFD643444E4AE747ACA8A3A4AEBA0DB786
:10417000B2AFA6E4EEEAE7E2E1ED0FE966616D6950
:10418000BBB5BFB6ECE80BE3525C656F5853540CFB
:104190005E5B555F312F9A0B0B5A2B9E0289593B60
:1041A0000E516CEBDAE631F6F0550108EC550108DA
:1041B0000C5601080856010804560108005601086B
:1041C000DC550108D4550108FC550108F4550108D7
:1041D000E45501081056010814560108D05501088D
:1041E0000D0A0000000000000000000000000000B8
:1041F00000000000000000000000000000000000BF
:1042000000000000000000000000000000000000AE
:10421000000000000000000000000000000000009E
:10422000000000000000000000000000000000008E
:104230003F20303132333435363738396162636488
:1042400065666768696A6B6C6D6E6F7071727374A6
:1042500075767778797A4142434445464748494ADA
:104260004B4C4D4E4F505152535455565758595A26
:104270002C2E2F3B275C5B5D2D3D607E214023244F
:10428000255E262A28295F2B7B7D3A227C3C3E0036
:104290000000003C424262020408080018180000B6
:1042A000000000000000000000000000000000000E
:1042B00000000018244242424242424224180000B8
:1042C000000000107010101010101010107C000072
:1042D0000000003C4242420404081020427E0000DC
:1042E0000000003C4242041804020242443800002C
:1042F000000000040C14242444447E04041E000026
:104300000000007E404040586402024244380000F1
:104310000000001C2440405864424242241800001F
:104320000000007E44440808101010101010000017
:104330000000003C4242422418244242423C000019
:104340000000001824424242261A020224380000CB
:10435000000000000000003C421E2242423F0000DC
:10436000000000C04040405864424242645800008F
:10437000000000000000001C22404040221C000001
:10438000000000060202021E22424242261B0000DA
:10439000000000000000003C427E4040423C000023
:1043A0000000000F1110107E10101010107C000083
:1043B000000000000000003E444438403C42423CC3
:1043C000000000C04040405C6242424242E70000C0
:1043D000000000303000007010101010107C000041
:1043E0000000000C0C00001C0404040404044478C5
:1043F000000000C04040404E4850684844EE000075
:10440000000000701010101010101010107C000030
:1044100000000000000000FE4949494949ED000044
:1044200000000000000000DC6242424242E700005F
:10443000000000000000003C42424242423C0000BA
:1044400000000000000000D864424242447840E08E
:10445000000000000000001E22424242221E02070D
:1044600000000000000000EE3220202020F80000B4
:10447000000000000000003E42403C02427C000080
:10448000000000000010107C10101010100C000034
:1044900000000000000000C642424242463B0000CD
:1044A00000000000000000E7422424281010000053
:1044B00000000000000000D79292AAAA4444000025
:1044C000000000000000006E241818182476000078
:1044D00000000000000000E742242428181010E02B
:1044E000000000000000007E44081010227E000042
:1044F0000000001010182828243C444242E7000025
:10450000000000F8444444784442424244F8000029
:104510000000003E4242808080808042443800009B
:10452000000000F8444242424242424244F8000045
:10453000000000FC424848784848404242FC0000E5
:10454000000000FC424848784848404040E00000F5
:104550000000003C44448080808E84444438000045
:10456000000000E7424242427E42424242E70000EF
:104570000000007C1010101010101010107C0000B3
:104580000000003E0808080808080808080888F025
:10459000000000EE444850705048484444EE00008B
:1045A000000000E0404040404040404042FE0000EB
:1045B000000000EE6C6C6C6C5454545454D60000E3
:1045C000000000C7626252524A4A4A4646E2000070
:1045D0000000003844828282828282824438000055
:1045E000000000FC424242427C40404040E000006B
:1045F00000000038448282828282B2CA4C380600AF
:10460000000000FC4242427C4848444442E300002F
:104610000000003E4242402018040242427C00005A
:10462000000000FE92101010101010101038000042
:10463000000000E74242424242424242423C000005
:10464000000000E7424244242428281810100000EB
:10465000000000D692929292AAAA6C4444440000B0
:10466000000000E7422424181818242442E7000020
:10467000000000EE444428281010101010380000EC
:104680000000007E840408081020204242FC000044
:10469000000000000000000000000000606020C07A
:1046A000000000000000000000000000606000004A
:1046B00000000102020404080810102020404000FD
:1046C000000000000000001000000000001010209A
:1046D00000606020C000000000000000000000003A
:1046E00000004040202010101008080404040202BA
:1046F000001E1010101010101010101010101E00BE
:104700000078080808080808080808080808780059
:1047100000000000000000007F000000000000001A
:10472000000000000000FE000000FE00000000008D
:104730000060100000000000000000000000000009
:10474000304C4300000000000000000000000000AA
:1047500000000010101010101010000018180000B9
:1047600000000038445AAAAAAAAAB4424438000059
:10477000000000242424FE484848FE484848000021
:104780000000103854545030181414545438101079
:1047900000000044A4A8A8A8541A2A2A2A44000009
:1047A000001C2200000000000000000000000000CB
:1047B00000000030484848506EA494888976000074
:1047C000000000001010D63838D61010000000008D
:1047D000000204080810101010101008080402004D
:1047E0000040201010080808080808101020400099
:1047F000000000000000000000000000000000FFBA
:104800000000000010101010FE101010100000002A
:10481000000304040404040804040404040403005E
:104820000060101010101008101010101010600010
:104830000000000000001818000000001818000018
:1048400000123624480000000000000000000000B4
:1048500008080808080808080808080808080808D8
:10486000000000020408102040201008040200008C
:10487000000000402010080402040810204000003E
:10488000BFDA00000000003FF820082008200820C0
:104890000820082008200820083FF8200800000011
:1048A0000000007D2829313233343536373839302D
:1048B0002D3A202C6B65793D25782E2100080008C3
:1048C000000800080008000800080008000C0006A6
:1048D000000C000800080008000800080008000894
:1048E0000008003800000000000000000000200068
:1048F0004000800080010001000000020002000270
:10490000000200020002000100010000800080009F
:1049100040002000000000000000000000600030A7
:104920000018000800040004000400040000000255
:104930000002000400040004000400080018001035
:104940000020000000000000000000000000000047
:1049500000020006000E0012000200020002000227
:104960000002000200020002000200020002000039
:104970000000000000000000000000000000000730
:10498000001FC038C0206020600060004000C001EF
:10499000800100030006000C00180030003FE0001A
:1049A0000000000000000000000000000000000700
:1049B000000FC010C030602060004000C0038003C2
:1049C0008000C0006000602060306038C01F80063A
:1049D00000000000000000000000000000000000D7
:1049E000C000C001C003C003C004C00CC008C01098
:1049F000C030C020C07FF07FF000C000C000C00009
:104A000000000000000000000000000000000000A6
:104A1000001FC010001000100030003F8039C0207F
:104A2000400060006000604060604030C01F800E49
:104A30000000000000000000000000000000000175
:104A40008001000300060004000C001F801FC0301E
:104A5000603020203020302030302038601FC007E8
:104A60000000000000000000000000000000000046
:104A7000003FE00020006000400080008001000155
:104A800000030002000600060004000C000C0000F9
:104A9000000000000000000000000000000000070F
:104AA000001F8030C020402060204030C01F801F89
:104AB0008030C0206060206020206030C01FC007B0
:104AC00000000000000000000000000000000007DF
:104AD000001F8030C02060606060606060604030B7
:104AE000C01F80078001000300020006000C0008C0
:104AF00000000000000000000000000000000007AF
:104B0000000F8018C030403060206020202020201E
:104B1000202020202020603060304018C00F800608
:104B20000000000000000000000000000000000085
:104B30000000000000000000000000000000007FF6
:104B4000E000000000000000000000000000000085
:104B50000000000000000000000000000000000055
:104B60000000000000000000000000060006000039
:104B70000000000000000000000000060006000623
:104B80000000000000000000000000000000000025
:104B90000000000000000000000000000000000015
:104BA0000000000000000000000000000000000005
:104BB00000000000000000000000000000000000F5
:104BC00000000000000000000000000000000000E5
:104BD00000000000000000000000001000100010A5
:104BE0000010000000000000000000000000002095
:104BF000002000200020002000200020C021802371
:104C00000026003E0031003180308030C0306030FE
:104C10002000000000000000000000000000000074
:104C200000000000000000000000000F8019C030EC
:104C30004020603FE020002000306018401FC00787
:104C40000000000000000000000000000000000064
:104C50000000000000000000000000206020603024
:104C60004010C01880088009800F00070007000668
:104C70000006001C001800000000000000000000FA
:104C80000000000000000000007FE00000000000C5
:104C90000000007FE07FE000000000000000000056
:104CA00000000000000000000000000000000010F4
:104CB000003840480048804800480048003800124A
:104CC0004000E00520012009200120112000E00023
:104CD0004000000000000000000000000000000094
:104CE0000000000000000000000000306010C0095B
:104CF000800F00070006000F00098018C030402018
:104D00006000000000000000000000000000000043
:104D10000000000000000000000000000000000093
:104D20000000000000000000000000100010001053
:104D30000000000000000000000000000006000667
:104D40000006000600060002000200020002000247
:104D5000000200020002000000000006000600063B
:104D600000000000000000000000000000C9EEDBB1
:104D7000DACAD000000000000000000000000000BF
:104D800000000000000000400010FFF81C00080CAC
:104D900009880010486002007C020000FFFF0182C9
:104DA0003E0002040C326038623030C218218204A6
:104DB00000020000000000000000000000000000F1
:104DC00000000000000000000000000000000210D1
:104DD000180631180211980211181F91182611187F
:104DE00002111802111803F1183F11187C31180034
:104DF000E11803C318018018000000000000000043
:104E000000000000303132333435363738396162D2
:104E1000636465666768696A6B6C6D6E6F707172EA
:104E2000737475767778797A4142434445464748AA
:104E3000494A4B4C4D4E4F5051525354555657586A
:104E4000595A202122232425262728292A2B2C2D94
:104E50002E2F3A3B3C3D3E3F405B5C5D5E5F600019
:104E600000003844444444444438000000001070BA
:104E700010101010101000000000384444081020DA
:104E8000407C00000000384404380404443800002A
:104E9000000018182828487C0808000000007C4002
:104EA000407804044438000000003844407844440A
:104EB0004438000000007C040808081010100000AE
:104EC000000038444438444444380000000038446A
:104ED00044443C04443800000000000038443C4492
:104EE000443C0000000040407844444444780000C2
:104EF0000000000038444040443800000000040432
:104F00003C444444443C00000000000038447C40E1
:104F100044380000000030207020202020200000B5
:104F2000000000003C4444443C044438000040403D
:104F30007844444444440000000010001010101055
:104F400010100000000010001010101010101020A1
:104F500000004040485060605048000000001010C1
:104F6000101010101010000000000000685454547D
:104F700054540000000000007844444444440000BD
:104F800000000000384444444438000000000000A1
:104F90007844444444784040000000003C44444489
:104FA000443C0404000000003820202020200000A1
:104FB0000000000038443008443800000000202081
:104FC00070202020203000000000000044444444B1
:104FD000443800000000000044442828101000005D
:104FE0000000000054545454282800000000000021
:104FF00044281010284400000000000044444428C5
:105000002810106000000000780810204078000090
:10501000000010102828287C444400000000784438
:105020004478444444780000000038444040404004
:10503000443800000000784444444444447800006C
:1050400000007C40407C4040407C000000007C40F0
:10505000407840404040000000003844405C4444F8
:105060004C34000000004444447C44444444000068
:1050700000001010101010101010000000000808A0
:105080000808084848300000000044485060504874
:10509000444400000000404040404040407C00004C
:1050A000000044446C6C54545444000000004464B8
:1050B0006454544C4C44000000003844444444447C
:1050C00044380000000078444444784040400000E8
:1050D00000003844444444544C38040000007844F0
:1050E00044447844444400000000384440300804FC
:1050F0004438000000007C10101010101010000048
:105100000000444444444444443800000000444403
:1051100044282828101000000000545454545428E7
:1051200028280000000044442810102844440000AF
:1051300000004444282810101010000000007C08D3
:1051400008101020207C000000000000000000007B
:1051500000000000000010101010101000100000DF
:10516000000028280000000000000000000028289F
:105170007C28287C2828000000103854503018144F
:1051800054381000000020545830285454080000AF
:1051900000003048483054484834000000001010E7
:1051A0000000000000000000000810102020202057
:1051B0001010080000201010080808081010200027
:1051C0000000000010107C1028000000000000000B
:1051D00010107C1010000000000000000000000013
:1051E000001010200000000000007C000000000003
:1051F000000000000000000000101000000404087F
:1052000008101020204040000000000010000000A6
:10521000100000000000000010000000102000003E
:10522000000000000C3040300C00000000000000C6
:10523000007C007C000000000000000060180418E2
:105240006000000000003844040810100010000046
:10525000000038444C5454545C403800001810107E
:10526000101010101010180000005454FC54542852
:1052700028280000003010101010101010103000FE
:1052800000001028440000000000000000000000A2
:105290000000000000007C00000010100000000072
:1052A000000000008000000000000000000000007E
:1052B00000000000000000000000000000000000EE
:1052C00000000000000000000000000000000000DE
:1052D00000000000000000000000000000000000CE
:1052E00000000000004040404040404040404141FC
:1052F00041414140404040404040404040404040AB
:105300004040404040050202020202020202020244
:105310000202020202202020202020202020200241
:1053200002020202020290909090909010101010D1
:10533000101010101010101010101010101010106D
:105340000202020202028888888888880808080801
:1053500008080808080808080808080808080808CD
:105360000202020240000000E552010820324720FC
:1053700000000000203347200000000020344720B8
:10538000000000004155544F284C54452C574344CD
:105390004D4129004155544F284C544529000000E7
:1053A0004155544F285743444D412C4C54452900F6
:1053B0004155544F285444532C4C54452900000067
:1053C0004155544F202854454C45434F4D2900002A
:1053D0004155544F285743444D412C47534D2900C4
:1053E0004155544F28484452290000004155544F1C
:1053F000285444532900000041504E310000000061
:1054000041504E320000000041504E330000000079
:1054100041504E34000000005444532047534D2067
:105420005743444D41000000544453205743444DDA
:1054300041000000544453205743444D41204C54F4
:105440004500000043444D4120484452204C5445FF
:105450000000000043444D4120484452205743443B
:105460004D412047534D000043444D4120414E449F
:105470002047534D0000000043444D412048445212
:10548000000000004C544520414E44205444530039
:105490004C5445205743444D41204F4E4C59000039
:1054A00043444D41204F4E4C590000004C54452080
:1054B0004F4E4C59000000005743444D4120475384
:1054C0004D204F4E4C5900004C54452047534D2021
:1054D0004F4E4C5900000000484452204F4E4C594A
:1054E00000000000544453204F4E4C59000000006F
:1054F000554D5453204F4E4C590000004175746F68
:105500000000000041504E312E626D70000000001E
:1055100041504E2E626D700053657273656C2E6241
:105520006D7000005365722E626D7000B5CDB9A626
:10553000BAC4C4A3CABD0000CAD2C4DAC4A3CABDD7
:1055400000000000CAD2CDE2C4A3CABD0000000022
:10555000B3A3B9E6C4A3CABD00000000B3ACB3A4B2
:10556000B9A6BAC4000000004950B7D6B7A2B7FE2A
:10557000CEF1C6F700000000C9BDB6ABB7FECEF154
:10558000C6F70000BCAFC8BAB7FECEF1C6F7000040
:10559000BABCD6DDB7FECEF1C6F70000D7D4B6A8A8
:1055A000D2E5B7FECEF1C6F7000000004D61696C90
:1055B000312E626D700000004D61696C322E626D9B
:1055C00070000000B8F1CABDBBAF0000C9BEB3FD9A
:1055D0000000000052414343000000005341434398
:1055E00000000000525245430000000054470000F4
:1055F000544D00005241504E0000000041504E00FA
:105600005247500053475000524D5000534D5000E8
:10561000564552004241540070656F706C65312EE2
:10562000626D700047726F7570312E626D70000090
:1056300070656F706C65322E626D700047726F75A9
:1056400070322E626D700000D6D5B6CBD0C5CFA219
:1056500000000000CEC4B1BECFFBCFA2000000000E
:10566000392EB6D4BDB2B0E6B1BEC9FDBCB600009D
:10567000362EB3A1BEB0C4A3CABD000031302EB1D6
:10568000B8D3C300322E4C4344C9E8D6C30000004F
:10569000312E41504EC9E8D6C3000000CFB5CDB37E
:1056A000C9E8D6C300000000B1B1B6B7C9E8D6C397
:1056B00000000000382EC4A3CABDC9E8D6C300004C
:1056C000332ECDF8C2E7C9E8D6C30000352ECCE1B1
:1056D000CABED2F4C9E8D6C300000000372EB1E03C
:1056E000C2EBC6F7C9E8D6C300000000342EB7FEEF
:1056F000CEF1C6F7C9E8D6C300000000B3C9D4B1E3
:10570000D1A1D4F100000000C8BAD7E9D1A1D4F1E9
:10571000000000003457010800000020BC03000016
:105720000449000878580108BC030020EC49000037
:10573000E01C0108412D010203040450090607087A
:105740000902040608846CDC02691C013F6BFFFF40
:1057500005F1F2012F3530323830302C892EE92412
:10576000180AFC5401086C53010874041A7C0441A3
:105770002AF80819181A08041A10041BD055081919
:10578000041A0404290C011C29201AF0341A944428
:105790001A68081AEC081AAC081AE4041A28041A41
:1057A00018041A34041AD8041AC01C1AE0041A4443
:1057B0000C1A78041AA0041AB0101A84041AD0041F
:1057C0001AA0041A90141AB8041A84041AC8041AE5
:1057D00054041ACC04411A2C6C1A5C045A50981ABE
:1057E00038049A44A41A24085A18101A90041A78F3
:1057F000041A68041A84040A1D9CCC12012202199E
:1058000003C11AAC309AB8381ACC080A11C4488BB4
:10581000E7030409165E014CF21E1AFF01697B09B9
:10582000426A2950091B20992429051E9056010817
:1058300084041AC0041AEC041ACC041A70041ADC8A
:10584000041AB4041A60041A7C047DD0550108417E
:10585000B11A241C9A3C201A300C2904AA1834B11D
:105860001E08570108FC1C1A54041A9C041AA804A8
:085870009A482C021F01000000
:04000005080041515D
:00000001FF
